:020000040800F2
:10000000002000100151030895430308B53700088C
:1000100093430308914303088F4303080000000043
:100020000000000000000000000000008D430308F5
:100030008B4303080000000089430308E92C0008F3
:10004000695103086951030869510308695103089C
:1000500069510308695103083938000865390008F7
:1000600029390008ED380008B1380008017E000881
:10007000F17D0008E17D0008D17D0008C17D000808
:10008000AD7D0008997D0008695103086951030896
:10009000F5430308695103086951030875380008DE
:1000A000191E0008BD2200084D1D00083924000853
:1000B00001220008452100087D200008695103083D
:1000C000695103086951030869510308695103081C
:1000D00069510308152E0008992D00081D2D0008F0
:1000E000FD37000869510308794303086951030883
:1000F000E51E000869510308B11F00086951030893
:10010000000000000000000000000000695103082A
:1001100069510308695103084501020829010208D1
:10012000857D0008717D00085D7D0008497D00081F
:10013000357D000869510308000000000000000040
:100140006951030869510308695103080000000060
:10015000000000000000000000000000000000009F
:100160000000000000000000695103086951030805
:1001700069510308000000000000000000000000BA
:080180000000000069510308B2
:1001880038B50B4C23688BB15A68821A002A054689
:1001980004DA0BE05A68AA1A002A07DB9A68226078
:1001A80018461A6890472368002BF3D138BD00BF62
:1001B8000C2C0020436A8269D154436A0169826B1E
:1001C80001338B4228BF002343623AB370B4EFF384
:1001D8001183502282F31288866B3268D20704D5C5
:1001E800DBB283F3118870BC7047716869B9D0E9D4
:1001F8000942944218D085691544F56018D9A21AA5
:1002080072608462002280F85420326842F0010251
:10021800DBB2326083F3118870BC7047026D1368DB
:1002280043F0800313607047012280F85420D7E719
:100238000469A21A72608162E4E700BF034610B441
:10024800446BD968406954B15A6C8C1A013A005D04
:100258005DF8044B08BF0A46C0B25A6470471A6A70
:10026800805C01328A4228BF2246C0B21A625DF819
:10027800044B7047836B13B190F854007047D0E972
:100288000903181AB0FA80F040097047D0E909123A
:100298000369914238BFC9188A1A816B013B19B1A9
:1002A80049680A449A4201D2981A70470020704758
:1002B800436B43B1426C5B689A4291BF981AC0681D
:1002C8009B1AC0187047D0E907239A422FBFD01A4B
:1002D800C0688018C01A70470A4B30B503F114047F
:1002E80093F900205D78072AC8BF143A81180433AF
:1002F8000D7313F8025C855413F8012C0A769C429E
:10030800EED130BDE056030803682DE9F041DD6900
:100318001DB12B46BDE8F0411847002A174611DDEC
:1003280004460E460F4400E023689B682046984721
:100338000028F9D0236816F8011B1B682046984747
:10034800BE42F1D1BDE8F081002303704370837091
:10035800C37070470028F0B403DA2D230B704042B5
:100368000131092804464FF0010307DD03EB83033D
:100378005B00B0FBF3F2092AF8D883B10F48A0FB61
:100388000326B4FBF3F2092A02F1570C02F13007F5
:1003980009DD03FB1244F30801F801CBEFD1002378
:1003A8000B70F0BC704703FB1244F30801F8017BA3
:1003B800E5D100230B70F0BC704700BFCDCCCCCC8E
:1003C800884270B44FF0010442D301FB04F4B0FB3F
:1003D800F4F58D42F9D2ECB142BB092D04FB1500AE
:1003E80005F1570605F130020EDDB4FBF1F403F810
:1003F800016B7CB1B0FBF4F5092D04FB150005F188
:10040800570605F13002F0DCB4FBF1F403F8012BD8
:10041800002CEFD100221A7070BC704703F8016BF2
:10042800B4FBF1F4002CF5D0B0FBF4F5092D04FB76
:10043800150005F1370605F13002EFDCB4FBF1F4E5
:1004480003F8012B002CEFD100221A7070BC704702
:100458000546002AEAD1C0E72DE9F04714461D46B3
:10046800064600234FF47A722046294634F078FC79
:10047800DFF848814B4A4C4F88FB00310144C317D1
:1004880082FB002CC3EB611188FB012887FB002746
:100498008444464AC3EBEC2CC1EB011E82FB0C29B9
:1004A800A0EB8E0E0744424A86F806E0C3EB2747C6
:1004B8004FEAEC7E08EB010ACEEBA90E82FB07821D
:1004C8004FEAE1780EEB4E0EC8EB6A18ACEBCE0C97
:1004D800C8EB0818DFF8E8E086F804C0A1EB88014B
:1004E80071718EFB0010F917C1EBE21240F2B551A1
:1004F80001FB1272C3EBE050B2F5896F4FEA800737
:100508003FDA40F2DA239A4243DCB2F5B77FB4BF50
:100518004FF0000E4FF0010E4FEA4E08254B08EB46
:100528000E0103EBC1031FFA8EFC588D224908EB1C
:100538000E0301EBC30116310B2301E031F8020D64
:1005480090421BDD013BF9D11A4BC64403EBCE0E9A
:100558000123BEF81400B37007F2B2770132121A01
:10056800BC44F270A6F800C0204629464FF47A72BF
:10057800002334F0F5FB3281BDE8F0870133DBB2AC
:10058800E9E74FF0030CE64640F296504FF00608B4
:10059800CCE74FF0020CE64640F229404FF0040841
:1005A800C4E700BFC5B3A29107452EC2ABAAAA2AC9
:1005B80073B06D16E0560308F456030889888888D6
:1005C800792D031103685A1C02601970704700BF27
:1005D8002DE9F047089C2578002B804689460CBFFA
:1005E8004FF0200A4FF0300A661C25B3002A26DD9A
:1005F800334601E0024698B113F8011B501E00294A
:10060800F8D1971E60B13D46013D51464046C84766
:100618006B1C002BF8DC257827EAE770013045B120
:10062800041B29464046C847301916F8015B002DBF
:10063800F7D1BDE8F087002A03DC2846F9E7002057
:10064800EEE7571EDFE700BF90ED057A90ED004A10
:10065800D0ED066AD0ED014AD0ED047A90ED035A48
:10066800D0ED025AA4EE007AB0EE406AB0EE470A26
:10067800B0EE667AA4EE867A67EEC07AA5EE407A86
:10068800E5EE867A80ED057AC0ED067A704700BF00
:10069800D0ED057A90ED013AD0ED003AD0ED064A5A
:1006A80090ED024A90ED077A90ED035A90ED086AB2
:1006B800D0ED045AC0ED067AF0EE406A27EE830AC0
:1006C800C0ED056AA3EEA60A80ED087AA4EE240A16
:1006D800A5EE470AA5EEC60A80ED070A704700BFD7
:1006E800D0ED007A90ED017A30EE670AE7EE007AF5
:1006F800B0EE670AC0ED007A704700BF704700BFD0
:100708000A44914215D030B40139551E41F22102F4
:1007180011F8014F082380EA042004044CBF82EA40
:1007280040004000013B80B2F7D18D42F0D130BC8F
:1007380070477047831E00F15002EA2123F8021F18
:100748009342FBD140F649134385CD2383804E2342
:10075800C380CE230381012380F8603080F86130A4
:1007680080F8623080F8633080F8643080F8663052
:1007780080F86B3080F8693080F85730142380F89F
:10078800563040F69803A0F852306423A0F854304D
:100798004FF42063A0F8583040F60123A0F85A30EF
:1007A8004FF6FF730022A0F85C3042F6140380F87D
:1007B800652080F8672080F86A2080F8682080F833
:1007C8006C20A0F85E307047054B93F857302BB972
:1007D8004FF4A4735843642390FBF3F0704700BFB1
:1007E800462700200E4B1B78022B17D00D4A537852
:1007F800127803EB83035B00C01A02EB8202C3EB9F
:100808004203C0EBC00090FBF3F00628A8BF062007
:1008180020EAE070C0F19600C0B270479720704798
:10082800813F0020843F00204FF48053838270472B
:10083800012380F85430704770B4D0E90041057B3B
:1008480002690223AB4063600B684FF6FE700340F9
:100858000B60EFF31183502181F31288966B316896
:10086800C9071CD4706870B9D2E909418C4213D009
:1008780095690D44F56017D81469611A7160906222
:10088800002182F85410326842F00102DBB2326073
:1008980083F3118870BC7047012182F85410DBB2D1
:1008A80083F3118870BC7047611A71609462E7E73E
:1008B80070B40468037B2268022101FA03F31A4228
:1008C80017D002691249134802EB420201EB4212A7
:1008D80005785068016875B9C568528928684FF667
:1008E800FE7630402860C868D24392B20240CA609F
:1008F800636070BC7047406902684FF6FE752A4015
:100908000260CA684FF6FF600240CA60F0E700BFA5
:10091800C86D0020C46D002070B4174B1D784DB30E
:10092800164A174B11784FF4987202FB053540F2BE
:100938000D3610E058681C894460046844F00104CE
:100948000460A2F84860D06803F5987340F480709A
:10095800AB42D0600ED01A680029EBD15162B3F8CF
:100968002C01D4682043D06003F5987323F8041C45
:10097800AB42F0D170BC7047C8700020C46D002035
:10098800CC70002010B40268047B11680223A340D5
:10099800194209D00649406800240C7001684FF6D6
:1009A800FE742140016053605DF8044B704700BF3E
:1009B800934000202DE9F0478C4A8D4B12781C7823
:1009C800D207064648D58B4D012C00F091801ED3E6
:1009D800022C40F09B808849884A09881288884FF1
:1009E800914201D901241C70EB7AFBB12B89EBB140
:1009F800844B1B78D3B11FF0DBFB002800F0E280AA
:100A08002B7B83422CBF012300233B700FE0DFF8D0
:100A1800E8C17B4F7C4CBCF800002288697B521AE5
:100A28008242DFDAEB7A0024002BDFD13B782A7987
:100A3800632A07D87549022C087800F0B880002886
:100A480040F0A0807249AA7A9C4238BF1C460C70BC
:100A5800002A44D1BDE8F087DFF89CC1654DBCF899
:100A68000000BCF8021095F803E06A4F411A00290B
:100A7800A4F10302B8BF4942704597F80080D2B28A
:100A880011D32F7887420ED3012A45D9B8F1020F26
:100A98009AD15C48604A007890800229CCBF002136
:100AA8000121D18090E7B0EB4E0FEDDC012A40F236
:100AB8008C800229EADC0324514F524852494F4A9C
:100AC8001C70B8F1020F4FF000033C7003700B80EC
:100AD800138089D1504A01219380D18084E7012C69
:100AE8006BD0022CB6D10720BDE8F04720F0C2BB7E
:100AF800424A41491288687B0988121A914207DDE7
:100B0800414A12888A423CBF00241C703C4F6BE764
:100B180002241C703A4F67E70229B7DC95F800E019
:100B280090FBFEFE0EF1010EBEF1080FDFF8D4A017
:100B3800AA786978DFF8C490334C314FA8BF4FF0DA
:100B4800080E8AF800E01FFA8EFA11FB0AF112FB70
:100B58000AF2DFF8B8A0A9F8001092B200214FF00D
:100B68006409B8F1020F228039701970CAF80410AC
:100B78008AF801907FF452AF274A0121A2F804E0D5
:100B8800D18048E74868301A244EB042C8BF4A703E
:100B98003FF758AFC2F16402214E00FB02F086FB1A
:100BA8000062C017A0EBA250643048704AE70028E2
:100BB800E8D101274E600F70ECE70820BDE8F04748
:100BC80020F058BB02233B7031E7032C7FF471AF50
:100BD800B8F1020F9AD10B4A0F4B12789A8002296A
:100BE800CCBF00210121D980054FFDE6643F0020DC
:100BF800784A0020843F00208C4000207C4A002056
:100C0800884A0020444300207A4A0020804A002075
:100C1800813F0020603D0020643D00207F969800C1
:100C28006BCA5F6B2DE9F04F013083B0C3B20193FB
:100C3800884C894E894DDFF838820A239B462FF06D
:100C48006FFCDFF820C24FF4FA7A4FF0100E4FF421
:100C58007A77DCF80430C3F30803002B40F0DD801A
:100C6800EFF31183002B40F0D8802168AA6800BFF9
:100C780023689942F9D1306807FB00F39A1AB2FB4E
:100C8800F0F207FB0121DCF80430C3F30803002B62
:100C980040F08880EFF31183002B40F083802368B5
:100CA800A86800BF22689342F9D1D6F8009007FBE4
:100CB80009F2101AB0FBF9F007FB03035B1AB3F54E
:100CC8007A7FE0D3BAF1010AC3D101982FF08EFAE6
:100CD8004FF47A7ADFF88CC157464FF0100EDCF8E3
:100CE8000430C3F30803002B7BD1EFF31183002BEF
:100CF80077D12168AA6800BF23689942F9D1306882
:100D080007FB00F39A1AB2FBF0F207FB0121DCF8AB
:100D18000430C3F3080333BBEFF311831BBB236811
:100D2800A86800BF22689342F9D1D6F8009007FB63
:100D380009F2101AB0FBF9F007FB03035B1AB3F5CD
:100D48007A7FE4D3BAF1010AC9D15B46013B9B46DD
:100D58007FF475AF4249434B4348444A0860DA6020
:100D680003B0BDE8F08FEFF311808EF31288D5F849
:100D780008902B68DB0304D50123C8F80030D5F8A8
:100D880008902368D8F80020C0B280F31188306832
:100D9800134407FB00F2A2EB0902B2FBF0F207FBD7
:100DA8000323CBE7EFF311808EF31288D5F8089070
:100DB8002B68DB0304D50123C8F80030D5F8089068
:100DC8002368D8F80020C0B280F311883068134433
:100DD80007FB00F2A2EB0902B2FBF0F207FB0323C8
:100DE8006CE7EFF311828EF31288A8682B68D90399
:100DF80003D50123C8F80030A8682368D8F8001084
:100E0800D2B282F311883268194407FB02F31B1A25
:100E1800B3FBF2F307FB013179E7EFF311828EF3AD
:100E28001288A8682B68D90303D50123C8F80030B5
:100E3800A8682368D8F80010D2B282F31188326803
:100E4800194407FB02F31B1AB3FBF2F307FB01314A
:100E580019E700BF58600020BC60002010E000E0E7
:100E6800FC9F002000ED00E0EFBEADDE0400FA05B7
:100E7800B860002030B50446006D61710368A2684F
:100E880023F00103036087B0A379009213F0040FE5
:100E98004FEA03324FEA032314BF4FF4805500256D
:100EA80003F4806302F400520195CDE90223002582
:100EB80011F0010305952ED1049308238D07694687
:100EC80048BF04931AF0BCFC6079236DA17900F047
:100ED8000202002A15BF4FF440324FF480324FF41B
:100EE8000034002410F0010F586808BF2246CC07D0
:100EF8004CBF024320EA02025A609A6809074CBFB5
:100F080042F0080222F008029A601A6842F00102D0
:100F18001A6007B030BD042304930C23CEE700BF4A
:100F280030B50446006DA160036823F00103036037
:100F3800A379657987B013F0040F4FEA03324FEABB
:100F4800032303F4806302F40052CDE902230091E5
:100F580014BF4FF480510021EB0748BF04230191CF
:100F68004FF00001CDE9041154BF082304936946EA
:100F780048BF0C23AD0748BF04931AF061FC6079A1
:100F8800236DA17900F00202002A15BF4FF4403208
:100F98004FF480324FF40034002410F0010F5868E9
:100FA80008BF2246CC074CBF024320EA02025A601F
:100FB8009A6809074CBF42F0080222F008029A60BA
:100FC8001A6842F001021A6007B030BD2DE9F341FA
:100FD800056906460F467DBBD0F80080C8F30A03B2
:100FE80023B30023D6F80080019330F09BFB04283C
:100FF80019D1224C236943F001032361BBB2A8F83D
:10100800003030F08FFB04282ED108F10203019341
:10101800019B3F0C1F8030F085FB2369042823F0D7
:101028000103236125D06FF0010505E030F07AFB5C
:10103800042805D04FF0FF35284602B0BDE8F081FE
:101048000E4C236943F002032361C4F8148023691A
:1010580043F04003236130F065FB2369042823F043
:1010680002032361BDD0E5E7236923F0010323616F
:10107800D9E7336804333360DEE700BF002002405D
:10108800F8B504460D468E180027B54201D12069EF
:10109800F8BDE368591CE160234415F8012B1A7266
:1010A8000429F2D1A1682046FFF790FFC4E9037034
:1010B800EBE700BF022828BF022010B4084C094BF8
:1010C800207000EB8002C0EBC20207495DF8044BB8
:1010D800013003EB4203C0B20B6020F009B900BF36
:1010E800EC970020242800209043002038B5434B7B
:1010F8009A89D989914224BF00229A81598A1A8AE9
:10110800914224BF00221A82DA788AB3072A2FD0A4
:101118003B493C4D91F85C00012400210A282C70C1
:101128009C70D9713DD00C2865D0DFED377A8ABB29
:10113800364C9FED370AA278002918BFF0EE407AA6
:10114800062A04D8334901EB820191ED1D0A217961
:1011580059B3013A032A0AD8F7EE007A87EE800AD3
:1011680034F06EFA2388984228BF1846208038BD8C
:10117800D97921B198780428B8BF042098702048FC
:1011880090F85C000A280CD00C28CED1DFED227A2A
:10119800002ACDD0072ACBD00A282CD1DFED1F7A20
:1011A800C6E70A20DFED1E7AC1E79B78154907EEEE
:1011B800103A0A78B8EEC77A67EE277A07EE102A4F
:1011C800B8EEC77A27EE277AB4EEC70AF1EE10FA1E
:1011D800CDDD80EE277AFDEEC77A17EE903A102B18
:1011E800A8BF1023012BB8BF0123DBB29A4238BF36
:1011F8001A460A7038BDDFED0B7A99E7A067002020
:10120800D0670020503300206F120339A06D0020F2
:101218006F120338E05603080AD7A3390F506E3A05
:101228005304E9386F12833A38B50C4C0C4DAC4274
:1012380006D26168204614341FF0BEF9AC42F8D3D8
:10124800084A094B094C1460002209491A705A705F
:1012580008480860BDE838401CF004BA6CBB0308B5
:101268001CC0030890430020EC970020242800208D
:101278009443002034290020F0B40C292BD8DFE84F
:1012880001F0752A2A2A502A2A2A2C2A2A2A0700F3
:10129800046AB2F80CC0978816686B4D24F4805421
:1012A8000462036A4468C16923F4005343EA0C33B7
:1012B80021F4E641A84243EA073341EA062100F057
:1012C800BC8005F50065A84200F0B78092684460CC
:1012D800C16102640362F0BC7047046AB2F80CC0D2
:1012E80097881668584D24F480740462036A446829
:1012F800C16923F4007343EA0C2321F07301A84267
:1013080043EA072341EA060100F0848005F50065F9
:10131800A8427FD092684460C161F0BCC263036296
:101328007047046AB2F80CC097881668464D24F0D6
:1013380010040462036A4468816923F0200321F0E1
:10134800807143EA0C1321F4E641A84243EA0713EB
:1013580041EA06214BD005F50065A84247D09268BE
:1013680044608161F0BC826303627047046A9389B8
:10137800B2F804C01768344E24F001040462046A09
:101388004568816921F4803124F0020443EA0C03A2
:1013980021F07301B04243EA040341EA07010ED089
:1013A8002A4CA0420BD004F54064A04207D004F5B3
:1013B8008064A04203D004F58064A04210D1D4898F
:1013C800168A578AB2F806C023F00803234325F487
:1013D800407523F0040346EA07044CEA0303254357
:1013E800926845608161F0BC426303627047D589A9
:1013F800178AD68823F0800343EA051324F440644F
:10140800558A23F0400344EA870443EA061344EA72
:101418008504A4E7D589178AD68823F4006343EAAC
:10142800052324F44054558A23F4806344EA0714BE
:1014380043EA062344EA05146CE7158A24F4804439
:1014480044EA851442E700BF002C01400034014003
:101458002DE9F84F4FF4A0720021DFF818827B487D
:101468007B4C7C4E7C4FDFF81092DFF810A234F0F2
:1014780033F87A497A48DFF808C2DFF808E208F555
:101488008C7245462B688B4200F0B780B3F1804FD1
:1014980000F0BA80A34200F0BE80B34200F0C980D9
:1014A800BB4200F0C880634500F0C780734500F078
:1014B8009D804B4500F0C380534500F0C380DFF8A2
:1014C800C8B15B4508BF4FF4802B00F091801C35F4
:1014D800AA42D7D1634F644E4FF0030A4FF0020976
:1014E80098F80630002B7AD098F804301C09013C93
:1014F800052C03F00F0372D837F8140040FA03F2F2
:10150800D2076CD54FF0010B0BFA03F3013B1840DF
:1015180033F076FC554B1B5D184416EBC0045ED0C7
:1015280056F83030524898F8081003F13842920AB9
:10153800825C02F01F005209022A0BFA00FB72D0EB
:10154800032A6AD0012A04D1454842694BEA0202BB
:101558004261B4F804C0BCFA8CF2C2F11F0292B224
:10156800D00803EB800002F00702046A92004FF0F3
:101578000F0E0EFA02FE24EA0E040462046A01FA4F
:1015880002F2224302624FF0010E00220EFA02F428
:1015980034EA0C0120D15000D3F808B00AFA00F15F
:1015A800C9430BEA010BC3F808B0D3F808B0C3F875
:1015B80008B0B3F804B02BEA04049C809C88A4B259
:1015C8009C801C680C401C601C6809FA00F02043D1
:1015D8001860D8680140D9600132102AD6D108F1C4
:1015E8001C0845457FF47CAFBDE8F88F4FF4005BDD
:1015F800836943EA0B03836169E783694FF4006BEE
:1016080043EA0B03836162E70123D0F81CB043EA85
:101618000B03C3615BE70223F7E71148C2694BEA92
:101628000202C26195E70E4882694BEA02028261B2
:101638008FE70423E9E71023E7E72023E5E74FF4E2
:10164800803BD5E74FF4003BD2E700BFC0600020E5
:10165800000400400008004000100040002C014039
:10166800001002403C7D030868660020487D03089E
:10167800EC7B0308F47B0308004001400044014070
:1016880000140040003401400048014000B9704790
:1016980003682DE9F04F03F138449C4EA40A012554
:1016A800345D04F01F066409022C05FA06F500F003
:1016B8007481032C00F06C81012C00F02281808859
:1016C800B0FA80F4C4F11F04A4B2E50803EB850561
:1016D80004F007042E6AA4000F27A74026EA07068D
:1016E8002E622E6A01F00307A2407C1E3243012CB1
:1016F800C1F3810EC1F300182A62C1F3411140F20F
:101708000981C6070BD51A6822F003021A601A6805
:101718003A431A60DA6822F003020A43DA6085075E
:101728000DD51A6822F00C021A601A6842EA87027C
:101738001A60DA6822F00C0242EA8102DA60440791
:101748000DD51A6822F030021A601A6842EA0712A8
:101758001A60DA6822F0300242EA0112DA600207FF
:101768000DD51A6822F0C0021A601A6842EA871278
:101778001A60DA6822F0C00242EA8112DA60C6060C
:101788000DD51A6822F440721A601A6842EA0722D4
:101798001A60DA6822F4407242EA0122DA608506A9
:1017A8000DD51A6822F440621A601A6842EA872244
:1017B8001A60DA6822F4406242EA8122DA6044065A
:1017C8000DD51A6822F440521A601A6842EA0732A4
:1017D8001A60DA6822F4405242EA0132DA600206FC
:1017E8000DD51A6822F440421A601A6842EA873214
:1017F8001A60DA6822F4404242EA8132DA60C605A9
:101808000DD51A6822F440321A601A6842EA074273
:101818001A60DA6822F4403242EA0142DA60850549
:101828000DD51A6822F440221A601A6842EA8742E3
:101838001A60DA6822F4402242EA8142DA604405FA
:101848000DD51A6822F440121A601A6842EA075243
:101858001A60DA6822F4401242EA0152DA6002059C
:101868000DD51A6822F440021A601A6842EA8752B3
:101878001A60DA6822F4400242EA8152DA60C60449
:101888000DD51A6822F040721A601A6842EA076297
:101898001A60DA6822F0407242EA0162DA6085046E
:1018A8000DD51A6822F040621A601A6842EA876207
:1018B8001A60DA6822F0406242EA8162DA6044041F
:1018C8000DD51A6822F040521A601A6842EA077267
:1018D8001A60DA6822F0405242EA0172DA600204C1
:1018E8000DD51A6822F040421A601A6842EA8777D2
:1018F8001F60DA6822F0404242EA8171D960BDE88F
:10190800F08F034C666935436561D8E6EC7B0308C4
:101918000010024000224FF0010C4FF003090CFAAE
:1019280002F636EA00042ED15400D3F808A009FACA
:1019380004F5ED4305EA0A0AC3F808A0D3F808B08D
:101948000EFA04FA4AEA0B0AC3F808A0B3F804A08E
:101958002AEA06069E80B3F804A008FA02F646EAC8
:101968000A06B6B29E801E682E401E60D3F800A0FC
:1019780007FA04F646EA0A061E60DE6801FA04F46D
:1019880035402C43DC600132102AC8D1BDE8F08F05
:10199800044CE6693543E56191E6024CA669354396
:1019A800A5618CE60010024003682DE9F04F03F1B1
:1019B8003845A94EAD0A0124755D05F01F066D096D
:1019C800022D04FA06F400F08D81032D00F08581C4
:1019D800012D00F03B818088B0FA80F4C4F11F0427
:1019E800A4B2E50803EB850504F007042E6AA400F9
:1019F8000F27A74026EA07062E622E6A01F0030782
:101A080002FA04F47A1E3443012AC1F3810EC1F3A9
:101A180000182C62C1F3411140F22281C60700F17F
:101A28000881850700F1F680440700F1E480020789
:101A380000F1D280C60600F1C080850600F1AE80B4
:101A4800440600F19C80020600F18A80C60578D41D
:101A5800850567D4440556D4020545D4C60434D454
:101A6800850423D4440412D4020401D4BDE8F08FC1
:101A78001A6822F040421A601A6842EA87771F60A3
:101A8800DA6822F0404242EA8171D960EEE71A68CA
:101A980022F040521A601A6842EA07721A60DA683D
:101AA80022F0405242EA0172DA60DDE71A6822F059
:101AB80040621A601A6842EA87621A60DA6822F09D
:101AC800406242EA8162DA60CCE71A6822F040722A
:101AD8001A601A6842EA07621A60DA6822F04072ED
:101AE80042EA0162DA60BBE71A6822F440021A602F
:101AF8001A6842EA87521A60DA6822F4400242EA17
:101B08008152DA60AAE71A6822F440121A601A6849
:101B180042EA07521A60DA6822F4401242EA015295
:101B2800DA6099E71A6822F440221A601A6842EAD1
:101B380087421A60DA6822F4402242EA8142DA6077
:101B480088E71A6822F440321A601A6842EA0742A3
:101B58001A60DA6822F4403242EA0142DA6077E732
:101B68001A6822F440421A601A6842EA87321A60F8
:101B7800DA6822F4404242EA8132DA6066E71A689B
:101B880022F440521A601A6842EA07321A60DA6888
:101B980022F4405242EA0132DA6054E71A6822F429
:101BA80040621A601A6842EA87221A60DA6822F4E8
:101BB800406242EA8122DA6042E71A6822F44072FF
:101BC8001A601A6842EA07221A60DA6822F4407238
:101BD80042EA0122DA6030E71A6822F0C0021A608D
:101BE8001A6842EA87121A60DA6822F0C00242EAEA
:101BF8008112DA601EE71A6822F030021A601A6849
:101C080042EA07121A60DA6822F0300242EA011248
:101C1800DA600CE71A6822F00C021A601A6842EAC5
:101C280087021A60DA6822F00C0242EA8102DA605E
:101C3800FAE61A6822F003021A601A683A431A6030
:101C4800DA6822F003020A43DA60EAE6034D6E69B5
:101C580034436C61BFE600BFEC7B03080010024010
:101C680000224FF0010C4FF003090CFA02F636EA95
:101C780000042ED15400D3F808A009FA04F5ED4366
:101C880005EA0A0AC3F808A0D3F808B00EFA04FA5D
:101C98004AEA0B0AC3F808A0B3F804A02AEA060621
:101CA8009E80B3F804A008FA02F646EA0A06B6B21D
:101CB8009E801E682E401E60D3F800A007FA04F626
:101CC80046EA0A061E60DE6801FA04F435402C4331
:101CD800DC600132102AC8D1C8E6054DEE693443EC
:101CE800EC6178E6024DAE693443AC6173E600BF3F
:101CF8000010024010B50409013C052C17D80E4B02
:101D080033F8142000F00F0042FA00F313F0010337
:101D18000FD0012303FA00F00138104033F070F8B7
:101D2800064A074B125D104403EBC00010BD0020AB
:101D380010BD184610BD00BF3C7D0308487D030850
:101D4800686600202DE9F8432F4D2A69EB6812EAEE
:101D5800030826D02D4E4FF00047B8FA88F327FA2B
:101D680003F2D2431B3B2A6108EA0208042B15D868
:101D7800DFE803F0372D23190300D6F83C31002B98
:101D880039D1EB6A1FFA83F9D6F8384134B12368A0
:101D98002046494698476468002CF8D1B8F1000FEE
:101DA800DBD1BDE8F883D6F81801696B036889B2FE
:101DB8009847B8F1000FD0D1F3E7D6F81C01A96B0A
:101DC800036889B29847B8F1000FC6D1E9E7D6F899
:101DD8002001E96B036889B29847B8F1000FBCD1BC
:101DE800DFE7D6F82401296C036889B29847B8F16F
:101DF800000FB2D1D5E703F1FF3900231FFA89F9A3
:101E0800C6F83C31C0E700BF00480140C060002070
:101E18002DE9F8432F4D2A69EB6812EA030826D00A
:101E28002D4E4FF00047B8FA88F327FA03F2D24351
:101E38001B3B2A6108EA0208042B15D8DFE803F0E7
:101E4800372D23190300D6F8EC30002B39D1EB6A73
:101E58001FFA83F9D6F8E84034B12368204649468A
:101E680098476468002CF8D1B8F1000FDBD1BDE8C1
:101E7800F883D6F8C800696B036889B29847B8F147
:101E8800000FD0D1F3E7D6F8CC00A96B036889B26C
:101E98009847B8F1000FC6D1E9E7D6F8D000E96B4A
:101EA800036889B29847B8F1000FBCD1DFE7D6F8CC
:101EB800D400296C036889B29847B8F1000FB2D1F1
:101EC800D5E703F1FF3900231FFA89F9C6F8EC308A
:101ED800C0E700BF00400140C06000202DE9F84382
:101EE8002F4D2A69EB6812EA030826D02D4E4FF0D1
:101EF8000047B8FA88F327FA03F2D2431B3B2A615A
:101F080008EA0208042B15D8DFE803F0372D231957
:101F18000300D6F8C430002B39D1EB6A1FFA83F9D5
:101F2800D6F8C04034B123682046494698476468CB
:101F3800002CF8D1B8F1000FDBD1BDE8F883D6F852
:101F4800A000696B036889B29847B8F1000FD0D137
:101F5800F3E7D6F8A400A96B036889B29847B8F1EB
:101F6800000FC6D1E9E7D6F8A800E96B036889B283
:101F78009847B8F1000FBCD1DFE7D6F8AC00296C60
:101F8800036889B29847B8F1000FB2D1D5E703F1D9
:101F9800FF3900231FFA89F9C6F8C430C0E700BF2B
:101FA80000340140C06000202DE9F8432F4D2A6914
:101FB800EB6812EA030826D02D4E4FF00047B8FA16
:101FC80088F327FA03F2D2431B3B2A6108EA020886
:101FD800042B15D8DFE803F0372D23190300D6F8B2
:101FE800C430002B39D1EB6A1FFA83F9D6F8C04008
:101FF80034B123682046494698476468002CF8D1D4
:10200800B8F1000FDBD1BDE8F883D6F8A000696B02
:10201800036889B29847B8F1000FD0D1F3E7D6F832
:10202800A400A96B036889B29847B8F1000FC6D11C
:10203800E9E7D6F8A800E96B036889B29847B8F1D0
:10204800000FBCD1DFE7D6F8AC00296C036889B271
:102058009847B8F1000FB2D1D5E703F1FF39002353
:102068001FFA89F9C6F8C430C0E700BF0034014040
:10207800C06000202DE9F8432E4D2A69EB6812EA6A
:10208800030826D02C4E4FF00047B8FA88F327FAF9
:1020980003F2D2431B3B2A6108EA0208042B15D835
:1020A800DFE803F0352B22190300D6F89C30002B0B
:1020B80037D1EB6A1FFA83F9D6F8984034B1236810
:1020C8002046494698476468002CF8D1B8F1000FBB
:1020D800DBD1BDE8F883B06F696B036889B29847B4
:1020E800B8F1000FD1D1F4E7F06FA96B036889B29A
:1020F8009847B8F1000FC8D1EBE7D6F88000E96B34
:10210800036889B29847B8F1000FBED1E1E7D6F865
:102118008400296C036889B29847B8F1000FB4D1DC
:10212800D7E703F1FF3900231FFA89F9C6F89C3075
:10213800C2E700BF00080040C06000202DE9F84356
:102148002B4D2A69EB6812EA030824D0294E4FF078
:102158000047B8FA88F327FA03F2D2431B3B2A61F7
:1021680008EA0208042B13D8DFE803F03229201705
:102178000300736F002B34D1EB6A1FFA83F9346FB5
:1021880034B123682046494698476468002CF8D142
:10219800B8F1000FDDD1BDE8F883306D696B0368D5
:1021A80089B29847B8F1000FD3D1F4E7706DA96BE5
:1021B800036889B29847B8F1000FCAD1EBE7B06D50
:1021C800E96B036889B29847B8F1000FC1D1E2E71B
:1021D800F06D296C036889B29847B8F1000FB8D13F
:1021E800D9E703F1FF3900231FFA89F97367C6E7B6
:1021F80000040040C06000202DE9F8434FF08045FE
:102208002A69EB6812EA030824D0294E4FF00047E8
:10221800B8FA88F327FA03F2D2431B3B2A6108EA8B
:102228000208042B13D8DFE803F032292017030033
:10223800F36C002B34D1EB6A1FFA83F9B46C34B118
:1022480023682046494698476468002CF8D1B8F1BD
:10225800000FDDD1BDE8F883B06A696B036889B205
:102268009847B8F1000FD3D1F4E7F06AA96B036877
:1022780089B29847B8F1000FCAD1EBE7306BE96B28
:10228800036889B29847B8F1000FC1D1E2E7706BD3
:10229800296C036889B29847B8F1000FB8D1D9E71B
:1022A80003F1FF3900231FFA89F9F364C6E700BF79
:1022B800C06000202DE9F8435A4D2A69EB6812EAFC
:1022C800030825D0584E4FF00047B8FA88F327FA8C
:1022D80003F2D2431B3B2A6108EA0208042B14D8F4
:1022E800DFE803F04A41382F0300736A002B40F0FF
:1022F8009280EB6A1FFA83F9346A34B12368204666
:10230800494698476468002CF8D1B8F1000FDCD131
:10231800464D2A69EB6812EA03084AD0424E4FF04C
:102328000047B8FA88F327FA03F2D2431B3B2A6125
:1023380008EA0208042B39D8DFE803F05B51473D6F
:1023480027003068696B036889B29847B8F1000FB5
:10235800BBD1DDE77068A96B036889B29847B8F10B
:10236800000FB2D1D4E7B068E96B036889B2984727
:10237800B8F1000FA9D1CBE7F068296C036889B2DE
:102388009847B8F1000FA0D1C2E7D6F81431002B56
:1023980039D1EB6A1FFA83F9D6F8104134B12368B2
:1023A8002046494698476468002CF8D1B8F1000FD8
:1023B800B7D1BDE8F883D6F8F000696B036889B235
:1023C8009847B8F1000FACD1F3E7D6F8F400A96B41
:1023D800036889B29847B8F1000FA2D1E9E7D6F8A7
:1023E800F800E96B036889B29847B8F1000F98D1F3
:1023F800DFE7D6F8FC00296C036889B29847B8F182
:10240800000F8ED1D5E703F1FF3900231FFA89F9B0
:10241800C6F81431C0E703F1FF3900231FFA89F920
:10242800736269E7002C0140C0600020004401404D
:102438002DE9F8432B4D2A69EB6812EA030824D0EA
:10244800294E4FF00047B8FA88F327FA03F2D2432F
:102458001B3B2A6108EA0208042B13D8DFE803F0C3
:10246800322920170300736A002B34D1EB6A1FFA54
:1024780083F9346A34B1236820464946984764682A
:10248800002CF8D1B8F1000FDDD1BDE8F883306831
:10249800696B036889B29847B8F1000FD3D1F4E7A4
:1024A8007068A96B036889B29847B8F1000FCAD160
:1024B800EBE7B068E96B036889B29847B8F1000F99
:1024C800C1D1E2E7F068296C036889B29847B8F18E
:1024D800000FB8D1D9E703F1FF3900231FFA89F9B2
:1024E8007362C6E7002C0140C0600020F0B50668A2
:1024F800504CB30AA34200F0848061D94E4CA342E9
:1025080000F0828074D94D4CA34268D00134A342B4
:1025180055D107254FF49C7790F805C002232CFA73
:1025280003F084468340A800002970D0D6F80CE058
:1025380044190CEB440C9BB2414C43EA0E030CF1DA
:10254800040E44F82C1044F82E20F360E319EFF33E
:102558001181502282F31288421904EBC202D2F888
:1025680010C0BCF1000F03D044F807C0136904334E
:10257800421904EBC202576917B11F60536904334B
:10258800421904EBC202976917B11F6093690433BB
:10259800421904EBC202D76917B11F60D36904332B
:1025A8000022C9B21A6081F31188284404EBC004E0
:1025B800236AC3B9F3684FF6FE721340F360F0BDA7
:1025C8004A3CA3421AD00134A34205D0B3F5801F78
:1025D800F5D1012548279FE7032598279CE706257D
:1025E8004FF4887798E7F36843F00103F360F0BD90
:1025F800033CA342E3D10425C0278DE702257027B9
:102608008AE70025202787E70525E82784E7D6F805
:102618000CE00B4CDB439BB203EA0E0300EB050E08
:102628000CEB4E0CF3600CF1040344F82C1044F846
:1026380023208BE74B0010005000100051001000C1
:10264800C060002030B503685A4D18885A4CB4FB56
:10265800F2F20139013AAB4294B283B089B282B244
:102668000DD0564883420AD0B3F1804F07D0A0F569
:102678009830834203D000F58060834202D122F073
:10268800700292B24E4883426AD000F5806083425D
:1026980041D022F4407200F58C3092B283421A8005
:1026A800D9621C8565D100221A8601225A611A88CE
:1026B800404942F001028B421A806AD0B3F1804F40
:1026C80069D0404A934268D002F58062934266D04E
:1026D80002F50062934264D002F58062934262D0B0
:1026E80002F59032934260D002F5406293425ED088
:1026F80002F58062934217D002F58062934208BFC8
:10270800092212D002A84FF0012340F8043D18F026
:10271800CDFD03B030BD01201A80D9621C855861F7
:102728001A8802431A80C9E70822274B03EBC20321
:1027380001A893F895408DF80440012300228DF8F4
:1027480005308DF807308DF8062018F0AFFD1B2CEA
:10275800DFD11E4B019301A818F0A8FD03B030BDCE
:1027680001201A80D9621C8558611A8802431A8090
:10277800A7E7124A934296D002F54062934292D05C
:1027880002F5806293428ED002F5806293428AD02D
:102798008BE70022C9E70122C7E70222C5E7032227
:1027A800C3E70422C1E70522BFE70622BDE70722E7
:1027B800BBE700BF002C014000A24A0400340140DE
:1027C8000010004000040040E05603081901000111
:1027D800204B98422DD0B0F1804F2CD0A3F59433E4
:1027E80098422AD003F58063984228D003F5006305
:1027F800984226D003F58063984224D003F590339D
:10280800984222D003F54063984220D003F58063B4
:10281800984207D003F58063984208BF092202D086
:102828000020704708220C4B03EBC20393F8940076
:1028380070470022F7E70122F5E70222F3E70322B7
:10284800F1E70422EFE70522EDE70622EBE707228E
:10285800E9E700BF002C0140E05603082DE9F04FDE
:1028680083B08E4DDFF8408201908B460BF1FF3329
:102878009B46013300F00E812DF052FE884C894FA3
:10288800DFF828C24FF4FA7A4FF0100E4FF47A7638
:10289800DCF80430C3F30803002B40F0DF80EFF3CB
:1028A8001183002B40F0DA802168AA6800BF2368F2
:1028B8009942F9D1386806FB00F39A1AB2FBF0F294
:1028C80006FB0121DCF80430C3F30803002B40F0B9
:1028D800A680EFF31183002B40F0A1802368A8683D
:1028E80000BF22689342F9D1D7F8009006FB09F29D
:1028F800101AB0FBF9F006FB03035B1AB3F57A7FF5
:10290800E0D3BAF1010AC3D1019B581CC0B22DF023
:102918006DFCDFF898C1DCF804304FF47A7AC3F321
:10292800080356464FF0100E002B38D1EFF31183F1
:10293800002B34D12168AA6800BF23689942F9D1D5
:10294800386806FB00F39A1AB2FBF0F206FB012185
:10295800DCF80430C3F30803002B41D1EFF31183F3
:10296800002B3DD12368A86800BF22689342F9D1A3
:10297800D7F8009006FB09F2101AB0FBF9F006FB35
:1029880003035B1AB3F57A7FE2D3BAF1010A3FF485
:102998006DAFDCF80430C3F30803002BC6D0EFF3A7
:1029A80011828EF31288A8682B68D90303D50123F6
:1029B800C8F80030A8682368D8F80010D2B282F3AB
:1029C80011883A68194406FB02F31B1AB3FBF2F3A9
:1029D80006FB0131DCF80430C3F30803002BBDD03B
:1029E800EFF311808EF31288D5F808902B68DB037B
:1029F80004D50123C8F80030D5F808902368D8F822
:102A08000020C0B280F311883868134406FB00F236
:102A1800A2EB0902B2FBF0F206FB0323B1E7EFF3E6
:102A280011808EF31288D5F808902B68DB0304D543
:102A38000123C8F80030D5F808902368D8F800209A
:102A4800C0B280F311883868134406FB00F2A2EB89
:102A58000902B2FBF0F206FB03234EE7EFF3118203
:102A68008EF31288A8682B68D90303D50123C8F808
:102A78000030A8682368D8F80010D2B282F3118811
:102A88003A68194406FB02F31B1AB3FBF2F306FB80
:102A9800013117E703B0BDE8F08F00BF10E000E098
:102AA80058600020BC600020B860002000ED00E005
:102AB800204B5B68C3F3080330B4BBB9EFF3118351
:102AC800A3B91D4A1D481368846800BF11688B426A
:102AD800F9D11B4A11684FF47A7202FB01F0001B0E
:102AE80030BCB0FBF1F002FB03007047EFF311823A
:102AF800102383F312881149124D8C680B68DB038D
:102B080044BF01232B600C4B48BF8C681B682868A6
:102B1800D2B282F311880A4A11684FF47A721844C3
:102B280002FB01F31B1B30BCB3FBF1F302FB0030CB
:102B3800704700BF00ED00E05860002010E000E0A2
:102B4800BC600020B86000202DE9F84F0746264EEB
:102B5800264DFFF7ADFF264A2649DFF89CC04FF007
:102B6800100E4FF47A744FF001086B68C3F3080332
:102B7800CBB9EFF31183B3B91368D1F808A000BF3C
:102B8800D2F800904B45F7D1D6F8009004FB09FB2A
:102B9800ABEB0A0ABAFBF9FA04FB03A31B1ABB4204
:102BA800E3D3BDE8F88FEFF3118A8EF31288D1F8DA
:102BB80008B00B68DB0344BFCCF80080D1F808B03C
:102BC8001368DCF800905FFA8AFA8AF31188D6F85D
:102BD80000A04B4404FB0AF9A9EB0B09B9FBFAF96D
:102BE80004FB0393DAE700BFBC60002000ED00E0BF
:102BF8005860002010E000E0B8600020012805D0EF
:102C080003D3022805D00020704751E7024B18680B
:102C18007047014B58687047282200202DE9F84F6B
:102C28002A4C2B4E2B4D2C4F804618F1FF384AD397
:102C3800FFF73EFF29494B68C3F308034FF0100C18
:102C48004FF47A724FF0010EEBB9EFF31183D3B959
:102C58002368D5F808A000BFD4F800904B45F7D1F9
:102C6800D6F8009002FB09FBABEB0A0ABAFBF9FAAB
:102C780002FB03A31B1AB3F57A7FD6D24B68C3F3C2
:102C88000803002BE1D0EFF3118A8CF31288D5F8F2
:102C980008B02B68DB0344BFC7F800E0D5F808B0DC
:102CA8002368D7F800905FFA8AFA8AF31188D6F871
:102CB80000A04B4402FB0AF9A9EB0B09B9FBFAF98E
:102CC80002FB0393D6E7BDE8F88F00BF58600020E9
:102CD800BC60002010E000E0B860002000ED00E0DB
:102CE80030B4EFF31183102282F312880649074C9F
:102CF8000A680748013200250A602560DBB20268CD
:102D080083F3118830BC704758600020B8600020F9
:102D180010E000E01D4B70B59C68236D626BDD69A7
:102D2800CAB1A36B33B12B0700D470BD236D082241
:102D38001A6270BD2A06F6D5D4E909028242216DCD
:102D480011D0501CA669A062B25C26690A85B042FF
:102D5800E9D3A362E7E7A906E3D5E26A42B1988C12
:102D6800216B9047DDE70B6823F080030B60DAE7FF
:102D7800E1699B8C6069DBB24E1CE6614354E169F2
:102D8800E368994228BFE261CBE700BF8056002084
:102D98001D4B70B55C68236D626BDD69CAB1A36BAE
:102DA80033B12B0700D470BD236D08221A6270BDA1
:102DB8002A06F6D5D4E909028242216D11D0501CA9
:102DC800A669A062B25C26690A85B042E9D3A3620B
:102DD800E7E7A906E3D5E26A42B1988C216B9047F0
:102DE800DDE70B6823F080030B60DAE7E1699B8C71
:102DF8006069DBB24E1CE6614354E169E3689942BD
:102E080028BFE261CBE700BF805600201D4B70B59C
:102E18001C68236D626BDD69CAB1A36B33B12B07E4
:102E280000D470BD236D08221A6270BD2A06F6D53B
:102E3800D4E909028242216D11D0501CA669A06212
:102E4800B25C26690A85B042E9D3A362E7E7A9061E
:102E5800E3D5E26A42B1988C216B9047DDE70B68B5
:102E680023F080030B60DAE7E1699B8C6069DBB2D1
:102E78004E1CE6614354E169E368994228BFE26168
:102E8800CBE700BF80560020002A12DD70B504464B
:102E98000D468E18236820469B6898470028F9D06D
:102EA800236815F8011B1B6820469847B542F1D1E5
:102EB80070BD704703685B6A03B11847704700BF6D
:102EC80003681B6A03B11847704700BF03682DE900
:102ED800F041DD691DB12B46BDE8F0411847002AD5
:102EE800174611DD04460E460F4400E023689B6830
:102EF800204698470028F9D0236816F8011B1B685C
:102F080020469847BE42F1D1BDE8F08103689B692D
:102F1800184700BF0368DB68184700BF03689B6851
:102F2800184700BF03685B68184700BF03681B6841
:102F3800184700BF014B5869F8E700BF2822002056
:102F4800054B53F8203033B11A689B88918A0B429D
:102F580018BF1B049361704788600020036803F161
:102F680038422DE9F04F920AA74DAA5C02F01F05DE
:102F780052090124022A04FA05F400F09F81032A69
:102F880000F09781012A00F0518101F003077A1EB1
:102F9800012AC1F3810EC1F300188488C1F34111DD
:102FA80040F24981E60700F13181A50700F11A8155
:102FB800600700F10581220700F1F080E60600F1C4
:102FC800DB80A50600F1C680600600F1B18022060C
:102FD80000F19C80E60500F18780A50572D46005A4
:102FE8005FD422054CD4E60439D4A50426D4600461
:102FF80013D4220401D4BDE8F08F1A6822F04042AD
:103008001A601A6842EA87771F60DA6822F040423D
:1030180042EA8171D960BDE8F08F1A6822F0405207
:103028001A601A6842EA07721A60DA6822F0405297
:1030380042EA0172DA602204DDD5DEE71A6822F07E
:1030480040621A601A6842EA87621A60DA6822F0F7
:10305800406242EA81626004DA60CAD5DDE71A6834
:1030680022F040721A601A6842EA07621A60DA6847
:1030780022F0407242EA0162A504DA60B7D5DDE7C2
:103088001A6822F440021A601A6842EA87521A60E3
:10309800DA6822F4400242EA8152E604DA60A4D5F2
:1030A800DDE71A6822F440121A601A6842EA0752E9
:1030B8001A60DA6822F4401242EA0152DA60220504
:1030C80091D5DDE71A6822F440221A601A6842EAAC
:1030D80087421A60DA6822F4402242EA8142600597
:1030E800DA607FF57EAFDCE71A6822F440321A60B6
:1030F8001A6842EA07421A60DA6822F4403242EA61
:103108000142A505DA607FF56AAFDBE71A6822F4A9
:1031180040421A601A6842EA87321A60DA6822F472
:10312800404242EA8132E605DA607FF556AFDBE7D6
:103138001A6822F440521A601A6842EA07321A6082
:10314800DA6822F4405242EA0132DA6022067FF558
:1031580041AFDBE71A6822F440621A601A6842EA53
:1031680087221A60DA6822F4406242EA8122600605
:10317800DA607FF52CAFDBE71A6822F440721A6038
:103188001A6842EA07221A60DA6822F4407242EAB0
:103198000122A506DA607FF517AFDBE71A6822F08F
:1031A800C0021A601A6842EA87121A60DA6822F0C6
:1031B800C00242EA8112E606DA607FF502AFDBE779
:1031C8001A6822F030021A601A6842EA07121A6076
:1031D800DA6822F0300242EA0112DA6022077FF54B
:1031E800EDAEDBE71A6822F00C021A601A6842EAB0
:1031F80087021A60DA6822F00C0242EA810260074C
:10320800DA607FF5D8AEDBE7EC7B03081A6822F0BA
:1032180003021A601A683A431A60DA6822F0030255
:103228000A43A507DA607FF5C3AEDBE7264A55698E
:103238002C435461A9E600224FF0010C4FF003091A
:103248000CFA02F636EA04002ED15000D3F808A092
:1032580009FA00F5ED430AEA050AC3F808A0D3F80D
:1032680008B00EFA00FA4AEA0B0AC3F808A0B3F845
:1032780004A02AEA06069E80B3F804A008FA02F61B
:1032880046EA0A06B6B29E801E682E401E60D3F833
:1032980000A007FA00F646EA0A061E60DE6801FA90
:1032A80000F035402843D8600132102AC8D1BDE863
:1032B800F08F054AD5692C43D46166E6024A9569C0
:1032C8002C43946161E600BF001002402DE9F04FE5
:1032D8004A484B4B4B4C4FF090414FF0010A4FF08E
:1032E80002094FF004084FF0080E4FF0100C202789
:1032F8004026802530F8022B12F0010F03D0196008
:10330800A3F804A0083312F0020F03D01960A3F841
:103318000490083312F0040F03D01960A3F8048056
:10332800083312F0080F03D01960A3F804E008333B
:1033380012F0100F03D01960A3F804C0083312F07C
:10334800200F02D019609F80083312F0400F02D07E
:1033580019609E80083312F0800F02D019609D809A
:10336800083312F4807F05D04FF4807B1960A3F8EE
:1033780004B0083312F4007F05D04FF4007B1960C5
:10338800A3F804B0083312F4806F05D04FF4806BB3
:103398001960A3F804B0083312F4006F05D04FF495
:1033A800006B1960A3F804B0083312F4805F05D0ED
:1033B8004FF4805B1960A3F804B0083312F4005F7F
:1033C80005D04FF4005B1960A3F804B0083312F479
:1033D800804F05D04FF4804B1960A3F804B0083330
:1033E800D20B04D04FF4004219609A80083301F5DB
:1033F8008061A1427FF47EAFBDE8F08F3C7D030879
:10340800686600200018004800B97047036803F197
:1034180038422DE9F04F920AB24DAA5C02F01F051E
:1034280052090124022A04FA05F400F05F81032AF4
:1034380000F05381012A00F00D8101F003077A1E84
:10344800012AC1F3810EC1F300188488C1F3411128
:1034580040F20581E6070BD51A6822F003021A60CC
:103468001A683A431A60DA6822F003020A43DA60FB
:10347800A5070DD51A6822F00C021A601A6842EAEC
:1034880087021A60DA6822F00C0242EA8102DA60E6
:1034980060070DD51A6822F030021A601A6842EAED
:1034A80007121A60DA6822F0300242EA0112DA6082
:1034B80022070DD51A6822F0C0021A601A6842EA7B
:1034C80087121A60DA6822F0C00242EA8112DA60D2
:1034D800E6060DD51A6822F440721A601A6842EAA4
:1034E80007221A60DA6822F4407242EA0122DA609E
:1034F800A5060DD51A6822F440621A601A6842EAD5
:1035080087221A60DA6822F4406242EA8122DA608D
:1035180060060DD51A6822F440521A601A6842EA09
:1035280007321A60DA6822F4405242EA0132DA605D
:1035380022060DD51A6822F440421A601A6842EA37
:1035480087321A60DA6822F4404242EA8132DA604D
:10355800E6050DD51A6822F440321A601A6842EA64
:1035680007421A60DA6822F4403242EA0142DA601D
:10357800A5050DD51A6822F440221A601A6842EA95
:1035880087421A60DA6822F4402242EA8142DA600D
:1035980060050DD51A6822F440121A601A6842EACA
:1035A80007521A60DA6822F4401242EA0152DA60DD
:1035B80022050DD51A6822F440021A601A6842EAF8
:1035C80087521A60DA6822F4400242EA8152DA60CD
:1035D800E6040DD51A6822F040721A601A6842EAA9
:1035E80007621A60DA6822F0407242EA0162DA6021
:1035F800A5040DD51A6822F040621A601A6842EADA
:1036080087621A60DA6822F0406242EA8162DA6010
:1036180060040DD51A6822F040521A601A6842EA0E
:1036280007721A60DA6822F0405242EA0172DA60E0
:1036380022040DD51A6822F040421A601A6842EA3C
:1036480087771F60DA6822F0404242EA8171D960C8
:10365800BDE8F08F244A55692C435461EDE60022F9
:103668004FF0010C4FF003090CFA02F636EA040099
:103678002ED15000D3F808A009FA00F5ED430AEA64
:10368800050AC3F808A0D3F808B00EFA00FA4AEA07
:103698000B0AC3F808A0B3F804A02AEA06069E801D
:1036A800B3F804A008FA02F646EA0A06B6B29E8003
:1036B8001E682E401E60D3F800A007FA00F646EAFE
:1036C8000A061E60DE6801FA00F035402843D8601B
:1036D8000132102AC8D1BDE8F08F034AD5692C43BE
:1036E800D461AAE6EC7B030800100240024A9569FF
:1036F8002C439461A1E600BF0010024010B103689A
:1037080082881A85704700BF10B1036882889A6161
:10371800704700BF18B1838811B102689361704780
:103728001B04FAE70E4B1B8801463BB90D4B0E4AAA
:103738001B7810680BB981F00101EBE70B4B5A6954
:103748001AB11A6810B910605874704708480949C6
:10375800008891FBF0F1012011605874704700BF98
:103768009460002096600020986000209C600020F3
:10377800B460002020A1070010B40A4B0A4A1C7844
:1037880001238340234052F8200029B9B3FA83F17A
:1037980049095DF8044BBDE7191C18BF01215DF804
:1037A800044BB7E7846000208860002008B5012139
:1037B8000220FFF7E1FF094B1B7803F00503052BF7
:1037C80008D000210120FFF7D7FF00210846FFF7A6
:1037D800D3FFFEE729F02FFBF3E700BF7C5600205C
:1037E80030B102688388128A1A4214BF012000206F
:1037F800704700BF2DE9F0410B4E356873691D40D5
:1038080010D0DFF828800127B5FA85F4C4F11F0429
:1038180008EB840307FA04F4986903689847A543FA
:103828007461F1D1BDE8F081000401402822002034
:103838002DE9F0410B4E356873691D4010D0DFF853
:1038480028800127B5FA85F4C4F11F0408EB840326
:1038580007FA04F4986903689847A5437461F1D19D
:10386800BDE8F08100040140282200202DE9F04144
:103878000B4E356873691D4010D0DFF8288001278A
:10388800B5FA85F4C4F11F0408EB840307FA04F4BD
:10389800986903689847A5437461F1D1BDE8F08140
:1038A80000040140282200202DE9F0410B4E356824
:1038B80073691D4010D0DFF828800127B5FA85F418
:1038C800C4F11F0408EB840307FA04F49869036839
:1038D8009847A5437461F1D1BDE8F0810004014027
:1038E800282200202DE9F0410B4E356873691D40F0
:1038F80010D0DFF828800127B5FA85F4C4F11F0439
:1039080008EB840307FA04F4986903689847A54309
:103918007461F1D1BDE8F081000401402822002043
:103928002DE9F0410B4E356873691D4010D0DFF862
:1039380028800127B5FA85F4C4F11F0408EB840335
:1039480007FA04F4986903689847A5437461F1D1AC
:10395800BDE8F08100040140282200202DE9F04153
:103968000B4E356873691D4010D0DFF82880012799
:10397800B5FA85F4C4F11F0408EB840307FA04F4CC
:10398800986903689847A5437461F1D1BDE8F0814F
:1039980000040140282200200D490E4B8A6942F09C
:1039A800010210B58A611A680B4C42F400621A6071
:1039B8001A6842F480521A6004F11800402200216B
:1039C80031F08AFD4FF0FF33A365C4F85B3010BDBA
:1039D80000100240000001402822002003681B6AF2
:1039E800184700BF70B44E1C0568C2728672AC6975
:1039F800A44670BC604700BF2DE9F0410446184654
:103A08000D4616461F4631F0A3F92844A0722068D7
:103A1800E672294645693B4632462046AC46BDE833
:103A2800F041604770B50B4C054616460B460246FA
:103A380002212068FFF7E0FF2A46074B206814217F
:103A4800FFF7DAFF33462A4620681621BDE87040A2
:103A5800D2E700BFB0560020C29A0308036810B529
:103A680004461B689847236820469B689847A37BB1
:103A78000133A37310BD00BF10B5036804469B68EB
:103A88009847FF2301226373227310BD08B5FEF720
:103A980031F938B12D2282710022C2712021BDE88E
:103AA8000840B1E408BD00BF0B4B984211D0A3F504
:103AB8007843984202D04FF0FF3070470122074BFD
:103AC80003EB02135A89013292B25A81588980B2A3
:103AD80070470022F3E700BF00300140A4620020D5
:103AE8002DE9F04F90F8643087B00746002B40F07E
:103AF800DB84AA4B0093009B93F85F30D7E905025B
:103B0800002B00F01581038823F040031B041B0CD5
:103B1800038003889BB223F0380343F03803038003
:103B2800038843F04003038097F8621012B11368CA
:103B380092881A8540F2E93302E0002B00F00985EB
:103B48000289013B12F0020F9BB2F6D01A230373CD
:103B580000F10C0440F2E93302E0002B00F0F98494
:103B68000289013B12F0010F9BB2F6D023787869E5
:103B780040F2E93302E0002B00F0E7840289013BC0
:103B880012F0020F9BB2F6D0017340F2E93302E063
:103B9800002B00F0DA840289013B12F0010F9BB27E
:103BA800F6D0037BBB6913B11A689B889361FEF753
:103BB8007FFF0446FEF77CFF8442FBD078690388C8
:103BC80023F040031B041B0C0380038823F03803F5
:103BD8001B041B0C0380038843F0400303803B7CD9
:103BE800022B36D0B7F952305BB2013302D007B09E
:103BF800BDE8F08F97F950300133F8D10A262CF040
:103C08008FFC4FF4FA75FEF753FF0446FEF750FF9A
:103C1800001BB0F57A7FF9D3013DF4D107202CF0D1
:103C2800E5FA4FF47A75FEF743FF0446FEF740FFC6
:103C3800001BB0F57A7FF9D3013DF4D1013EDED106
:103C48005749584B5848594A0860DA6007B0BDE8E8
:103C5800F08FBB6913B11A689B88138540F2E9336A
:103C680002E0002B00F0F5840289013B12F0020FFC
:103C78009BB2F6D0C323037340F2E93302E0002B72
:103C880000F0E7840289013B12F0010F9BB2F6D0E5
:103C9800037B78698389038999074FF0050C04AD84
:103CA8004FF47A724FF0FF064FF6FF7406D4531E96
:103CB8009BB2E2B11A4603899907F8D506734FF407
:103CC8007A7302E08BB2A34211D00289D20703F1C2
:103CD800FF31F7D5027BD2B20DB12A7001350CF154
:103CE800FF32BCF1000F04D094461A46E3E7FFF711
:103CF800DBFEBB6913B11A689B8893619DF812506B
:103D08009DF813309DF810409DF811109DF814008F
:103D18009DF8152043EA05231BB241EA042142EA33
:103D28000022A7F85230A7F85010A7F854205BE7F4
:103D3800038823F040031B041B0C038003889BB2F9
:103D480023F0380343F038030380038843F040032B
:103D5800038012B1136892881A8540F2E93302E0B1
:103D6800002B00F066840289013B12F0020F9BB21F
:103D7800F6D06B23037300F10C0140F2E93302E043
:103D8800002B00F056840289013B12F0010F9BB210
:103D9800F6D00B78786940F2E9330CE0282200204D
:103DA800FC9F002000ED00E0EFBEADDE0400FA0548
:103DB800002B00F03A840289013B12F0020F9BB2FB
:103DC800F6D08023037340F2E93302E0002B00F0C1
:103DD8002C840289013B12F0010F9BB2F6D0037BC1
:103DE800BB6913B11A689B8893619623A84CA94EA6
:103DF800DFF8A882A84DDFF8A89201974FF0100AC3
:103E08001F46FEF755FE4FF47A7C4FF0010ED8F8A6
:103E18000430C3F30803002B40F02883EFF3118329
:103E2800002B40F023832368A96800BF22689342CF
:103E3800F9D132680CFB02FBABEB0101B1FBF2F1EB
:103E48000CFB03131B1AB3F57A7FE0D3013FD8D1DB
:103E5800019FBB6913B11A689B881385786940F282
:103E6800E93302E0002B00F0F1830289013B12F0F4
:103E7800020F9BB2F6D06823037340F2E93302E0E5
:103E8800002B00F0E3830289013B12F0010F9BB283
:103E9800F6D0037B786940F2E93302E0002B00F0AA
:103EA800D2830289013B12F0020F9BB2F6D00323A2
:103EB800037340F2E93302E0002B00F0C483028967
:103EC800013B12F0010F9BB2F6D0037BBB6913B123
:103ED8001A689B8893619623DFF8C0816E4DDFF8DE
:103EE800C09101974FF0100A1F46FEF7E1FD4FF40D
:103EF8007A7C4FF0010ED8F80430C3F30803002B86
:103F080040F09682EFF31183002B40F091822368F2
:103F1800A96800BF22689342F9D132680CFB02FB02
:103F2800ABEB0101B1FBF2F10CFB03131B1AB3F568
:103F38007A7FE0D3013FD8D1019FBB6913B11A68DA
:103F48009B881385786940F2E93302E0002B00F082
:103F580077830289013B12F0020F9BB2F6D06B23E4
:103F6800037340F2E93302E0002B00F06983028911
:103F7800013B12F0010F9BB2F6D0037B786940F247
:103F8800E93302E0002B00F058830289013B12F06C
:103F9800020F9BB2F6D00323037340F2E93302E029
:103FA800002B00F04A830289013B12F0010F9BB2FB
:103FB800F6D0037BBB6913B11A689B889361FEF73F
:103FC80077FD0446FEF774FD001B0E28FAD9BB697D
:103FD80013B11A689B881385786940F2E93302E0C7
:103FE800002B00F061830289013B12F0020F9BB2A3
:103FF800F6D06A23037340F2E93302E0002B00F0A5
:1040080053830289013B12F0010F9BB2F6D0037B68
:10401800786940F2E93302E0002B00F0428302891C
:10402800013B12F0020F9BB2F6D01023037340F24B
:10403800E93302E0002B00F034830289013B12F0DF
:10404800010F9BB2F6D0037BBB6913B11A689B883A
:104058009361FEF72DFD0446FEF72AFD001B0E288E
:10406800FAD9BB6913B11A689B881385786940F23D
:10407800E93302E0002B00F011830289013B12F0C2
:10408800020F9BB2F6D06C23037340F2E9330CE0C5
:1040980058600020BC60002010E000E000ED00E067
:1040A800B8600020002B00F0F9820289013B12F071
:1040B800010F9BB2F6D0037B786940F2E93302E046
:1040C800002B00F0E8820289013B12F0020F9BB23C
:1040D800F6D00023037340F2E93302E0002B00F02E
:1040E800DA820289013B12F0010F9BB2F6D0037B02
:1040F800BB6913B11A689B889361FEF7D9FC044623
:10410800FEF7D6FC001B0E28FAD9BB6997F8631096
:1041180013B11A689B881385786940F2E93302E085
:10412800002B00F0B5820289013B12F0020F9BB20E
:10413800F6D01923037340F2E93302E0002B00F0B4
:10414800A7820289013B12F0010F9BB2F6D0037BD4
:10415800786940F2E93302E0002B00F09682028988
:10416800013B12F0020F9BB2F6D0017340F2E93323
:1041780002E0002B00F089820289013B12F0010F56
:104188009BB2F6D0037BBB6913B11A689B88936115
:10419800FEF78EFC0446FEF78BFC001B0E28FAD9AE
:1041A800BB6913B11A689B881385786940F2E933B3
:1041B80002E0002B00F066820289013B12F0020F38
:1041C8009BB2F6D01B23037340F2E93302E0002BC5
:1041D80000F058820289013B12F0010F9BB2F6D021
:1041E800037B786940F2E93302E0002B00F0478254
:1041F8000289013B12F0020F9BB2F6D01823037319
:1042080040F2E93302E0002B00F039820289013BD9
:1042180012F0010F9BB2F6D0037BBB6913B11A6889
:104228009B889361FEF744FC0446FEF741FC001BA3
:104238000E28FAD9BB6913B11A689B881385786967
:1042480040F2E93302E0002B00F016820289013BBC
:1042580012F0020F9BB2F6D01C23037340F2E9332D
:1042680002E0002B00F008820289013B12F0010FE6
:104278009BB2F6D0037B786940F2E93302E0002B69
:1042880000F0F7810289013B12F0020F9BB2F6D0D1
:104298001023037340F2E93302E0002B00F0E981B8
:1042A8000289013B12F0010F9BB2F6D0037BBB6978
:1042B80013B11A689B889361FEF7FAFB0446FEF770
:1042C800F7FB001B0E28FAD9BB6913B11A689B8843
:1042D8001385786940F2E93302E0002B00F0C681CB
:1042E8000289013B12F0020F9BB2F6D03723037309
:1042F80040F2E93302E0002B00F0B8810289013B6B
:1043080012F0010F9BB2F6D0037B786940F2E933D3
:1043180002E0002B00F0A7810289013B12F0020F96
:104328009BB2F6D01023037340F2E93302E0002B6E
:1043380000F099810289013B12F0010F9BB2F6D07F
:10434800037BBB6913B11A689B889361FEF7B0FBC6
:104358000446FEF7ADFB001B0E28FAD9BB6913B162
:104368001A689B881385786940F2E93302E0002BCC
:1043780000F076810289013B12F0020F9BB2F6D061
:104388003823037340F2E93302E0002B00F0688120
:104398000289013B12F0010F9BB2F6D0037B7869CA
:1043A80040F2E93302E0002B00F057810289013B1B
:1043B80012F0020F9BB2F6D00123037340F2E933E7
:1043C80002E0002B00F049810289013B12F0010F45
:1043D8009BB2F6D0037BBB6913B11A689B889361C3
:1043E800FEF766FB0446FEF763FB001B0E28FAD9AE
:1043F8007A69138823F040031B041B0C138013886D
:1044080023F038031B041B0C1380138843F040036C
:104418001380FEF74DFB0446FEF74AFB8442FBD0AF
:1044280000990123D7E9050281F85F30FFF76BBBDC
:10443800EFF311818AF31288D5F808B02B68DB03F3
:1044480044BFC9F800E0D5F808B02368D9F80020BF
:10445800C9B281F31188316813440CFB01F2A2EB55
:104468000B02B2FBF1F20CFB03235FE5EFF31181C2
:104478008AF31288D5F808B02B68DA0344BFC9F864
:1044880000E0D5F808B02368D9F80020C9B281F354
:104498001188316813440CFB01F2A2EB0B02B2FB4A
:1044A800F1F20CFB0323CDE41D09013D052D03F0BA
:1044B8000F0352D8834A32F8150040FA03F2D407A2
:1044C8004BD5012404FA03F3013B184030F098FC63
:1044D8007D4BDFF810825E5D064418EBC6053CD0C4
:1044E80020220023AA71EB7158F83600774A00F1B0
:1044F80038439B0AD25C02F01F035209022A04FACD
:1045080003F300F0D980032A32D0A24200F0CF8012
:10451800AB88049304A90024059417F0EBF9AB8841
:104528006B4AFA60B3FA83F2C2F11F02501C24D11D
:10453800684A0092B3FA83F3C3F11F03591C3FF48E
:10454800DAAA012202FA03F30CE0FFF7ADFAFFF74B
:1045580029BBFFF7A9FAFFF70ABB5D4B5D4AFB6071
:10456800009201235C490A6813430B60FFF7C3BA42
:104578005A4AD1690B43D361CAE7D1B201F0FC03AF
:1045880003F1804303F5803301F00300D3F808C03A
:10459800504958F83690009180004FF00F0E0EFAEF
:1045A80000FE2CEA0E0C01EB820E07F10C08CEF887
:1045B8001880C3F808C0D3F808E0494EDFF828C1CE
:1045C800C9F38721814041EA0E01B0184FF0010874
:1045D800996008FA02F3CCF8003090F8E090049261
:1045E800082304A88DF815308DF816808DF814402E
:1045F8002BF08AFD009901EB090393F85820F02A63
:1046080011D94E44F02196F8F0208DF80C2003A81B
:1046180003228DF80E408DF80F8083F858108DF81E
:104628000D2016F043FEAB8884E7FFF73DFAFFF74D
:10463800D7BBFFF739FAFFF7ADBBFFF735FAB9E497
:10464800FFF732FA9AE4FFF72FFA3FE4FFF72CFA64
:1046580020E4FFF729FAFFF71CBBFFF725FABAE6B3
:10466800FFF722FA9BE6FFF71FFA6AE6FFF71CFA44
:104678004BE6FFF719FA1AE6FFF716FAFBE5FFF71C
:1046880013FACAE5FFF710FAABE5FFF70DFA7AE57A
:10469800FFF70AFA5CE5FFF707FA29E5FFF704FADE
:1046A8000AE5FFF701FACFE4FFF7FEF9B0E40B4A99
:1046B80051690B4353612BE7084A91690B43936196
:1046C80026E700BF3C7D0308487D0308EC7B030810
:1046D8003908000828220020000401400010024088
:1046E800E05603086866002014040140F0B58369A9
:1046F80083B0064613B11A689B8813857069DFF882
:10470800A0C08389C3244FF47A7306276D464FF6F9
:10471800FF710CF1010C03E0013B9BB28B421CD0F2
:1047280002899207F8D504734FF47A7302E0A3B2B2
:104738008B4212D00289D20703F1FF34F7D5027BEE
:10474800D2B20DB12A7001354FB1013FFF24BCF13F
:10475800000FE5D09CF80040DBE7FFF7A5F9B36947
:1047680013B11A689B8893619DF805009DF8015064
:104778009DF802109DF803409DF804209DF806302E
:1047880041EA052143EA002342EA04220120A6F86F
:104798005010A6F85220A6F8543003B0F0BD00BF60
:1047A800D8570308037A022B01D000207047F0B5D0
:1047B800036983B013B11A689B881385014640F2D8
:1047C800E933C06801E0002B5ED00289013B12F09A
:1047D800020F9BB2F7D0BB23037340F2E93301E029
:1047E800002B51D00289013B12F0010F9BB2F7D088
:1047F800037BC868838903899C074FF005076E46C9
:104808004FF47A724FF0FF0C4FF6FF7506D4531E23
:104818009BB2D2B11A4603899C07F8D580F80CC020
:104828004FF47A7302E0A3B2AB420ED00289D207EA
:1048380003F1FF34F7D5027BD2B20EB132700136E4
:104848007A1E27B117461A46E5E7FFF72DF90B69D7
:1048580013B11A689B8893619DF800609DF8010068
:104868009DF802509DF803209DF804409DF80530FE
:1048780040EA062042EA052243EA0423C8820120CE
:104888000A834B8303B0F0BDFFF70EF9B1E700BF11
:10489800427A4AB110B5044604F10A01D0E9003061
:1048A80098470023637210BD704700BF437A5A1CB3
:1048B8000344D2B242729972037A93420AD84AB137
:1048C80010B5044604F10A01D0E9003098470023E6
:1048D800637210BD704700BFA8B10D4B012210B420
:1048E80002FA01F103F1750402E00333A3420BD08D
:1048F80013F8012C8242F8D11A780A42F5D0012027
:104908005DF8044B7047704700205DF8044B704712
:10491800E157030830B40A4D002305F5807401E01F
:10492800272B0AD003EB43020133A15C8142F7D164
:104938002A4430BC92F802017047002030BC70470E
:10494800E0560308024A136823EA00001060704723
:10495800283000202DE9F84F0BF09AFADFF8408351
:10496800AF4B434525D2DFF83C93AE4F03F1140615
:104978009A464C462588621985B1BA420ED2052D51
:104988000CD936F8143C6188C3F30B03994200F044
:10499800E280144625886219002DEED156F8101CC5
:1049A80050460AF1140A1BF007FEC24506F1140628
:1049B800DFD39D490B78A3F11702022A0FD99B4A2E
:1049C80012F83300002840F0FC80D80002445278E6
:1049D8002AB1974A12F83330002B00F01A81954B10
:1049E8005A78052A40F2E08000225A701A789248D4
:1049F80092490160022A00F2E08002EB8201904BAA
:104A0800C2EBC10203EB4203998C5A8C8D4C914244
:104A1800236001D300225A848B4B9A78042A00F031
:104A2800D98032B91A88B2F5F07F84BF4FF4F0729A
:104A38001A80864DFCF75AFB2B68854A1A40002AD3
:104A480000F0EA80D80700F1DF80590400F1D78030
:104A58001A0700F1CF809B0400F1C5802CF00EFDF1
:104A680010B97C481AF0D2FA8020FFF76BFF4FF498
:104A78000070FFF767FF4FF40030FFF763FF4FF454
:104A88000010FFF75FFF4FF00070FFF75BFF4FF07C
:104A98008060FFF757FF29F005F8002130226E48A3
:104AA80030F01AFD206827F065FB6C4B256803F190
:104AB800640102E00533994274D01A78002AF9D1CA
:104AC8009C78D8788442F5D26549664B0E79664C55
:104AD800C820642111FB060159600021634883F84E
:104AE8002010C3E90211C3E90411C3E9061183F8D0
:104AF80021105F4B5F492270056019600AF0A6FF1C
:104B08005D4B9FED5E5A1B885D4A9FED5E6A50794A
:104B18005D4906EE903AF8EEE66A1388C5EE265A25
:104B280007EE103A53881279C1ED005A07EE903A11
:104B3800B8EEC77AF8EEE77A544B27EE067A67EEB6
:104B4800867A18725A7283ED017AC3ED007ABDE84D
:104B5800F84F0BF043B963799B077FF41AAF56F807
:104B6800101C94F804B050461BF026FD36F8143C8F
:104B7800BBEB133F07D00AF1140AC24506F114062D
:104B8800FFF4F7AE15E736F8123C56F8100CAA1FDA
:104B9800C3F30B039A4204F10601A8BF1A4630F08A
:104BA8003BFCE8E701228FE72449234801EB021187
:104BB8001A780160022A7FF620AF00221A70204B73
:104BC80022E7D80014186468002C7FF4FFAE17247D
:104BD8000C70FBE69A8AB2F57A7FBFF42AAF4FF4DD
:104BE8007A729A8225E72A48FFF7ACFE4020FFF741
:104BF800A9FE33E72748FFF7A5FE2B682BE72648D1
:104C0800FFF7A0FE2B6823E72448FFF79BFE2B68DD
:104C18001BE718230B70E2E643F008032B6011E74B
:104C28006CBB03080000040894320020B07D030820
:104C380040640308EC9700209443002034290020A6
:104C48002428002090430020A06D00202830002058
:104C58000960000200620020AC3C0020843700207C
:104C6800B05D0020943F002048200020E03C002058
:104C7800D43B002066330020F0510020C0C9FB4817
:104C8800643B002017B7D138F451002004580020A5
:104C980009400002016000020920000208600002C9
:104CA8001CC0030802F00308F8B5174D2B78A92B90
:104CB80028D16B78BE2B25D1022229464FF6FF70EA
:104CC800FBF71EFD114FAC1C22884AB1A618BE4244
:104CD80018D2052A16D92146FBF712FD3446F3E708
:104CE80021460222FBF70CFD0222A118FBF708FD62
:104CF8000634074B641B1C8041F60F53C31A5842F5
:104D08005841F8BD0020FCE700F003080000040843
:104D1800705800202DE9F04FDFF844914B4F8BB0CD
:104D28000326A7EB09071022002106A830F0D4FBC0
:104D3800CDE90497464B1A69120604D5454A5A60CC
:104D480002F188325A6001228DF824203422DA6078
:104D5800414B424C1B88ADF800300222694604A83A
:104D6800FCF78EF9022269464FF6FF70FBF7C8FC84
:104D7800DFF8F0A080464FF0000B544536D30AAC5C
:104D8800002524F8245D0222214604A8FCF778F9BE
:104D9800022221464046FBF7B3FC40BAC043ADF8B7
:104DA8000800022202A904A8FCF76AF9079860B172
:104DB80006ABC0F104022946184430F08DFB069971
:104DC80004A8FCF703F9CDE907509DF82430089AA8
:104DD80023B11F490B6943F080030B61013E2DD0BD
:104DE800002AA0D1FFF760FF50B32CE065888DF84A
:104DF8000DB0C5F30B05AB1DADF808302388C3F320
:104E08000B02ADF80A201B0B062202A904A88DF894
:104E18000C30FCF735F9062202A94046FBF770FC76
:104E2800616880462A4604A8FCF72AF9616840466A
:104E38002A46FBF765FC143480469EE7002AD1D049
:104E48000520FBF7EFFE0BB0BDE8F08F000004086B
:104E58000020024023016745555803086CBB03082E
:104E680000F003081CC0030808B50BF011F8FFF7A1
:104E780051FF0AF0B3FFFFF76DFD0120BDE80840C0
:104E88001CF036BA08B5FCF7CFF90BF001F8FFF7BC
:104E980041FFBDE808400AF0A1BF00BF08B50AF00D
:104EA800F7FFFFF737FFBDE808400AF097BF00BFDC
:104EB8000378202B024600F10100F9D0092BF7D026
:104EC8002D2B00F0A4802B2B03BF5378B7EE000ADC
:104ED8000246B7EE000AA3F13001C8B209289FEDD7
:104EE800577A10D8F2EE046A07EE901AF8EEE77ACD
:104EF80012F8013FE7EE267AA3F13001C8B209287B
:104F0800B0EE677AF0D92E2B63D003F0DF03452B80
:104F180002D020EE070A704710B451782D294FD0DF
:104F28002B2979D0A1F13003092B02F101027AD89B
:104F38000024002303EB830301EB430312F8011F52
:104F4800A1F130000928A3F13003F3D9B3F59A7F12
:104F58001A4628BF4FF49A72072B6CD9DFED386ACE
:104F68001346F7EE007A083B072B67EEA67AFAD8C5
:104F780002F00702DAB1F2EE046A012A67EEA67AB5
:104F880015D0022A67EEA67A11D0032A67EEA67A10
:104F98000DD0042A67EEA67A09D0052A67EEA67A0C
:104FA80005D067EEA67A062A18BF67EEA67A002C07
:104FB8003BD087EE277A5DF8044B20EE070A70474E
:104FC8009178A1F13003092B02F1020230D80124B3
:104FD800AFE75378A3F13001C8B2092802F1010202
:104FE80093D8F2EE046AF0EE665A07EE901AF8EEDD
:104FF800E77A12F8013F87EEA66AA3F13001C8B23A
:10500800092866EEA56A37EE067AEED97DE7537869
:10501800BFEE000A02465EE79178A1F13003092B42
:1050280002F1020284D9F7EE007A27EE277AC2E766
:10503800F7EE007ABDE7F7EE007A9BE70000000084
:1050480020BCBE4CF8B5064615460846B6FBF2F439
:1050580034B905FB14640C4B1B5D00F8013BF8BD2B
:10506800B4FBF2F75FB905FB1747074B05FB146460
:10507800DA5D00F8012B1B5D00F8013BF8BD3846EE
:10508800FFF7E0FFEFE700BF8C830308B5EEC00A27
:10509800DFED677A674AF1EE10FACCBF30EE270AE7
:1050A80030EE670ADFED647A20EE270A2DE9F04733
:1050B800FDEEC07A88B017EE904A84EAE4760023C1
:1050C800A6EBE476CDE902330493A2FB06325FEA4D
:1050D800D208054641D105AF58483946554BA3FB80
:1050E8000623DB0803EB8303A6EB4303002CC35C16
:1050F8000B704FF00002ACBF20232D234A703846B6
:105108008DF808302FF024FE0128394639D00228BE
:1051180042D0032805BF302302A802A88DF8093021
:1051280030F0E2F902A82FF013FE0338C4B2224689
:1051380002A9284630F00EFA00232B5528462FF0F6
:1051480007FE2E22431C02A92A542144E81830F0F5
:10515800E7F9284608B0BDE8F087394BA3FB0623DA
:105168005B0922D105AF35483946324AA2FB0832DD
:10517800D20802EB8202A8EB4202835C01F8013BF1
:10518800ACE7302302A88DF809308DF80A308DF885
:105198000B3030F0A9F9C5E7302302A88DF80930A3
:1051A8008DF80A3030F0A0F9BCE7264AA2FB0612B7
:1051B8005FEA92190ED105AF204839461D4AA2FB75
:1051C80003C2D20802EB8202A3EB4203C35C01F8DC
:1051D800013BCAE71C4AA2FB06125FEA523A0ED10B
:1051E80005AF16483946134AA2FB09C2D20802EB9A
:1051F8008202A9EB4202825C01F8012BDEE7134828
:10520800B6FBF0F058B905AF39460A20BAFBF0F200
:1052180000FB12A20948825C01F8012BE3E705AF05
:1052280039460A220193FFF70DFF019B0146ECE77F
:105238006F12033ACDCCCCCC00007A448C8303089F
:105248001F85EB51D34D62105917B7D1A0860100C5
:105258000F4B2DE93048D3E9004554EA05020AD13D
:10526800034640F2011200201880988098715A80F5
:105278001881BDE83088074B1A6814EB020B45F11A
:10528800000C5A466346FBF7E7F80120BDE8308872
:10529800083C00205860002030B403888278164DFE
:1052A800C478A3F2B27303F0030101EB4101013AA0
:1052B80002EB810205EB4202611E958A027940F2F7
:1052C800B5549B0804FB03132B4403EB430302EB85
:1052D800C303427981790089C3EB031302EB83038B
:1052E800C3EB031301EB83034FF47A720021C2FB73
:1052F800030130BC704700BFE056030802B370B426
:105308008E1803E0121B14D1B14215D010F8012BEE
:10531800A2F14103192B11F8013BA3F1410598BFF4
:105328002032192D03F12004ECD9D21A01D1002B17
:10533800EAD1104670BC70470022104670BC704716
:105348001046704770B5044608460D462FF000FD1C
:10535800064602E014F8013F43B13246294620468A
:10536800FFF7CCFF0028F5D1204670BD1C4620462B
:1053780070BD00BF4FF0FF32FFF7C0BFA0F161035F
:10538800192B98BF20387047A0F14103192B98BFFB
:1053980020307047202805D0093804288CBF002009
:1053A800012070470120704738B501460B78184630
:1053B800FFF7F0FF0A4601310028F7D12B2B27D041
:1053C8002D2B24D0A3F13004392B4FF00001154DBB
:1053D800E4B20FD8092C01EB81030BD8A94213D8EA
:1053E80010D004EB430112F8013FA3F13004392B2C
:1053F800E4B2EFD978B1B1F1004F28BF4FF00041C6
:10540800484238BD052CECD94FF0FF31EBE70120BD
:1054180053780132D6E76FF00040884228BF08462B
:1054280038BD00BF99999919613819288CBF002097
:1054380001207047413819288CBF0020012070478F
:10544800303809288CBF002001207047A0F13003B4
:10545800092B07D920F02000413819288CBF0020DB
:10546800012070470120704730B402681146531C70
:10547800036011F8024B0160D31C517803609378E4
:10548800151D05601B0443EA0123D078234343EA32
:10549800006030BC704700BF0368591C1A460160A1
:1054A80012F8021B0260587841EA0020704700BFDA
:1054B80003685A1C02601878704700BF2DE9F04F46
:1054C800C44B1D788DB0002D52D1C34BC34C93F8FB
:1054D80000B0DFF83C93DFF83CA30BF0010B04F5B8
:1054E8001C7754F80F0C38B1FDF71CFD002840F06C
:1054F800078114F8073C3BB9D034BC4205F10105DB
:10550800EFD10DB0BDE8F08FDAF8002054F80B1C8D
:10551800521A632AF0D9012B00F02482022BEBD116
:10552800AF4BB049DB78B04A89F86900003318BF3F
:1055380001230B70AD4854F80F3C1360C9F81430C0
:10554800C9F86430AA4B0360A248AA4AC9F8602087
:1055580001214023017089F86830A74825F098FC9C
:10556800A64824F0B9FB4FF480500DF053FDC3E773
:105578009E4B18680028C4D0FFF78AF9DFF868A2A4
:10558800DFF89482DAF80000FDF7CCFC0028B8D0E8
:10559800DAF80000DFF88492FDF7BCFC0928D9F896
:1055A80000601AD03F2818D0002E6CD1042800F0D3
:1055B800D3810C2800F09D807F28E3D0A0F1200340
:1055C800DBB25E2BDED82028DCD0731C08F806007E
:1055D800C9F8003024F078FBD4E7002E67D1884B57
:1055E800354603F59877002D46D00833BB42FAD1EB
:1055F800DFF82CB22868DBF80020845D935D9C42BC
:10560800304402EB060140F0AB81741E444432463C
:1056180013B9FD2A40F2378104F8013F0132C9F875
:10562800002010F8013F11F8017F9F42F0D00AB125
:10563800AB4513D0734824F04FFBAB4508D355F85E
:10564800080B24F049FB092024F03EFB5D45F6D900
:105658006A4824F041FBD9F800200026964291D2EE
:10566800741E444414F8010F24F02EFBD9F80030BE
:1056780001369E42F6D385E703F10802BA421D4679
:10568800B6D01346AFE70C2833D00A2800F0CC80F8
:105698000D2800F0C9807F2800F02581FF2E3FF6F5
:1056A80071AFA0F12003DBB25E2B8ED96AE7544CB0
:1056B8004FF0000B04F598775D4602E00834BC42D1
:1056C8000DD0324621684046FFF718FE0028F5D174
:1056D800A346002DF2D125460834BC42F1D1002D55
:1056E80088D1BBF1000F3FF44DAF464824F0F4FADF
:1056F800A5E7454824F0F0FA404824F0EDFA41E7E0
:10570800DAF80020414B44F80B2CD02202FB053379
:1057180000260193DFF80C8104F8076CA4F10F034D
:10572800009354F80F0CFDF7FDFB00283FF4E4AE9E
:1057380054F80F0CFDF7EEFB14F8023C7BB9242853
:1057480030D0BBF1000FECD1232800F0DA8098F8B4
:1057580032308342E5D1012304F8073CE1E7012B0D
:1057680024D0022B28D0032B00F0B080042B00F0AB
:10577800E880052B00F09780062BD2D114F801CCD5
:10578800BCF1000F00F0F580BCF1010F00F038818A
:10579800002304F8023CD034BC4205F101057FF433
:1057A800A0AEAEE6012304F8023CBAE74D2800F0AB
:1057B800A48004F8026CB4E73C2804F8026C6CD0AE
:1057C8003E28AED10122032304F8012C04F8023C40
:1057D800A7E700BF6C410020643F0020E36200207F
:1057E800EC970020084B002030590020D8570020A3
:1057F8008822002011030008F0830308BC830308F3
:10580800DC670308B4830308C4830308D462002058
:105818002822002058600020045C0020045D00203D
:10582800046903080062002024F0D9FA232187487C
:105838002FF069FE002846D0A0EB0803C9F8003015
:1058480093B15A1E18F80210202940F0F880023B44
:10585800434404E013F80119202956D10246501E8A
:10586800002AF7D1C9F800204FF480720021404681
:105878002FF032FE764B1B78002B3FF442AE754872
:1058880024F02AFA7EE6511C202008F80200C9F804
:10589800001008F801300A46CAE6032304F8016C30
:1058A80004F8023C3DE714F8063C14F8051C14F80B
:1058B800042C994200F29A8090427FF47AAF062332
:1058C80004F8023C5AE7D9F80030B9E7C0283FF697
:1058D80070AF042304F8050C04F8066C04F8040CF3
:1058E80004F8023C1DE7013E00235B48C9F800604C
:1058F80008F8063024F0F0F944E6022304F8023CE4
:105908000FE7022304F8073C0BE7C9F80020534CC3
:10591800002304F5987708F8023003E00834BC4205
:1059280000F08F802168404629F0BCFA0028F5D0A5
:10593800BC4280F08680636898470023C9F800302D
:1059480092E714F8043C04F8030C5840052304F8C3
:10595800040C04F8023CE4E63C4827F049FAD0E598
:10596800324664E63E4A3F4B3F4911603F4ADA609F
:10597800C2E53F4BADF82AC00FCB0DF1300E04AE97
:1059880086E80F004EF824CD14F8051C14F8033CE3
:10599800089404EB010C724631464FF0010E08A83A
:1059A800CDF824C0ADF828308DF82CE00DF03AFB86
:1059B80038B1049A2F4B00983146CDE904321AF0D9
:1059C80035FE039E002304F8023C002E3FF494ADFC
:1059D80054F80F0C1AF0AEFED03454F8DF0CB04770
:1059E800BC4205F101057FF47CAD8AE501991944B3
:1059F8004240013304F8042C04F8063CC87390E6CE
:105A080014F8053C14F8032C0894234409936E2ACF
:105A18004FF00003ADF82E30CDF82A30ADF828202D
:105A28007FF4B6AE08A8FFF743FD08A8FFF734FDDA
:105A380008A8FFF731FD08A8FFF72EFDA8E61A46CB
:105A480065E70D4824F048F977E700BF045C0020BB
:105A58006C410020BC830308EC830308DC6703085F
:105A6800FC9F002000ED00E0EFBEADDE0400FA056B
:105A780058580308FC970020D083030838B504461B
:105A8800006815462FF0C8FC22682A44226038BDF9
:105A9800036810B40A0A5C1C04601A7003685A1C74
:105AA800026019705DF8044B704700BF03685A1C08
:105AB800026010B4197003680A0A5C1C04601A704A
:105AC80003680A0C5C1C04601A700368090E5A1CEF
:105AD800026019705DF8044B704700BF03685A1CD8
:105AE800026019700368090A5A1C0260197070472D
:105AF8002DE9F043002489B006460D461F46A0460E
:105B080005E025290CD030460134A847039A531CD8
:105B1800039311780029F4D1204609B0BDE8F08339
:105B2800931CCDE903385078302842D0A0F13003D7
:105B3800DBB2092B4FF0000945D96C282AD064281C
:105B480073D019D9732858D063D9752840F082804A
:105B580007F1040C386805AB00220A216746FAF7FA
:105B68002FFC05AB049A009329464B463046FAF7BA
:105B78002FFD039A0444CAE725283CD051D9582858
:105B88006BD06328C2D139783046A847043701342E
:105B9800039ABCE7039B5A1C03921B78642B52D0D0
:105BA80016D8252B27D064D9582B18D0632BEAD0C8
:105BB800ADE7D31C03939078A0F13003DBB2092B37
:105BC8004FF00109B9D804AA03A92AF035FEB4E7B1
:105BD800732B12D051D9752B2DD0782B97D1A3F1D7
:105BE8005802B2FA82F23868520905AB102104371C
:105BF800FAF7E6FBB5E7252185E73B68049A0093A9
:105C0800294600233046FAF7E3FC04370444039A94
:105C18007DE76E287FF47AAF039A3B6804371C60EF
:105C280075E700283FF478AF70E7386805A9FAF7F8
:105C380091FB043795E7386805AB00220A21FAF78B
:105C4800BFFB04378DE73B1D386805A91F46FAF7E7
:105C580081FB86E778287FF459AFA0F15802B2FAA1
:105C680082F23868520905AB1021FAF7A9FB04370C
:105C780077E7002B3FF450AF49E76E2BCDD046E7CE
:105C88000EB400B584B005AB019053F8042B064957
:105C9800039301A8FFF72CFF019B00221A7004B0A0
:105CA8005DF804EB03B07047CD0500082DE9F04717
:105CB80007468CB01E469246002A5DD1154614460A
:105CC8000A8840F2B1739A4236D98B78581E0B284D
:105CD80032D891F803C00CF1FF301E282CD891F867
:105CE80004E0BEF1170F27D891F80590B9F13B0FE2
:105CF80022D888793B281FD8B1F80880B8F57A7F70
:105D08001AD24FF001085EBB09890491002CB4BF78
:105D18002D212B21002CB8BF6442CDE90290CDE99A
:105D280005140795CDE900CE38462B49FFF7A8FFA3
:105D380040460CB0BDE8F08700232849ADF828306C
:105D48004FF0010C18468DF82A30ADF82C309946E2
:105D58009E461A4698460991634609A9002ED3D053
:105D6800CDE90290CDE900CE38461D49FFF788FFFE
:105D780040460CB0BDE8F0871A4C84FB0234A318E7
:105D8800D417C4EB6314C4EB0415A2EB85052DB23C
:105D9800002D0846B8BF6D42FFF77EFA4FF47A72BD
:105DA8000023804689462EF0DBFF3C230AFB030ACA
:105DB8004FF47A720023404649462EF0D1FF4FF443
:105DC8007A7192B20023C1FB0A2309A8FAF744FBAF
:105DD80024B209A974E700BF188403080000010170
:105DE800F88303088988888837B51B4B2C3204460A
:105DF80033F8125005F00F0039B1621CC8B10228FF
:105E08008CBF20239C2323701446FCF7F7FEC5F3B0
:105E180003153C23012D1149B0FBF1F191FBF3F27D
:105E280003FB121307D00E49204603B0BDE83040EB
:105E380026E79B23E7E7642542F21071B0FBF1F0F7
:105E4800B0FBF5F105FB1100009006492046FFF76D
:105E580017FF03B030BD00BF4627002040420F00A7
:105E6800BA810308C481030813B5947813780194A0
:105E7800527800920A460249FFF702FF02B010BDAD
:105E8800D381030837B5044608461546FAF79CFC43
:105E9800642190FBF1F301FB13031049642291F88C
:105EA800571090FBF2F2002AB8BF52420028B8BF40
:105EB800524200290CBF0F210C2100910A200849E9
:105EC80093FBF0F30748002BB8BF5B42002D18BFC7
:105ED80001462046FFF7D4FE03B030BD4627002018
:105EE800ED810308E28103080FB430B583B006AB37
:105EF8000B490C4853F8042B096800680193FFF715
:105F0800F7FD094C0546606903685B6998470028F6
:105F1800F9D0284603B0BDE8304004B0704700BF50
:105F2800745600207856002028220020DFED2E7AB3
:105F3800B4EEE70AF1EE10FA4ADDDFED2C6A9FEDC8
:105F48002C7A01E0B0EE670AB4EEC70AF1EE10FA57
:105F580070EE667AF6DC9FED277AF4EEC77AF1EEFA
:105F680010FA3ED5DFED216A9FED237A01E0F0EECD
:105F7800407AF4EEC77AF1EE10FA37EEA60AF6D4B4
:105F8800DFED1E7AB4EEE70AF1EE10FA14DDDFED6C
:105F9800167A37EEC00A60EE006A9FED196A9FED27
:105FA800197ADFED197AA6EE867A20EE266AE6EEF1
:105FB800877AA6EE270A7047DFED147AB4EEE70A6F
:105FC800F1EE10FA44BFDFED0B7A37EEC00AE2E7D4
:105FD8009FED087AF0EE407AF4EEC77AF1EE10FA07
:105FE800C0D4B0EE670ACBE7DB0F4940DB0FC940EE
:105FF800E4CB1641DB0F49C0E4CB16C1DB0FC93F28
:1060080092E741B99730083C15A82ABEDB0FC9BFF3
:1060180009B909E0194690FBF1F301FB130308469F
:10602800002BF7D10846704701460846704700BF65
:10603800DFED317A30EE277AFDEEC76A16EE903A38
:106048002033402B02D99FED2D0A7047B4EEE70AA2
:10605800F1EE10FA4DDD9FED2A6ADFED2A6A01E0C4
:10606800B0EE677AB4EEE67AF1EE10FA77EE467A99
:10607800F6DC9FED257AF4EEC77AF1EE10FA35D505
:10608800DFED1F6A9FED217A01E0F0EE407AF4EE31
:10609800C77AF1EE10FA37EEA60AF6D4DFED167AD3
:1060A800B4EEE70AF1EE10FA1BDCDFED197AB4EE74
:1060B800E70AF1EE10FA44BFDFED137A37EEC00AB3
:1060C80060EE006A9FED136A9FED137ADFED137A95
:1060D800A6EE867A20EE266AE6EE877AA6EE270AEC
:1060E8007047DFED0F7A37EEC00AE9E7B0EE670ACE
:1060F800D4E7F0EE477ABCE7DB0FC93F00000000A9
:10610800DB0FC940E4CB1641DB0F49C0E4CB16C115
:10611800DB0FC9BF92E741B99730083C15A82ABEE2
:10612800DB0F494007EE901AF8EE677A9FED837A05
:1061380027EE800A20EE070AFDEEC07A17EE903AA5
:106148002033402B00F28180DFED7D7AB4EEE70A40
:10615800F1EE10FA40F3E680B0EE407A9FED796AEE
:10616800DFED796A01E0B0EE677AB4EEE67AF1EE37
:1061780010FA77EE467AF6DC9FED747AF4EEC77A79
:10618800F1EE10FA40F1D1809FED6E6ADFED706A92
:1061980001E0F0EE477AF4EEE67AF1EE10FA37EE27
:1061A800867AF6D4DFED6B7AB4EEE77AF1EE10FA80
:1061B80040F3A780DFED627A37EEC77A27EE076AE9
:1061C800DFED655ADFED657ADFED656A9FED655AAB
:1061D800E6EE257A67EE065AE6EE276AF7EE007ACB
:1061E800A5EEA67AF0EE675AE7EE055AE7EE457A8D
:1061F80087EEA55ADFED577A30EE277AFDEEC76AAB
:1062080016EE903A2033402B24D99FED577AF6EEBC
:10621800006AB7EE006AF7EE004AC4EEA57A0023DA
:10622800836143610362C36180ED045A67EEA66A25
:1062380027EE866A27EE877AC0ED006AC0ED026A0B
:1062480080ED016A80ED037A7047B7EE005AF0EEF0
:10625800455ACFE7B4EEE70AF1EE10FA6BDD9FED91
:10626800396ADFED396A01E0B0EE677AB4EEE67AB2
:10627800F1EE10FA77EE467AF6DC9FED347AF4EE1A
:10628800C77AF1EE10FA53D59FED2E6ADFED306A2A
:1062980001E0F0EE477AF4EEE67AF1EE10FA37EE26
:1062A800867AF6D4DFED2B7AB4EEE77AF1EE10FABF
:1062B80033DCDFED2E7AB4EEE77AF1EE10FA44BF64
:1062C800DFED227A37EEC77A27EE076ADFED224A3A
:1062D800DFED226ADFED227AE6EE246A67EE064AEF
:1062E800E6EE267AB7EE006AA4EEA77AF6EE006A22
:1062F80036EE476AF8EE007A27EE277A66EE266AC7
:1063080089E7DFED1A7AB4EEE77AF1EE10FA44BFC6
:10631800DFED0E7A37EEC77A50E7DFED097A37EE10
:10632800C77AD1E7F0EE407A26E7B0EE677A39E728
:10633800B0EE677AB6E7F0EE477A9EE727D4D23612
:10634800DB0F4940DB0FC940E4CB1641DB0F49C0E6
:10635800E4CB16C1DB0FC93F92E741B99730083C3F
:1063680015A82ABEF304353F00000000DB0FC9BFA3
:1063780070B406688E4217D90139751E002311F8CA
:10638800014F0822634013F0800F4FEA430318BF00
:1063980083F0D503013ADBB2F5D18D42EFD1721CFF
:1063A8000260337070BC7047721C00230260337047
:1063B80070BC704710B44C09012250F8243001F029
:1063C8001F0102FA01F10B4340F824305DF8044B39
:1063D800704700BF4B0901F01F0150F8232001232B
:1063E80003FA01F1114214BF18460020704700BF9C
:1063F8005FEA930CF0B433D04FEA0C1C00F11004A0
:1064080004EB0C0701F1100602F1100514ED046A03
:1064180056ED044A54ED026A14ED037A54ED017AFC
:1064280016ED025A56ED035A26EE246A66EE856A80
:1064380005ED046A16ED016A45ED026A27EE257A34
:1064480067EE867A1034BC4205ED037A45ED017A91
:1064580006F1100605F11005D8D160446144624484
:1064680013F003030BD000EB8303F0EC017AB1ECDB
:10647800017A67EE877A9842E2EC017AF5D1F0BCAE
:10648800704730B585B0054601A8FEF7E1FE044621
:1064980018B92870204605B030BD044A0123B2F966
:1064A800002001A92846FFF701FCF3E73833002054
:1064B8002DE9F04FA94E36F81040074614F4006055
:1064C8008FB000F01D8207F01F0201239340790965
:1064D800A34A52F82120134204D0A24B1B78002B68
:1064E80040F0D5831C2200210DEB020004F01F05AB
:1064F8000691C4F344142EF0EFFF262F00F2C78351
:10650800DFE817F027003C0086018E01D6018E00D7
:106518008E00D400F8001001680156006700C5031A
:10652800C503880001020802100218022602300280
:106538009002C503C503AA02FA02FA021603510320
:10654800C503C50365037D036F009803B603940074
:10655800C103854B85491A88642353439B12632BD7
:10656800A8BF6323012206A8FFF78AFB804806AB71
:10657800224629460068FDF73FFA97E17D4B1E88C1
:106588007D4B0A2101FB06F01B7890FBF3F0FAF72C
:1065980029F9B6FBF1F201FB126306218DF8180008
:1065A80000919BB275490DF11900FFF769FBDDE712
:1065B800734B1B68002BB8BF5B4264219A2093FB86
:1065C800F1F2009001FB123306A86E49FFF758FB61
:1065D800CCE76B4A6C499268072306A8FFF750FB83
:1065E800C4E76A4B0A22B3F9043093FBF2F31B01A8
:1065F80003F5B9534FF4B4721433B3FBF2F3644A9E
:1066080003F00F03134406AA186859681B7A03C2DB
:106618001370ABE70122002106A8FFF733FCA5E7BA
:106628007A1F012106A8FFF7DFFB9FE7544B9FED78
:10663800597A9A68B6F8523007EE902AF8EEE76A67
:1066480007EE903AF8EEE77A67EE877AF4EEE76AB3
:10665800F1EE10FA04D5504906A8FFF711FB85E7BB
:10666800934204DA4D4906A8FFF70AFB7EE79B1A16
:1066780007EE903A4A4B4B4AB8EEE77AD3ED007AE8
:10668800F8EE677A3C2167EE277A06A887EEA67AA5
:10669800FDEEC77A17EE903AB3FBF2F393FBF1F2F3
:1066A80001FB12334049FFF7EBFA5FE73F4B1B88CA
:1066B8005A0504D53E4906A82EF032FF56E7DF07F3
:1066C80004D53C4906A82EF02BFF4FE79E0704D5BA
:1066D800394906A82EF024FF48E726F0DDFF20B14F
:1066E800364906A82EF01CFF40E7354906A82EF0CB
:1066F80017FF3BE733490A7806AE22B932493046DC
:106708002EF00EFF32E70022885C28B1FEF736FE35
:10671800B0540132102AF7D10EAB1A44002302F804
:10672800203C23E740F20453ADF81830274B2849A2
:10673800B3F90620B2F5FA6FA8BF4FF4FA62B2F5C2
:106748007A7FB8BF4FF47A720A23A2F57A720DF1F4
:106758001A0092FBF3F2FFF793FA07E746270020A7
:1067680010270020000000207E3F0020F78103084A
:10677800B05600208C40002044430020FD810308CF
:106788007840002007820308128203084C43002047
:1067980068580308CDCCCC3D188203081E82030834
:1067A8002822002040420F00BA810308E040002060
:1067B80024820308298203082E82030833820308EF
:1067C800388203083C3300203D820308B84000208B
:1067D800DE810308A849A94A0B78D65CA84B4A78F9
:1067E80053F822708B788DF81730A64B186828B1AB
:1067F8000B7A1BB10DF1170106F081FB9DF81730DC
:10680800009332463B46A04906A8FFF739FAADE6A1
:1068180047F62663ADF8183027238DF81A30A5E619
:1068280096F85F20994996F85E30B1F9000002EBBE
:1068380082025200574203EB8303B8424FEA4303F4
:1068480003DB9042A8BF10460746B1F9022059421F
:106858008A4203DB9A42A8BF1A46114619224A43C4
:106868004FEA870892FBF3F36FF00306A3F1290BB5
:106878004FF040094FF0090A98FBF9F3A3EB0B031B
:10688800512B0ED893FBFAF202EBC2015B1A804837
:10689800803B2244A919DBB2D2B2C9B20068FDF725
:1068A800A1F80136052EA8EB0708E5D1012027E05D
:1068B800A5F10709764E6FF002075FFA89F904EB34
:1068C80007085FFA88F81323424649463068FDF7FF
:1068D80089F8013713234246E91D3068FDF782F82D
:1068E800042FECD1A91F03232246C9B23068FDF753
:1068F80079F802232246A91D3068FDF773F80120B4
:106908000FB0BDE8F08F634B63491A6806A8FFF71C
:10691800ABFA2BE65F4B61491A6806A80332FFF70A
:10692800A3FA23E65B4B5E491A6806A80632FFF70E
:106938009BFA1BE65B4B5C491A885C4B1B6806A8F4
:1069480053434FF47A7293FBF2F2FFF799F90DE68D
:10695800574A5849537812780133013206A8FFF78D
:106968008FF903E6B6F85C60534B30071F7806D5FD
:10697800022F04D1514906A82AF062F8F6E5B106BB
:1069880007D54F4B1B7823B14E4906A82AF058F873
:10699800ECE5F20717D5002026F08CFE98B14A4B9B
:1069A8001A6882B10023012101FA03F0104206D0CF
:1069B800464A06A852F823102AF042F8D6E50133D1
:1069C800122BF1D1D2E5730706D5012F04D1404926
:1069D80006A82AF035F8C9E5B00713D53D4B1B7852
:1069E80099070FD477B93C4A2E4B11783B4A1B883C
:1069F800927B93FBF1F39A4204D9394906A82AF00D
:106A08001FF8B3E5F20608D5364B93F8AC3023B13E
:106A1800354906A82AF014F8A8E5002106A82AF0A6
:106A28000FF8A3E51F4B1B880A2159432A4B1B78F3
:106A380091FBF3F10846F9F7D5FE64238DF81800A9
:106A4800062091FBF3F2009003FB12130DF11900DD
:106A58002649FFF715F989E52549B1F90600B1F985
:106A68000230B1F900200190B1F90410009106A894
:106A78002049FFF705F979E5D43F0020CC5F0308EA
:106A8800D45F0308C83F0020488203084C43002015
:106A9800B056002090430020528203085682030813
:106AA8005A8203088C4000205E8203087840002048
:106AB800EC97002063820308813F00206982030865
:106AC8003050002073820308B83F0020187703086D
:106AD8007E820308643F002044430020843F002056
:106AE8008A8203082822002096820308809B0308D4
:106AF800643D0020A0820308664B1A2F0CBFB3F92F
:106B08000200B3F900000A21002890FBF1F301FB11
:106B18001301ACBF20222D220029B8BF4942002B07
:106B28000091B8BF5B425C4906A8FFF7A9F81DE5CC
:106B38005A4B1A895A4B9B68D31A9342A8BF1346DB
:106B480023EAE37307EE903A0B23B2FBF3F300EE6C
:106B5800103AF8EEE77AB8EEC00A87EE800A2EF00F
:106B680029FD0EA98A2201F8202D0122FCEEC07A07
:106B7800CDED037A9DF80C309342B4BF8D208B2065
:106B8800505401320C2AF7D18F228DF824205A1E36
:106B9800092A04D80EAA13448E2203F81F2C0023B6
:106BA8008DF82530E2E43F4B1B78DB0704D43E49DF
:106BB80006A8FFF765F8D9E43C4B93F8AD30002BF5
:106BC8007FF4D4AC3A4906A8FFF75AF8CEE4314B23
:106BD8000A22B3F9043093FBF2F31A0102F5B95211
:106BE8004FF4B4711432B2FBF1F2C2F1080202F0B0
:106BF8000F0260322F4906A8FFF742F8B6E40020DA
:106C0800F9F7E2FD64210A2290FBF1F301FB13017D
:106C180091FBF2F10029B8BF4942002B0091B8BF9F
:106C28005B4225490028ACBF6822602206A8FFF70E
:106C380027F89BE41D4BD3F8B03093F9011096F870
:106C4800573001EB8102510033B901EB02110522E3
:106C580091FBF2F101F5A071002B0CBF46234323F1
:106C68000A2206A891FBF2F21449FFF709F87DE41D
:106C78000E4BD3F8B0200AB1B2F90820104906A883
:106C8800FEF7FEFF72E406A8FFF7FBFB6EE40020A8
:106C980036E600BF4C430020B4820308843F00203E
:106CA80078400020643F0020C0820308282200208A
:106CB800C9820308D2820308D9820308E58203083F
:106CC800B08203082DE9F04F9F4BA04C1B788DB084
:106CD800814613B1012384F8AC30D4F8B4200523DD
:106CE800B2FBF3F303EB8303D21A40F0E581984E2D
:106CF80098493378087803F00103984288461FD0F2
:106D0800002B00F089804FF4C6034FF0FA75C4E9F0
:106D18000253914D626028682261FCF7ADFE8F4BEB
:106D2800286807220C21FCF767FE09F5F4238C4A32
:106D380003F590731360337803F0010388F800308B
:106D4800B4F90830B4F90A208649B4F90C00002BCC
:106D5800BCBF00232381844B1B889A42C8BF638130
:106D68000A68642392FBF3F212B29042B8BFA28180
:106D78007E4A12885343B4F90E20C3F387239A42FC
:106D8800C8BFE38184F8B830B4F91030002BBCBF19
:106D9800002323823378DA07884609D5D4F8BC3033
:106DA8002268A9EB03031A442260626813446360F3
:106DB8006B4FC4F8BC903B68674D3946002B42D0F6
:106DC800A9EB0303002B286839DA694AB2F906509F
:106DD80040F2D6639D4203DCB2F902209A4201DDFB
:106DE80000230B60FCF7FAFD002384F8AC30D4F8DC
:106DF800B4300133C4F8B430574B1B6823B193F94E
:106E08000E30002B00F35E815A4A136823F4804346
:106E180013600DB0BDE8F08F574A1746991891F8DE
:106E28006010002940F0588101330D2BF6D182E71C
:106E3800032577E1514904A8FEF722FF93E2FCF706
:106E48001BFE00233B604E4B4E4FB9FBF3F94E4BF4
:106E580009F0010983F800903B681B0104D5FF2065
:106E680015F038FCC4F8B0002B6823B193F90E3044
:106E7800002B00F31B810020F9F7A6FC434A3E498A
:106E8800136891F856C09246414A814694F8B80072
:106E9800127884458B468CBF43F0010323F001032D
:106EA800002A3AD123F4C00323F00203394A1278A6
:106EB800900745D443F48043CAF80030BBF85830F3
:106EC800039303F00F00FBF799FE039B324A1B0A5A
:106ED8005A4327D1DAF8003023F02003CAF80030EB
:106EE800BBF85A30039303F00F00FBF787FE039BB0
:106EF800294A1B0A5A431CD1DAF8003023F0400310
:106F0800BBF85200D8F80810DAF80420884245DDAA
:106F180023F0102322F0200244E043F4C00343F09E
:106F28000203C3E79042DAF80030D3D343F02003DA
:106F3800D4E78242DAF80030DED843F04003DFE7D6
:106F480023F48043B8E700BFBC3F0020282200207C
:106F5800643F0020B4560020B0560020C3820308C6
:106F680018270020784000208C4000207E3F002019
:106F7800B8400020B83F0020462700206F83030850
:106F8800400D0300A06B0020000000201027002007
:106F9800813F0020213300200087930343F0102312
:106FA80042F02002CAF80420642299FBF2F9BBF8E7
:106FB800542028689145ACBF43F4004323F40043B0
:106FC800CAF80030FCF758FD152026F073FB00289E
:106FD80069D13F4B1B68990702D50320FFF768FA70
:106FE8000120FFF765FA0020FFF762FA0220FFF799
:106FF8005FFA0420FFF75CFA0520FFF759FA06202C
:10700800FFF756FA2520FFF753FA0720FFF750FA43
:107018000920FFF74DFA0A20FFF74AFA0B20FFF77D
:1070280047FA0C20FFF744FA0820FFF741FA0F202F
:10703800FFF73EFA1020FFF73BFA1120FFF738FA66
:107048001220FFF735FA1320FFF732FA1420FFF762
:107058002FFA1520FFF72CFA1620FFF729FA192026
:10706800FFF726FA1A20FFF723FA1B20FFF720FA6A
:107078001C20FFF71DFA1D20FFF71AFA2020FFF742
:1070880017FA2120FFF714FA2220FFF711FA3B68BC
:107098001A0105D52320FFF70BFA2420FFF708FA79
:1070A8002620FFF705FA2868FCF798FC337803F0E8
:1070B800010384F8AD3097E6064B18680368DB686F
:1070C800984794E64FF480400BF0A4FFA1E600BF78
:1070D80048430020B0560020B44B1B689B0603D5DC
:1070E800538D18053FF527AEB14D2868FCF7C4FC51
:1070F8000222B04B28681146FCF77EFC97F86C30EA
:10710800002B3FF495AE04A8FFF7BBF918B9AA49BC
:1071180004A8FEF7B5FD286804AB03220221FCF79A
:107128006BFC042597F86830A3B10022114604A827
:10713800FEF75AFEB7F85830A04903F00F03284667
:1071480004AA51F8231005F1010AFCF76BFC5FFA59
:107158008AFA554697F86930A3B10122002104A89C
:10716800FEF742FEB7F85A30944903F00F03284659
:1071780004AA51F8231005F1010AFCF753FC5FFA41
:107188008AFA554697F8603093B18D4B1B7899076A
:107198000ED504A9B4F9080029F071FB284604AA01
:1071A800884905F1010AFCF73DFC5FFA8AFA554661
:1071B80097F86A30C3B1B4F91200F9F705FB97F8EC
:1071C80057308149002B02460CBF0F230C2304A81B
:1071D800FEF756FD284604AA7C4905F1010AFCF78A
:1071E80021FC5FFA8AFA554697F86130BBB1B4F9C9
:1071F8000A100A2391FBF3F203FB121306210091F4
:107208001BB2734904A8FEF73BFD284604AA71493E
:1072180005F1010AFCF706FC5FFA8AFA554697F869
:107228006730BBB16C4B19880A23B1FBF3F203FB3F
:107238001213062100919BB2654904A8FEF720FDB0
:10724800284604AA654905F1010AFCF7EBFB5FFA39
:107258008AFA554697F8623093B104A9B4F90E003A
:1072680029F00DFB5E4904A82EF03EF9284604AA31
:107278005C4905F1010AFCF7D5FB5FFA8AFA554625
:10728800594B9B794BB397F8633093B104A9B4F980
:107298000C0029F0F4FA554904A82EF025F92846DF
:1072A80004AA534905F1010AFCF7BCFB5FFA8AFA04
:1072B800554697F8643083B14E4A4349926807238C
:1072C80004A8FEF7DDFC284604AA4B4905F1010A8B
:1072D800FCF7A8FB5FFA8AFA554697F865307BB148
:1072E8000022B4F9101004A8FEF7CCFD284604AA21
:1072F800424905F1010AFCF795FB5FFA8AFA5546FF
:1073080097F86630002B38D03D4B9B78002B34D053
:10731800032B32D0022B7FF48DAD13F067FA0028CF
:107328003FF488AD374A92F82430002B3FF482AD01
:10733800354B597803297FF47DAD916A4FF4FA6291
:10734800B1FBF2F141F2781204A89A584FF47A236B
:10735800B2FBF3F28B1A64225A43B2FBF1F22B49C7
:1073680092B2FEF78DFC284604AA294905F1010AC4
:10737800FCF758FB5FFA8AFA554697F86B3073B1F9
:107388001F4B9B785BB1032B09D0224B04A91869CA
:1073980029F075FA04AA20492846FCF743FB002384
:1073A80063601E4B1E4A4B441360C4E4B83F002080
:1073B800B0560020EB820308FB820308805C0308B8
:1073C80021330020028303080C8303081183030878
:1073D8001E830308278303088C4000203383030897
:1073E8006D8303083F830308843F00203E9B030806
:1073F8004883030878400020548303085D8303080A
:10740800A82900203C620020C48500206A83030864
:1074180075830308C42900207E830308008793032B
:107428001827002008B540F2E93300E09BB1028933
:10743800013B12F0020F9BB2F8D0017340F2E9331E
:1074480000E043B10289013B12F0010F9BB2F8D072
:10745800007BC0B208BDFCF727FBC0B208BD00BF67
:10746800F8B584894FF6FF764FF47A742BB311B3CD
:107478000F78013101E0B44217D00589013CAD070E
:10748800A4B2F8D507734FF47A7402E0BCB2B442E0
:107498000BD00589ED0704F1FF37F7D5057BEDB271
:1074A8000AB115700132013BE0E7FCF7FDFA003044
:1074B80018BF0120F8BDFF27DFE70120F8BD00BF96
:1074C800028822F040021204120C0280038823F082
:1074D80038031B041B0C69B141F48071002991FA2F
:1074E800A1F1B1FA81F108BF4FF0FF31013943EA48
:1074F800C1039BB20380038843F0400303807047B5
:107508002DE9F84FDFF8C4902D48DFF8C4A02D4FBF
:107518000421FFF7D5FFD9F80000FCF7EFF80521A3
:107528002748FFF77FFF00212548FFF77BFF06214B
:107538002348FFF777FF00212148FFF773FF9AF8E8
:1075480000401F48042144F00104FFF76BFF214667
:107558001B48FFF767FF3B88B3B1DFF878801A4D07
:10756800174E444615F801BF07213046FFF75AFF6A
:1075780059463046FFF756FF2B7804F8013B3A8806
:10758800A4EB08039A42EDDC07210D48FFF74AFFF8
:10759800FF210B48FFF746FF9AF8004008480421EE
:1075A800FFF740FF21460648FFF73CFFD9F80000E7
:1075B800FCF7AAF802210248BDE8F84F80E700BFAF
:1075C80000300140180000202723002054650020C7
:1075D8000C30002030250020F8B5114D114FC1F1B5
:1075E800030646EA800604212846FFF769FF386843
:1075F800FCF784F8F6B21024E1B22846FFF712FF30
:10760800013431462846FFF70DFF202CF4D13868A5
:10761800FCF77AF802210248BDE8F84050E700BFBD
:107628000030014054650020F8B5414C4148042120
:10763800FFF746FF2068FCF761F83F4B1B78012BEA
:107648006CD057D3022B49D13C4D08232B704FF4F3
:10765800C3733B4E3B4F338002210020FFF7BCFF32
:1076680004213448FFF72CFF2068FCF747F82D78F1
:1076780030480021FFF7D6FE29462E48FFF7D2FEF4
:10768800314B2C481D780221FFF7CCFE29462948AA
:10769800FFF7C8FE2D4B27481D780321FFF7C2FED0
:1076A80029462448FFF7BEFE294B22481D780421AD
:1076B8000D43FFF7B7FE29461E48FFF7B3FE2068C3
:1076C800FCF722F802211B48FFF7FAFE328821480E
:1076D80000212DF001FF7B783BB9F8BD174D2B78C1
:1076E8005B06B4D54FF4F073B3E7FFF709FF002347
:1076F8007B70F8BDA0210F48104DFFF793FE0021C5
:107708000C48FFF78FFE00F00603022B03D000F0B1
:107718000500012808D008232B7098E7074D482357
:107728002B704FF4F07394E748232B70DAE700BF0F
:1077380054650020003001405865002011020020E7
:1077480018000020000000205F6500206065002010
:107758000C300020302500202DE9F047444C4548E6
:10776800454D464E0421FFF7ABFE2068FBF7C6FFE8
:1077780080214048FFF756FE00213E48FFF752FEA1
:1077880007462068FBF7C0FF02213A48FFF798FE3A
:107798002B78D6F80080BB420DD1394B1F7847B9FA
:1077A800DFF8E490D9F8C030A8EB0303B3F57A7F8B
:1077B80004D8BDE8F087BDE8F04735E704212D4837
:1077C800DFF8C8A0FFF77CFE2068FBF797FFA02131
:1077D8002848FFF727FE39462648FFF723FE0746C5
:1077E8002068FBF791FF02212248FFF769FE9AF80B
:1077F8000030182B0CD12B78224A03F04003002BC1
:1078080007F007010CBF0D20102013805180D08095
:10781800790706D50023C9F8C430C9F8C080BDE887
:10782800F08707F00507012F1AD0002FF5D12B7824
:107838005B06F2D5D9F8C430B3B13268D31A642BD9
:10784800EBD9FFF7F1FE9AF80030182BE5D1B9F81B
:10785800C8300C4A01339BB2A9F8C8309380DCE7E2
:107868002B785A06E6D5D8E73368C9F8C430D4E788
:1078780054650020003001401102002058600020AB
:1078880058650020643D002028220020603D00202B
:10789800074A00235168814202F11C0204D00133D7
:1078A8000C2BF7D100207047581CC0B2704700BF9E
:1078B800D020002000F1FF3C4FEACC002DE9F04336
:1078C800A0EB0C04A400374FDFF8FCE03E59364D1E
:1078D800DEF81490DFF8F4803C44AE420CBF012679
:1078E8000226656846EA09064545CEF8146083B065
:1078F800A16023613ED02D4B9D423DD014339D4263
:107908003CD014339D4232D014339D4239D01433C5
:107918009D4239D014339D4239D003F562739D429C
:107928003AD014339D4239D014339D4232D01433A7
:107938009D4235D01E491F4B8D420CBF1D46002568
:10794800A0EB0C0007EB80009209447B85610021C5
:10795800012301A88DF804408DF805208DF8061044
:107968008DF8073013F0A2FC03B0BDE8F0834FF4A4
:107978000055E5E70225E3E72025E1E74FF4007528
:10798800DEE74FF40035DBE74FF40015D8E74FF09A
:107998000075D5E7084DD3E7084DD1E7084DCFE787
:1079A800084DCDE7D0200020000002401C00024016
:1079B80058040240000002100002001002000010EB
:1079C80020000010002000100010024008000240B3
:1079D8000138C0EBC000094B8000F0B4084D1C58BA
:1079E800084F6E691844BC420CBF0123022333437D
:1079F8006B6101754275F0BC704700BFD020002054
:107A080000100240000002402DE9F04F534C54F89A
:107A1800204083B0002C5DD0A56DA1601F466B6827
:107A2800236504F15E0363618023C4E90333904650
:107A38004B4A226004F1DE02A2618146287E28F0CA
:107A4800C1F8E86860B1FFF723FF09F10102D2B27B
:107A58000C21FFF7BDFF236DEA6862632433E364FA
:107A6800A86898B1FFF714FF09F101020646D2B2DF
:107A78000B21FFF7ADFF2346EA7E3A493046FFF770
:107A880019FF236DAA68A2632833A36494F85D00E4
:107A9800FAF730F9064694F85C00FAF72BF93A073A
:107AA800824695F819B019D5C6B117F0110F4FF0E5
:107AB8000B0309F10100F07114BF4E213E21B3718F
:107AC8005A463046F9F7E2FDFB0743D5636B6BB3C3
:107AD800A36B5BB3204603B0BDE8F08F17F0010F2E
:107AE8000CBF2E274E2718F0020F0AD04EB10B22DA
:107AF80009F10103B271F37130465A463946F9F774
:107B0800C5FD18F0010FE1D0BAF1000FDED00C234B
:107B180009F101008AF807008AF806305A46394602
:107B28005046F9F7B3FD636B002BD1D12B7FAA7EAA
:107B38008DF804209B090021012201A88DF8053049
:107B48008DF806108DF8072013F0B0FB204603B01F
:107B5800BDE8F08F3046FBF7D1FDB7E7805600202F
:107B6800805803084108000800B97047F0B595B07F
:107B7800064628F08DFA644DC36802682A600446F8
:107B8800002B00F0AD803046FAF7B4F85F4BC3F82D
:107B9800CC0018B1292200238271C371227A5C4E6D
:107BA8002E21F9F773FD2868FAF712FE28F00AF873
:107BB8002868584A038823F001031B041B0C038020
:107BC8000F211E233380118000262D23012701A9B0
:107BD800CDE90173039628F00CFAE3790596602243
:107BE80004929A07CDE9066608967BD5DB0003F078
:107BF80008030422ADF81E30ADF81620002304AAAD
:107C0800617928680693F9F737FB2868617928F0C5
:107C1800D1F92868436C43F400434364038843F074
:107C280080030380E3799B0768D56179026A04239E
:107C38008B4022EA03020262026A134303622A6843
:107C4800354F138843F001031380207C002229213B
:107C5800FFF7BEFE3149207C00236022FFF72AFE91
:107C6800E068386013F05CF9386803684FF6FE7214
:107C78001340036013F054F909A813F023F92B6893
:107C88006279274938680A9134331344099380226A
:107C98001023002609A940F22A3C0E920B934FF4B8
:107CA80000724FF400530D961096139611960F928A
:107CB8001293ADF830C013F013F962792B680C2ACF
:107CC80098BF1849D86898BF31F812603A681649C1
:107CD8000643DE601368012043F002031360087056
:107CE80015B0F0BD5B0003F002034FF48072ADF8ED
:107CF8001C30ADF81470ADF820207FE701226179BF
:107D080013F00AFB9BE700BF143300202822002051
:107D18000633002004330020103300208D090008AA
:107D2800F4440020847D03080C3300200348D0F875
:107D38003C3113B100F59A7018477047D0200020E5
:107D48000348D0F8203113B100F58C7018477047FC
:107D5800D02000200348D0F804310BB1FC3018477C
:107D6800704700BFD02000200348D0F8E8300BB19E
:107D7800E0301847704700BFD02000200348D0F8F3
:107D8800CC300BB1C4301847704700BFD02000205A
:107D98000348D0F8B0300BB1A8301847704700BF7F
:107DA800D02000200348D0F894300BB18C3018470D
:107DB800704700BFD02000200248836F0BB170309D
:107DC80018477047D02000200248C36D0BB15430CB
:107DD80018477047D02000200248036C0BB1383098
:107DE80018477047D02000200248436A0BB11C3066
:107DF80018477047D02000200248836803B118470D
:107E0800704700BFD0200020038903F4C0530BB192
:107E1800012070470089C0F3C0107047F8B505010C
:107E2800594C5A4B625961199A4204EB050704BF31
:107E380001230B730646387A27F0C4FE3B7A03F019
:107E48001F015B090122022B02FA01F275D0032BF4
:107E58006ED0012B64D0631901361879F9F74AFFFF
:107E6800F6B2074610B11223C671837163195879A7
:107E7800F9F740FF10B11323C6718371631998791C
:107E8800F9F738FF10B11423C671837166190E21F2
:107E9800F2793846F9F7FAFB7079F9F72BFFF2799E
:107EA8000E21F9F7F3FBB079F9F724FFF2790E21E7
:107EB800F9F7ECFB6359364A934243D0334A93426D
:107EC80056D0344A934248D02C44227B6ABB0121C5
:107ED80002209A8822F480521204120C9A809A88FE
:107EE80042F480529A801A8802F4415242F4457250
:107EF8000A4302431A809A8822F470621204120C10
:107F080042F4E0629A809A8B22F400621204120C06
:107F180007219A8319821A8842F040021A80F8BD14
:107F28001D4B996A0A439A6295E700210846D0E7F3
:107F3800194B19690A431A618DE7174BD9680A4327
:107F4800DA6088E702F56042D16841F48051D16077
:107F5800D16821F48051D160B6E702F5EA3211699F
:107F680041F400411161116921F400411161ABE74D
:107F780002F5EC32116941F480411161116921F473
:107F880080411161A0E700BFA462002000380040D2
:107F980000300140003C0040001002401749184BD7
:107FA800184A194810B4D1F8884044F47004C1F84C
:107FB80088401C6844F001041C605C6822405A60D8
:107FC8001A6822F0847222F480321A601A6822F445
:107FD80080221A605A6822F4FE025A60DA6A22F095
:107FE8000F02DA621A6B002410404FF00062186327
:107FF8009C608A605DF8044B704700BF00ED00E0AC
:10800800001002400CC07FF8CCFC00FF027A407AD6
:1080180002FB00F0704700BF027A407A02FB00F0D2
:10802800704700BF0020704700207047012070474C
:10803800002070474FF0FF30704700BF00207047A6
:108048000F4B10B41C8894B10E4A117892F808327C
:10805800994210D11444531C02F5027205E013F83A
:10806800011B12F8010F884205D1A342F7D1012064
:108078005DF8044B704700205DF8044B704700BF63
:108088001800002028230020002070471E2000FB35
:108098000212024900208B54704700BF2823002099
:1080A80030B41C7874B11E25084815FB021202442E
:1080B800C91AC8181D28D8BF147013F8014F013207
:1080C800002CF6D1002030BC704700BF28230020C8
:1080D800014B1888704700BF18000020084B094959
:1080E800D3F8E803D3F8EC23014022F02002002063
:1080F800C3F8E813C3F8EC23C3F8F003704700BFD4
:10810800282300209C2F9FEF002302220271037076
:1081180043708370C3707047437913F0020308D02B
:108128000369D0E90920013B101A1840C0B2181A97
:1081380070471846704741717047704743799B07ED
:108148000AD5436A8269D154436A01690133B3FB92
:10815800F1F201FB123343627047437913F00103D4
:1081680006D0D0E90732C0689B1A0138184070471A
:108178001846704710B5437913F0010301460ED035
:10818800FFF7EBFF50B10B6A4A69CC68D05C01334A
:10819800B3FBF4F204FB1233C0B20B6210BD1846F5
:1081A800FCE790F8473830B53BB990F8451890F897
:1081B80046380124DAB2914200D830BDB0F84E58A2
:1081C80004FA03F22A43A0F84E280133F2E7D0E973
:1081D8000920131A584258417047034B9A780AB934
:1081E80001229A700020704718000020074BDA78A7
:1081F80052B11B7943B103EBC203093B044A32F87D
:108208001320044BA3F8F423704700BF1800002084
:10821800205F03082823002008B5174B1B780BB1F3
:10822800164AD370164B1B780BB1144A1371FFF71B
:10823800DDFF144B144A1B78013382F8F633134BD5
:108248001B887BB1192B0FD9642B0FD9C82B0FD9D9
:10825800B3F5C87F0ED9B3F5167F03D80423074AB0
:1082680001339370002008BD0023F8E70123F6E7E7
:108278000223F4E70323F2E7093D00201800002059
:108288000A3D0020043D002028230020063D002050
:1082980008B5054B1A791AB901221A71002008BDD0
:1082A800FFF7A4FFFAE700BF1800002008B5054B48
:1082B800DA781AB90122DA70002008BDFFF796FFB4
:1082C800FAE700BF18000020064B1A78064B1B7807
:1082D80003EBC203093B054A32F81320044B1A800A
:1082E800704700BF5E4100205F410020205F030807
:1082F800604100200A4B93F8F7230A4B5AB10A4A07
:10830800127822B903F114021A610020704703F1B0
:10831800DC021A61F9E703F5BE721A61F5E700BFDE
:10832800282300201800002066410020034BB3F8E2
:10833800F823034B4FF0FF301A80704728230020A2
:1083480064410020034B1A88034B0020A3F8F8234C
:10835800704700BF6441002028230020074B93F991
:108368000030012B06D0064BB3F8FC23A3F8FA2300
:10837800002070474FF0FF30704700BFE81A002018
:108388002823002008B5064B1A782AB1054A127826
:10839800012A1CBF00221A70FFF7ACFF002008BD9D
:1083A800664100205C410020064B93F90020064BF3
:1083B80012B91A70002070471A78002AFAD10122DF
:1083C800F7E700BFE81A002062410020104B114A6D
:1083D80093F8FE13517193F8FF13917193F80014F9
:1083E800117093F8042483F80124B3F80A24A3F83D
:1083F8000624B3F80C24A3F80824B3F81224A3F82D
:108408000E24B3F81424A3F810240020704700BFEA
:1084180028230020843F0020104A114B517983F80B
:10842800FE139179127883F8002493F8012483F8D5
:108438000424B3F80624A3F80A24B3F80824A3F8FC
:108448000C24B3F80E24A3F81224B3F8102483F8EC
:10845800FF13A3F814240020704700BF843F0020B6
:1084680028230020074B93F81B2483F8182493F83B
:108478001C2483F8192493F81D2483F81A24002057
:10848800704700BF28230020074B93F8182483F86F
:108498001B2493F8192483F81C2493F81A2483F8CE
:1084A8001D240020704700BF28230020104B93F89C
:1084B8008C2493F88E1402F00F0242EA012293F8FA
:1084C80090140901C9B20A43A3F8762493F88D24BD
:1084D80093F88F1402F00F0242EA012293F89114E4
:1084E8000901C9B20A43A3F878240020704700BFE5
:1084F800282300200E4BB3F8762402F00F0183F8EE
:108508008C14C2F30311120A83F88E24B3F878246A
:1085180083F8901402F00F0183F88D14C2F303114D
:10852800120A83F8911483F88F240020704700BF43
:1085380028230020074B93F8922483F87424B3F877
:108548009424A3F87024B3F89624A3F87224002086
:10855800704700BF28230020074B93F8742483F842
:108568009224B3F87024A3F89424B3F87224A3F8DF
:1085780096240020704700BF2823002008B505482E
:10858800522200F5936100F21E402CF045FF0020B6
:1085980008BD00BF2823002008B50548522200F274
:1085A8001E4100F593602CF037FF002008BD00BF86
:1085B80028230020084A0949B2F8EA340B8292F8C5
:1085C800EC3492F8ED2403EB83035B00CB81044B7E
:1085D80000209A70704700BF28230020A06D00205B
:1085E800EC970020084A094B118AA3F8EA14D289AB
:1085F8000A21B2FBF1F283F8EC24054A927883F859
:10860800ED240020704700BFA06D00202823002023
:10861800EC97002030B1007910F1FF3018BF4FF00F
:10862800FF3070474FF0FF307047074B93F8EE2448
:1086380042B9064A528802F0010283F8EF24012267
:1086480083F8EE240020704728230020A06B002028
:10865800034B002083F8F00483F8F104704700BF4F
:1086680028230020084B094A1B68B2F8F214198421
:10867800B2F8F4145984B2F8F614B2F8F8249984CC
:10868800DA830020704700BF904300202823002091
:108698000B4B93F8FA244E2101FB02320020B2F86A
:1086A8001C15A3F8F214B2F81E15A3F8F414B2F8C6
:1086B8002015B2F81A25A3F8F614A3F8F824704781
:1086C80028230020094A0A4B92F8E6155971B2F896
:1086D800E8159981B2F8EA15D981B2F8EC15B2F823
:1086E800EE2519825A820020704700BF28230020F7
:1086F800A0670020094A0A4B517983F8E615918949
:10870800A3F8E815D189A3F8EA15118A528AA3F8C3
:10871800EC15A3F8EE250020704700BFA0670020E5
:1087280028230020144B154993F8F025303281F89E
:10873800E12193F8FA244E2101FB0232002092F83D
:10874800331583F8F11592F8321583F8F21592F87B
:10875800111583F8F31592F8121583F8F41592F8A9
:10876800131583F8F515B2F83015B2F82E25A3F8CD
:10877800F615A3F8F82570472823002018000020D4
:108788000E4B0F4993F8F025303281F8E42193F825
:10879800FA25303281F8E62193F86C2603EB0212B1
:1087A80002F20C6103F2FC5302F21C6251F8040B52
:1087B80043F8040B9142F9D1002070472823002088
:1087C80018000020094B93F86C2603EB021203F201
:1087D800FC5102F20C6203F20C6351F8040B42F8EC
:1087E800040B9942F9D10020704700BF28230020CC
:1087F80030B50F4A0F4992F8F03592F8FA04303341
:1088080081F8E13102F2FC434E2100FB013102F212
:108818006D620023C85C9854CC18D018033365786F
:10882800A4784570092B8470F4D1002030BD00BFB6
:1088380028230020180000200749084B0A7883F8ED
:10884800FA24013283F8F0254A7883F86C2601323D
:1088580083F8FA2500207047EC9700202823002091
:108868000A4930B50A4C002201F27660135DA3F183
:108878006105052D9CBF203BDBB283540132072ADA
:10888800F4D1002081F87D0630BD00BF28230020E8
:1088980046840308094B93F87E26012A07D893F8E3
:1088A8007F26911E012988BF032283F88226B3F808
:1088B8008626A3F880260020704700BF28230020C2
:1088C80010B5044623790E2B00D110BD032B03D11C
:1088D800E3689868FFF7F4FF1434F3E70B49D1F81D
:1088E80088369A68134618790E280CD19B1A9A1064
:1088F800074B5343013B91F8912693FBF2F3013365
:1089080081F8903670471433EDE700BF2823002024
:10891800CDCCCCCC0C4BD3F89426824210DA93F809
:108928008226022A0AD0032A0CD1D3F898361B696A
:1089380023B19842B4BF012002207047012070473C
:10894800002070470220704728230020084B50B1B0
:10895800D3F8AC26C3F89C060132C3F8AC2605222E
:1089680083F8B0267047042283F8B026704700BF0A
:1089780028230020194BB3F8BC26D3F8B406D3F843
:10898800B81610B40132B3F9BE4692B201300131C3
:10899800A242C3F8B406C3F8B816A3F8BC260FDA87
:1089A800B3F8C226B3F9C4165DF8044B013292B28B
:1089B8008A42A3F8C226A4BF0022A3F8C2267047A1
:1089C800B3F8C0265DF8044B00210132A3F8C02695
:1089D800A3F8BC16A3F8C216704700BF28230020CE
:1089E80073B590F85738032B05460C462FD1002352
:1089F800204E8DF807309DF8073095F858289A4290
:108A080001D802B070BD9DF8073006EBC30393F898
:108A1800CC368BB184F0010383B19DF8073006EBA7
:108A2800C303D3F8C806FAF76FFE9DF80730013381
:108A3800DBB28DF80730DEE72346EDE79DF8073017
:108A480006EBC303D3F8C806FAF758FEEDE7C36B85
:108A5800806BDB79DB0748BF81F0010424B102B0E9
:108A6800BDE87040FAF750BE02B0BDE87040FAF7B2
:108A780045BE00BF2823002000230122C270837056
:108A88000380037143718371C3710372437270472A
:108A980000230A2203604360C381C0F80630C0F88F
:108AA8000A300280704700BF2DE9F0439B4B93F8D2
:108AB8000F1793F81027914200F0BC8093F80F1716
:108AC80093F80F27C1EBC10103EB8101C2EBC2028E
:108AD80003EB820291F8334792F81867A21E964278
:108AE80044D08F4AD3F8144712781B2A00F0A68086
:108AF800002093F80F278B490132A1FB0251490846
:108B080001EB4101521AD2B283F80F27002C77D01B
:108B1800854A5268C2F30802002A4FD1EFF3118246
:108B2800002A4BD18149824E0A68B56800BF0C689B
:108B3800A242F9D17F490E684FF47A7404FB06F11A
:108B48004D1BB5FBF6F504FB0252D3F89C17521ADD
:108B5800B2F5FA7F04DB002240F0040083F899277D
:108B6800D3F89427002A53D1BDE8F08393F80F2750
:108B780003F5E367C2EBC20207EB820264B1144457
:108B8800002112F8015B2944944289B2F9D1CAB292
:108B980002EB1121FF295DD0614AD3F814471278FE
:108BA8001B2AA5D1B3F86C276349013292B204207D
:108BB8008880A3F86C274A8000209AE7EFF3118495
:108BC800102282F312885A4D5C49AE682A68D20393
:108BD80044BF01220A60554A48BFAE6817680A6850
:108BE800E4B284F3118853490D684FF47A743A4417
:108BF80004FB05F1891BB1FBF5F104FB0212A4E7A4
:108C080093F89927002A83D1D3F89427002AABD068
:108C1800464909688A1AB2F5FA7FA5D993F86E27EA
:108C2800032A02D1464A002111800022C3F8942762
:108C3800BDE8F083D3F81447002067E7B3F86C2742
:108C48003D49013292B203208880A3F86C274A80FC
:108C580000204EE793F80F2701211C2404FB021281
:108C6800B918BA5CF2B1012A14D1082E3DD02C4AA9
:108C7800D3F8144712781B2A7FF43AAFB3F86C275D
:108C88002D49013292B206208880A3F86C274A80C9
:108C980000202EE7224A12781B2A18D0D3F814474E
:108CA800002026E7192ED3F814474DD01C4909781F
:108CB8001B297FF41DAFB3F86C171F4D013189B222
:108CC80006261046A3F86C176980AE8011E7B3F842
:108CD8006C271949D3F81447013292B205208880CD
:108CE800A3F86C274A80002003E793F89827002A06
:108CF800D4D04A78102A00F0078140F20281303A35
:108D0800012ACBD851F8010F0E4CC3F808078A790D
:108D18008888A080A271C3F81447E9E628230020B8
:108D2800603D0020ABAAAAAA00ED00E05860002030
:108D380010E000E0BC600020643D0020B860002026
:108D48007E3F0020302A002091F802C04D78026949
:108D580091F8038091F804908E79CF7991F808E022
:108D68000CF0070C45EA0C2508F03F0891F80AC0FA
:108D780015808D784FEA481848EAD5088D7BA2F807
:108D8800028091F803804FEA890040EA981091F830
:108D9800058008F0010840EA8820908006F00F0658
:108DA800487991F80780F60146EA50004E7AD0805B
:108DB8004FEA4E0E4EEAD81E06F0030691F80680DA
:108DC800C87A07F07F074EEA462E3F014E7BA2F88D
:108DD8000AE047EA1817178106F007078E7A91F814
:108DE80009E0C00040EA56100E7B0CF01F0C46EA62
:108DF800072605F03F054F7BD0816D014FEA8C1C9B
:108E080045EAD7004CEA9E0CA2F80CC016825082A4
:108E1800C87B91F80EE0CF7C91F8128091F811C0D0
:108E28008E7C4D7D800040EA9E1091F810E07F0016
:108E38000EF0010E47EAD8170CF00F0C91F81080CD
:108E480040EA8E204FEACC1C91F814E090824CEA5C
:108E5800580C887DA2F816C006F07F0691F811C05C
:108E68000EF0030E47EA4E27360146EA1C165783D2
:108E780091F814C04F7D168305F01F05AD01C000A1
:108E880040EA571045EA9C05D0839583CD7D93F839
:108E98006E6740F2147015F0010F14BF0746AD2736
:108EA80015F0020F08BFAD2015F0080F50840CBF55
:108EB80001200320032E17841ED10A7E93F86F57D2
:108EC800134FD3F87017642A03EB4506A8BF642232
:108ED8009202A7FB0272B6F874770135520905F0C1
:108EE8000F05C91B114483F86F570A4DA6F874275C
:108EF8000A09C3F870172A8007490A68C3F8942733
:108F0800F7E5002A7FF4CAAE012283F89927C5E65F
:108F18001F85EB517E3F002058600020724B5B6834
:108F2800C3F3080370B4B3B9EFF311839BB96F4A65
:108F38006F4D1368AC6800BF11688B42F9D16D4A58
:108F480015684FF47A7101FB05F2121BB2FBF5F2BA
:108F580001FB032220E0EFF31184102383F312882E
:108F680003F1E02364499D681A68D20342BF0122D5
:108F78000A609D685D4BE4B21E680B6884F3118833
:108F88005C4A14684FF47A7202FB04F13344491BBB
:108F9800B1FBF4F102FB0312584B002183F8A01730
:108FA80093F8A117012917D9D3F8A41740F6AC54A0
:108FB800511AA14210DD524909781B2909D1B3F889
:108FC8006C17504C013189B20125A3F86C176180E8
:108FD800A580002183F8A117C0B27E282AD093F873
:108FE800A1272AB393F8A1271B2A5ED893F8B027A4
:108FF800002A72D0002280F0200083F8B02793F86E
:10900800A127022A03D1012808BF83F8A80793F8EB
:10901800102793F8A14793F8A117C2EBC20203EBFC
:10902800820222440131C9B282F8170783F8A117D6
:1090380070BC704793F8A11701292FD993F810171E
:10904800314893F80F470131A0FB0150400800EB6D
:109058004000091AC9B28C420CD093F8A14793F882
:10906800100783F81017C0EBC00003EB8000611EE7
:1090780080F8331793F8A81739B10120002183F835
:10908800A00783F8A817C3F89C271D4909781B294E
:109098001DD00021C3F8AC2783F8B017012183F84D
:1090A800A117C3F8A42770BC7047154A127800218D
:1090B8001B2A83F8A117BBD1B3F86C2711490132D9
:1090C80092B20220A3F86C274A808880B0E7D3F8D0
:1090D800AC170C48511A0180DBE77D288FD101229B
:1090E80083F8B027A4E700BF00ED00E05860002037
:1090F80010E000E0BC600020B860002028230020B9
:10910800603D0020643D0020ABAAAAAA03788B42E8
:1091180083BF034B03EB4101B1F8B407002070474C
:1091280028230020044B93F8CC0718B1002283F8B9
:10913800CC270120704700BF28230020F0B4C24D7F
:1091480095F8F36705F5FA620244B41E1444A24286
:1091580000F07881013A013C002341F2210112F824
:10916800017F83EA07231FB2BBB2002FACBF5B00AD
:1091780081EA43039BB21F0454BF5B0081EA4303A7
:109188009BB21F0454BF5B0081EA43039BB21F04D8
:1091980054BF5B0081EA43039BB21F0454BF5B00CA
:1091A80081EA43039BB21F0454BF5B0081EA430377
:1091B8009BB21F0454BF5B0081EA43039BB21F04A8
:1091C80054BF5B0081EA4303A2429BB2C7D1064465
:1091D800B21E013E2A442E4492F8D01796F8D027A2
:1091E80002EB012292B29A4201D0F0BC704795F886
:1091F800F427002A00F02181431CDBB25C1C2C44BC
:109208002B444FF4AF6193F8D06794F8D03703EB51
:1092180006239BB201FB03F31B1303F54873012AD2
:10922800A5F8B43700F00981C31CDBB25C1C2C44E0
:109238002B44022A93F8D06794F8D03703EB06231F
:109248009BB201FB03F34FEA233303F54873A5F8F8
:10925800B63700F0F280431DDBB25C1C2C442B4473
:10926800032A93F8D06794F8D03703EB06239BB210
:1092780001FB03F34FEA233303F54873A5F8B83726
:1092880000F0DB80C31DDBB25C1C2C442B44042A99
:1092980093F8D06794F8D03703EB06239BB201FB11
:1092A80003F34FEA233303F54873A5F8BA3700F000
:1092B800C48000F10903DBB25C1C2C442B44052A52
:1092C80093F8D06794F8D03703EB06239BB201FBE1
:1092D80003F34FEA233303F54873A5F8BC3700F0CE
:1092E800AC8000F10B03DBB25C1C2C442B44062A37
:1092F80093F8D06794F8D03703EB06239BB201FBB1
:1093080003F34FEA233303F54873A5F8BE3700F09B
:10931800948000F10D03DBB25C1C2C442B44072A1B
:1093280093F8D06794F8D03703EB06239BB201FB80
:1093380003F34FEA233303F54873A5F8C0377CD00D
:1093480000F10F03DBB25C1C2C442B44082A93F871
:10935800D06794F8D03703EB06239BB201FB03F3E5
:109368004FEA233303F54873A5F8C23765D000F1F7
:109378001103DBB25C1C2C442B44092A93F8D067F8
:1093880094F8D03703EB06239BB201FB03F34FEAB3
:10939800233303F54873A5F8C4374ED000F11303FF
:1093A800DBB25C1C2C442B440A2A93F8D06794F84F
:1093B800D03703EB06239BB201FB03F34FEA2333B9
:1093C80003F54873A5F8C63737D000F11503DBB2AB
:1093D8005C1C2C442B440B2A93F8D06794F8D037A4
:1093E80003EB06239BB201FB03F34FEA233303F598
:1093F8004873A5F8C83720D000F11703DBB25C1C0E
:109408002C442B440C2A93F8D06794F8D03703EBFC
:1094180006239BB201FB03F34FEA233303F548739A
:10942800A5F8CA3709D000F11903DBB25A1C2A443F
:109438002B4493F8D03792F8D037012385F8CC37EE
:10944800F0BC70470023C2E628230020794B5B68F4
:10945800C3F3080370B5B3B9EFF311839BB9764A28
:10946800764D1368AC6800BF11688B42F9D1744A15
:1094780015684FF47A7101FB05F2141BB4FBF5F47F
:1094880001FB034320E0EFF31181102383F31288DB
:109498006A4C6C4AA5682368DE0344BF0123136045
:1094A800654B48BFA5681E681368C9B281F3118867
:1094B800634A14684FF47A71334401FB04F2521B77
:1094C800B2FBF4F201FB03235F4CD4F8F827C4F88D
:1094D800F8379B1AB3F5FA5F1AD9002384F8FC37DA
:1094E80084F8FD37A1282FD0A22800F09C8094F89A
:1094F800FD2794F8F3370025A2B16A1C6119D5B28B
:10950800C0B29D4281F8D00784F8FC570CD070BDDA
:1095180094F8FC57002DE5D094F8FD2794F8F3371C
:10952800002AEAD19D42F2D194F8FE37052B72D079
:10953800062B03D194F8D1371E2B0DD0002384F8C5
:10954800FC3784F8FD3770BD01221B2384F8FD2702
:1095580084F8F3370025D0E76A1E002A4FF000018F
:1095680050DD08460B462344013093F8D037DBB270
:1095780083EA0105ED074FEA530348BF83F08C03E4
:1095880083EA5105EE074FEA530348BF83F08C0383
:1095980083EA9105ED074FEA530344BF83F08C0338
:1095A800DBB283EAD105EE074FEA530344BF83F0E9
:1095B8008C03DBB283EA1115ED074FEA530344BF6E
:1095C80083F08C03DBB283EA5115EE074FEA5303AD
:1095D80044BF83F08C03DBB283EA9115ED074FEAB1
:1095E800530344BF83F08C03DBB283EAD1155908D7
:1095F800EB0748BF81F08C01C0B248BFC9B29042A6
:109608000346B0DB224492F8D0378B4296D1032030
:10961800FFF794FD92E70020FFF790FD94F8D1370B
:109628001E2B8BD198E70122232384F8FD2784F889
:10963800F3378FE700ED00E05860002010E000E00D
:10964800BC600020B86000202823002007299DBFA7
:10965800034B03EB8101B1F800080020704700BFFD
:10966800282300201A4B93F8202832B193F8242895
:109678000021A82A83F8201801D00020704793F809
:109688003728002AF9D110B4DFED126A03F6240155
:1096980003F2FC7003F63402B4EE047ACC780B794A
:1096A80003EB042307EE903AF8EEE77AB0EE666A29
:1096B800A7EE876A02318A42FCEEC67A17EE903A24
:1096C80040F8043FEAD101205DF8044B704700BF21
:1096D800282300200080BBC310B50446F9F7E8F939
:1096E8000F4BD3F83C28C3F83C08801A41F2883263
:1096F8009042E4B205D983F82448012283F840282F
:1097080010BD93F840289918142A81F8244803D1E9
:10971800012283F8202810BD0132D2B2EEE700BF43
:1097280028230020034B03EB4101B1F84408C0088B
:10973800704700BF28230020724B93F86428002A42
:1097480000F0C28070B493F86548B3F8665803EB2C
:109758004401002091F86B6891F86C2883F864083C
:1097680042EA0622954202D0002070BC704793F866
:109778006928012A00F0AA80812AF6D10320102C3A
:1097880040F2A68093F86D4893F86B5893F86C18DC
:1097980093F86E2841EA052142EA04221024A3F82E
:1097A8004418A3F8462883F8654893F86F1893F887
:1097B8007028032C42EA0122A3F84828D5D093F850
:1097C800711893F87228042C42EA0122A3F84A2857
:1097D800CBD093F8731893F87428052C42EA012229
:1097E800A3F84C28C1D093F8751893F87628062C5E
:1097F80042EA0122A3F84E28B7D093F8771893F8D5
:109808007828072C42EA0122A3F85028ADD093F813
:10981800791893F87A28082C42EA0122A3F85228EA
:10982800A3D093F87B1893F87C28092C42EA0122EC
:10983800A3F8542899D093F87D1893F87E280A2C19
:1098480042EA0122A3F856288FD093F87F1893F89C
:1098580080280B2C42EA0122A3F8582885D093F8D7
:10986800811893F882280C2C42EA0122A3F85A287E
:109878003FF47BAF93F8831893F884280D2C42EAC1
:109888000122A3F85C283FF470AF93F8851893F889
:1098980086280E2C42EA0122A3F85E283FF465AF21
:1098A80093F8871893F88828102C42EA0122A3F825
:1098B80060287FF45AAF93F8891893F88A2842EA07
:1098C8000122A3F8622850E700207047104656E7A7
:1098D800002C3FF44AAF93F86B1893F86C28012CCE
:1098E80042EA0122A3F844283FF43FAF93F86D18E9
:1098F80093F86E28022C42EA0122A3F846287FF446
:1099080054AF32E728230020654B5B68C3F3080394
:1099180070B4B3B9EFF311839BB9624A624D13680F
:10992800AC6800BF11688B42F9D1604A15684FF4E2
:109938007A7101FB05F2141BB4FBF5F401FB034338
:1099480020E0EFF31181102383F31288564C584A14
:10995800A5682368DE0344BF01231360514B48BF49
:10996800A5681E681368C9B281F311884F4A146844
:109978004FF47A71334401FB04F2521BB2FBF4F248
:1099880001FB03234B49D1F890289A1AB2F57A6F54
:1099980017D891F89428C1F89038BAB1022A20D083
:1099A800242A91F8653878D901320233D2B25B00A3
:1099B8009A4281F894281CDB01339A4265D070BC26
:1099C80070470022C1F8903881F89428A828F6D169
:1099D800002281F86428A1F8662891F865380446C1
:1099E80003E0C4B281F8654823468D1885F86848B5
:1099F800DAE7B1F86638C0B283EA002000B200287E
:109A0800B8BF41F2210283B2B4BF82EA43035B00CC
:109A18009BB2180446BF41F2210282EA43035B006D
:109A28009BB21A0446BF41F2210282EA43035B005B
:109A38009BB21E0446BF41F2210282EA43035B0047
:109A48009BB21D0446BF41F2210282EA43035B0038
:109A58009BB21C0446BF41F2210282EA43035B0029
:109A68009BB2180446BF41F2210282EA43035B001D
:109A78009BB21A0446BF41F2210282EA43035B000B
:109A88009BB2A1F8663870BC70470022012381F8A8
:109A9800942881F8643870BC7047C4B2A5E700BF49
:109AA80000ED00E05860002010E000E0BC600020FD
:109AB800B860002028230020F8B5124D95F8AD288D
:109AC80002B9F8BD104B1C682368DE693EB1204618
:109AD80005F69801B047002385F8AD38F8BD05F6BE
:109AE8009807BE1800E023689B682046984700281E
:109AF800F9D0236817F8011B1B6820469847B7421E
:109B0800F1D1E8E7282300208C44002003788B4219
:109B180010D9094B03EB810193F8E038D1F8B0086C
:109B28001BB900F5777080B27047400800F5777070
:109B380080B2704700207047282300202DE9F041AB
:109B4800C84C94F8E80808B9BDE8F08194F8E91819
:109B5800002384F8E838002900F03E8194F8EC38B6
:109B6800C14D94F8FC285BB213F1630FB8BF95F9A7
:109B7800E831002A40D013F1310F80F2B38113F19C
:109B8800380F80F2D28113F13D0F80F2D28113F1A8
:109B9800420F80F2D28113F1450F80F2D28113F186
:109BA800470F80F2D28113F1490F80F2D28113F16D
:109BB8004A0F00F0D28113F14B0F00F0D18113F15D
:109BC8004C0F00F0D18113F14D0F00F0D08113F14B
:109BD8005C0FB8BF642680F2CD81D4F80009A34F8A
:109BE80000FB06F087FB0076C017C0EB661004EB9D
:109BF800820680B2C6F8B00885F8E83194F8F8789B
:109C080094F8F93894F8FA0894F8FB681B0443EAC6
:109C18000763334343EA002303F0F020B0F1E02F59
:109C280000F0D180102794F80A0994F8EE38D4F897
:109C38000C6994F810C93678034103F00F039E426B
:109C480010D90B2B0ED8002A40F0038194F8EE8827
:109C580094F8EFE804EB83030CEA08080EEB082EEF
:109C6800C3F8B0E894F8F038034103F00F039E42BC
:109C780010D90B2B0ED8002A40F0EF8094F8F0880A
:109C880094F8F1E804EB83030CEA08080EEB082EBD
:109C9800C3F8B0E894F8F238034103F00F039E428A
:109CA80010D90B2B0ED8002A40F0FB8094F8F288CC
:109CB80094F8F3E804EB830308EA0C080EEB082E8B
:109CC800C3F8B0E894F8F438034103F00F039E4258
:109CD80010D90B2B0ED8002A40F0E78094F8F488AE
:109CE80094F8F5E804EB83030CEA08080EEB082E59
:109CF800C3F8B0E894F8F638034103F00F039E4226
:109D080042D80D2F24DD94F8F838034103F00F03EF
:109D18009E4210D90B2B0ED80AB19A420BD094F858
:109D2800F88894F8F9E804EB83030CEA08080EEBCA
:109D3800082EC3F8B0E8102F0AD194F8FA3843FA7D
:109D480000F000F00F00B04202D20B2840F29880D9
:109D5800B1B394F8AD389BB394F8EE381B062FD402
:109D6800F8F7A6FED4F8E43800F57A70C5F8F001E3
:109D78001BB15A68121A002A1CDB3D493D4AC5F836
:109D8800F43101200A60DFE60B2BBAD80AB19A42F7
:109D9800B7D094F8F68894F8F7E804EB83030CEA54
:109DA80008080EEB082EC3F8B0E8AAE75A68121A9A
:109DB800002AE3DA03F108019B68002BF6D1DDE7FE
:109DC8000120BDE8F08194F8EE0800063FF52AAFBF
:109DD80029480C27036026E7F8F76AFE224D274B2F
:109DE80095F8E921A3FB00135B0C1AB394F8EC086F
:109DF80094F8ED28D2B2122A18BF012A09D002F02D
:109E0800EF02A2F1A202B2FA82F252090AB985F867
:109E1800E921D4F8041994F8FC2899B18B4248D068
:109E2800591A012948D094F8E918A4F80809C4F87F
:109E38000439E3E694F8EC2894F8ED0800EB0220E6
:109E480080B2E6E7A4F80809C4F8043994F8E918D8
:109E5800D4E693427FF4FAAE04E793427FF40EAF60
:109E680018E700BF28230020180000201F85EB51A9
:109E78000C2C002004020020701B002083DE1B43F2
:109E880012B190423FF464AF94F8FA2894F8FB3882
:109E980004EB800002EA0C0C03EB0C23C0F8B0388A
:109EA80056E793427FF402AF0CE79A427FF416AF6D
:109EB80020E794F8E918A1E6002AB4D0B4F80869B4
:109EC800D4F800192D4F861B143E01FB06F187FBC1
:109ED8000176C917A1EBE60104EB820689B2C6F840
:109EE800B018A0E76FF0300C0126254806F1FF38BE
:109EF80000EB480E00EB46069EF801E0777810F973
:109F08001860A7EB0E07981B00FB07F0ACEB0606E2
:109F180090FBF6F0704440B2002801DA00265CE6B7
:109F28006428A8BF6420064657E66FF0370C02265F
:109F3800DBE76FF03C0C0326D7E76FF0410C0426F3
:109F4800D3E76FF0440C0526CFE76FF0460C0626E2
:109F5800CBE76FF0480C0726C7E79C460826C4E7FE
:109F68006FF04A0C0926C0E79C460A26BDE79C46C6
:109F78000B26BAE76FF05B0C0C26B6E767666666D9
:109F8800A8580308324B5B68C3F3080370B4B3B92D
:109F9800EFF311839BB92F4A2F4D1368AC6800BFAC
:109FA80011688B42F9D12D4A15684FF47A7101FB7B
:109FB80005F2141BB4FBF5F401FB034320E0EFF3B7
:109FC8001181102383F31288234C254AA56823683E
:109FD800DB0344BF012313601E4B48BFA5681E68FE
:109FE8001368C9B281F311881C4A14684FF47A7156
:109FF800334401FB04F2521BB2FBF4F201FB0323CE
:10A00800184AD2F81419C2F814395B1A41F2883187
:10A018008B420AD9C0B2012382F8EC0882F81839B9
:10A02800002382F8E83870BC704792F818390F2B73
:10A03800F9D8D1180133DBB2C0B2102B81F8EC0883
:10A0480082F81839ECD1012382F8E83870BC7047DF
:10A0580000ED00E05860002010E000E0BC60002047
:10A06800B860002028230020036933F8110000EBB2
:10A078008000C01000F55C7080B27047436993F8A7
:10A088002320002A00F0C3802DE9F043714ADC7DCB
:10A09800127800211A2A04F0040604F0080583F84F
:10A0A800231000F0B680002E40F0BE801DB11A8C3F
:10A0B80042F001021A8493F80290997993F801C04A
:10A0C8000269DE7893F80480DF7909F0070001F06F
:10A0D8000F014FEAC11E4CEA002106F03F06187A2C
:10A0E8001180997893F80AC0760146EAD106D978A2
:10A0F80056804FEA880848EA911193F805809E7BBC
:10A1080008F0010841EA8821918059794EEA510105
:10A11800D18007F07F07997993F807E03F0147EA74
:10A128001117597A1781400040EADE1001F0030147
:10A1380040EA41205F7BD97A50810CF01F0C587A95
:10A148004FEA8C1C4CEA90009081187B93F80AC067
:10A1580007F0070740EA072006F03F065F7B1082FA
:10A16800C90041EA5C117601D18146EAD7015182E2
:10A17800D97B93F80E8093F810E093F811C0DE7C39
:10A188009F7C587D890041EA98110EF0010E41EA42
:10A198008E21918293F812E0197C0CF00F0C760056
:10A1A8004FEACC1C46EADE1E4CEA51011E7D93F8AC
:10A1B80011C0D18207F07F073F01997D47EA1C173C
:10A1C80006F0030693F814C017834EEA46265F7D0F
:10A1D800568314F0010F40F2147300F01F0014BFEF
:10A1E8001E46AD26800114F0020F4FEAC10140EA75
:10A1F8009C0008BFAD2341EA5711002D9083D183FD
:10A20800168453840CBF01200320BDE8F083104658
:10A21800704711491F8C0C8066B147F002021A84FE
:10A2280012B29DB94A8046E71A8C4DB942F0020233
:10A238001A8440E745B147F001021A8412B2F1E7E7
:10A2480042F003021A8436E73AB2EBE747F003021A
:10A258001A84F3E7603D0020643D0020394B5B68B9
:10A26800C3F30803F0B413BBEFF31183FBB9364A09
:10A27800364E1368B56800BF1468A342F9D1344A52
:10A2880016684FF47A7404FB06F2551BCA69B5FBCD
:10A29800F6F504FB03539A1A40F6AC54A2422DDC9F
:10A2A80091F822406CB3182C37D9F0BC7047EFF303
:10A2B8001184102383F31288244D264AAE682B6834
:10A2C800DB0344BF012313601F4B48BFAE681F6800
:10A2D8001368E4B284F311881D4A15684FF47A7440
:10A2E80004FB05F23B44921BB2FBF5F204FB03238B
:10A2F800CA6940F6AC549A1AA242D1DD002281F80C
:10A3080022200F28D1D10122CB61087081F82220A8
:10A31800002381F82330F0BC7047631CDBB2192B93
:10A3280081F822300855F3D10B4B1B781A2B08BF44
:10A338000A4B4FF0010081F8230008BF9A80F0BC57
:10A34800704700BF00ED00E05860002010E000E01A
:10A35800BC600020B8600020603D0020643D002003
:10A368000A4BDFED0B6ADFED0B7A03EB8101D1F8C5
:10A378001C3907EE103AB8EE477AE7EE267AFCEE7B
:10A38800E77A17EE903A98B2704700BF282300206A
:10A3980001F11F3F00405C44714A92F85C3933B1C7
:10A3A80092F862390021162B82F85C1901D000203E
:10A3B800704792F86139022BF0B440F2CE8002F572
:10A3C8001660184402F66211D32311F8014F634056
:10A3D80013F0800F4FEA430318BF83F0D503DBB2B5
:10A3E80013F0800F4FEA430318BF83F0D503DBB2A5
:10A3F80013F0800F4FEA430318BF83F0D503DBB295
:10A4080013F0800F4FEA430318BF83F0D503DBB284
:10A4180013F0800F4FEA430318BF83F0D503DBB274
:10A4280013F0800F4FEA430318BF83F0D503DBB264
:10A4380013F0800F4FEA430318BF83F0D503DBB254
:10A4480013F0800F4FEA430318BF83F0D503884207
:10A45800DBB2BAD192F87919994202D00020F0BC47
:10A46800704792F8680992F8676992F86C1992F83F
:10A47800703992F8744992F86459B2F864C9D2F8FC
:10A48800647900F00F00C00140EA560001F01F0196
:10A4980092F86B69C2F82809890141EA960103F02C
:10A4A8003F0392F86F6992F87309C2F834195B0197
:10A4B80043EAD60392F86319C2F8403904F07F04DE
:10A4C800B2F86839D2F86869240105F0070544EA4A
:10A4D800101041EA0521C3F30A13C2F84C09B2F877
:10A4E8006C59C2F81C19B2F86E49D2F87009B2F862
:10A4F8007219C2F82C39D2F87439C0F38A10C1F332
:10A508004A01C3F3CA13CCF3CA0CC7F38A37C6F39C
:10A51800CA366D09C4F30A04C2F84409C2F84819D6
:10A52800C2F820C9C2F82479C2F83069C2F838598B
:10A53800C2F83C49C2F8503992F8783992F877094C
:10A54800B2F87619DB0043EA5013C1F38A01C2F866
:10A558005839C2F85419012081E7D3237AE700BF9C
:10A5680028230020944B5B68C3F3080370B443BBF3
:10A57800EFF311832BBB914A914D1368AC6800BF70
:10A5880011688B42F9D18F4A15684FF47A7101FB33
:10A5980005F2141B8C4AB4FBF5F401FB0343D2F813
:10A5A800A01901F24C41994233D201240021C2F88A
:10A5B800A03982F8600982F8A44982F85C1970BC55
:10A5C8007047EFF31181102383F312887C4C7F4A84
:10A5D800A5682368DE0344BF01231360774B48BF97
:10A5E800A5681E681368C9B281F31188754A146892
:10A5F8004FF47A7101FB04F23344521BB2FBF4F2BC
:10A6080001FB0323704AD2F8A01901F24C41994288
:10A61800CBD392F8A4190029C7D002298ABF92F88F
:10A628006149052402348C42C9DD4B1CDBB29C42D3
:10A638001144D4BF0125002582F8A43981F86009A6
:10A6480082F85C59BBDC92F862590023162D82F817
:10A65800A439B4D06B00290648BF83F0D503DBB218
:10A6680013F0800F4FEA430318BF83F0D503DBB222
:10A6780013F0800F4FEA430318BF83F0D503DBB212
:10A6880013F0800F4FEA430318BF83F0D503DBB202
:10A6980013F0800F4FEA430318BF83F0D503DBB2F2
:10A6A80013F0800F4FEA430318BF83F0D503DBB2E2
:10A6B80013F0800F4FEA430318BF83F0D503DBB2D2
:10A6C80092F8610913F0800F4FEA430318BF83F033
:10A6D800D5030228DBB247D93D490844023111F8B5
:10A6E800016F734013F0800F4FEA430318BF83F0E4
:10A6F800D503DBB213F0800F4FEA430318BF83F092
:10A70800D503DBB213F0800F4FEA430318BF83F081
:10A71800D503DBB213F0800F4FEA430318BF83F071
:10A72800D503DBB213F0800F4FEA430318BF83F061
:10A73800D503DBB213F0800F4FEA430318BF83F051
:10A74800D503DBB213F0800F4FEA430318BF83F041
:10A75800D503DBB213F0800F4FEA430318BF83F031
:10A76800D5038142DBB2BAD1224492F85F299A42DA
:10A778007FF425AF7A2D08D07C2D06D0282D7FF4C4
:10A788001EAF144B01221A7019E7134A136E572B88
:10A798003FF715AF114912480D684C6808219954C4
:10A7A80013440121C3F80150C3F80540136E01702A
:10A7B8000933136603E700BF00ED00E0586000208E
:10A7C80010E000E0BC60002028230020B8600020D2
:10A7D800882C002080440020904400208D2C0020EC
:10A7E8008144002070B54A4E4A4C337805462BB157
:10A7F800D4F8A83983429CBF00233370464B1B68AA
:10A80800D8070ED594F8AC3994F8AD299A4235D1C9
:10A81800D4F8E839ED1A002D2ADD012084F8AE09B4
:10A8280070BD990440D4D4F8D4393C489847C2073D
:10A8380014D500F00202002A3949D4F8B03914BFFF
:10A848000122002281F8F8212B440CBF01210021AC
:10A8580001223170C4F8A83984F8AE29430744BFEF
:10A86800012384F8E439D4F8E839ED1A002DD4DC52
:10A8780094F8AE39B3B994F8E40970BDD4F8B029A6
:10A88800274984F8AD392A4401230020C4F8A829AF
:10A8980081F8F80184F8AE393370D4F8E839ED1A44
:10A8A800002DBADC012070BDB4F8B4390BBBB4F884
:10A8B800B639F3B9B4F8B839DBB9B4F8BA39C3B9A9
:10A8C800B4F8BC39ABB9B4F8BE3993B9B4F8C039E7
:10A8D8007BB9B4F8C23963B9B4F8C4394BB9B4F820
:10A8E800C63933B9B4F8C8391BB9B4F8CA39002B1A
:10A8F8008ED0D4F8B0390A4A2B440021C4F8A839BC
:10A90800012382F8F81184F8AE393370C5E700BF27
:10A91800663F002028230020A06B0020F42C002094
:10A928001800002000207047002070470120704761
:10A93800024B03EB4101B1F8EC09704728230020D2
:10A94800044B93F8100A18B1002283F8102A01204A
:10A95800704700BF28230020024B03EB8101B1F8A8
:10A96800140A70472823002030B402460023052526
:10A978001E2400E00232032BD4BF0021012100F87D
:10A9880013100133042B04D0122B5470F2D130BCB5
:10A9980070475570EEE700BF024B03604360836069
:10A9A800C3607047E803D007024B03EB4101B1F8DD
:10A9B800B409704728230020024B03EB4101B1F88A
:10A9C800B409704728230020E14B93F84C2A0AB9B0
:10A9D800002070472DE9F04F93F84E2A93F84D4A1E
:10A9E8000021012A8BB083F84C1A00F0F88093F804
:10A9F800545A023D15F0FF0500F0A68103F65420D5
:10AA080005444FF6FF7210F8011B521AA84292B281
:10AA1800F9D1110A1C4494F8530A884240F09081F5
:10AA280094F8521AD2B2914240F08A8193F8742A6B
:10AA3800202A40F0858193F84F0A821C0192821DDA
:10AA4800029200F10802039200F10A02049200F156
:10AA58000C02059200F10E02069200F11002079214
:10AA680000F11602089200F1180200F1040A00F140
:10AA7800120800F11407099200F11A0B9DF804203E
:10AA880053FA82F19DF8082053FA82FC9DF80C20B5
:10AA98009CF8559A9CF854CA53FA82F201929DF890
:10AAA800102053FA82F69DF8142053FA82F59DF887
:10AAB800182053FA82F49DF81C2053FA82F202926D
:10AAC80053FA88F203929DF8202091F8558A91F85C
:10AAD800541A53FA82F2184405929DF8242053FA26
:10AAE8008AFE53FA87F790F855AA90F8540A049703
:10AAF80053FA82F29EF8557A06929EF854EA019A21
:10AB080000EB0A2001EB08210EEB072E92F8558A7C
:10AB180092F8547AC3F8140A96F8552A01920CEB65
:10AB28000920C3F8200A95F855CA96F8546A95F88A
:10AB3800545A019AC3F8181A06EB0226049A029985
:10AB4800C3F81CEA92F855EA92F8542A91F8559AF3
:10AB580091F8540A0399019602EB0E22C3F83C2A95
:10AB6800059A94F855AA019E94F8544AC3F8286A9D
:10AB780007EB082700EB092091F8558A91F8541A39
:10AB880092F8556AC3F8340A53FA8BFB92F8540AC0
:10AB9800069AC3F8247A05EB0C2504EB0A2401EB8A
:10ABA8000821C3F82C5AC3F8304A92F8555AC3F80A
:10ABB800381A9BF8554A92F8541A9BF8542A00EB15
:10ABC8000620C3F8400A01EB052102EB042201200C
:10ABD800C3F8441AC3F8482A0BB0BDE8F08F93F8BD
:10ABE8004F0AB3F8508A1D18821C019253FA82F258
:10ABF80095F8546A95F8557A92F855CA92F854EA35
:10AC080000F1040A53FA8AF2851D46442946029542
:10AC1800B64492F8555A92F8546A53FA81F20EEBF8
:10AC2800072E00F108070397764453FA87F792F83E
:10AC380054EA92F8552A06EB0C2600F10A0197F817
:10AC480055CA0491B64497F8546A53FA81F70EEB43
:10AC5800052500F10C0197F8558A05912E4497F8BF
:10AC6800545A53FA81F706EB022600F10E0197F8C1
:10AC7800542A0691354453FA81F605EB0C2500F168
:10AC8800100153FA81FE154496F8542A97F8557A1C
:10AC980096F855CA9EF8546A079105EB082500F105
:10ACA80012082A4453FA88F502EB072200F1140728
:10ACB80095F8559A9EF855EA324495F8546A53FA2D
:10ACC80087F500F1160102EB0C22324495F854CABC
:10ACD800089153FA81F602EB0E2200F1180195F85B
:10ACE800555A0991624496F854EA96F855CA02EB07
:10ACF800092253FA81F6724400F11A0B96F854EAC5
:10AD080096F8556A02EB052253FA8BF51C447244F7
:10AD180095F854EA94F8539A95F8555A94F8524A83
:10AD280002EB0C2296440EEB062E0EEB052E04EBDE
:10AD380009291FFA8EFE1FFA89F9F1453FF49EAEE4
:10AD480000200BB0BDE8F08FFF214FF6FF7261E6DF
:10AD5800282300204E4B5B68C3F3080370B4B3B9D3
:10AD6800EFF311839BB94B4A4B4D1368AC6800BF96
:10AD780011688B42F9D1494A15684FF47A7101FB81
:10AD880005F2141BB4FBF5F401FB034320E0EFF3D9
:10AD98001181102383F312883F4C414AA568236828
:10ADA800DB0344BF012313603A4B48BFA5681E6804
:10ADB8001368C9B281F31188384A14684FF47A715C
:10ADC800334401FB04F2521BB2FBF4F201FB0323F0
:10ADD800344AD2F8781A591AB1F5FA7F14D90021F1
:10ADE800C2F8783A82F87C1A82F87D1AC3B2042B2A
:10ADF80026D0202B24D092F8741A09B9552838D0B7
:10AE0800814216D1002109E092F87D1A99B992F889
:10AE18007C1AC2F8783AC3B20029E8D092F84D0AF1
:10AE280054180138814284F8543A1DD0013182F80F
:10AE38007C1A70BC7047013982F87D1A70BC704763
:10AE4800002102244FF6FF7082F84F4AA2F8500AF8
:10AE58005418581E814282F8743A82F84D3A82F8A2
:10AE68004E1A84F8543AE1D1012382F84C3A70BC66
:10AE7800704701241F2582F8740AA2F8501A82F834
:10AE8800543A82F84E4A82F84F4A82F84D5ACDE732
:10AE980000ED00E05860002010E000E0BC600020F9
:10AEA800B860002028230020082A07D808B50846DB
:10AEB80011461A4612F038F9002008BD00207047E4
:10AEC800F8B507460026F5B20024E0B2202229464C
:10AED800013412F029F90C2CF7D10136092EF2D1E0
:10AEE8001B4D422201200021441C12F01DF915F8C7
:10AEF800012FE4B22046002AF5D197F90E302BBB7A
:10AF0800144D14464D22E0B2022112F00DF915F845
:10AF1800012F0134002AF6D10F4D2B2202200321E4
:10AF2800441C12F001F915F8012FE4B22046002A5A
:10AF3800F5D10A4D2B2202200421441C12F0F4F80A
:10AF480015F8012FE4B22046002AF5D10020F8BDFB
:10AF5800BC840308AC840308A08403089484030811
:10AF6800F8B5084617465E1E16F8015F421CD4B2B3
:10AF780039462A462DB1082F01D812F0D5F82046B7
:10AF8800F2E72846F8BD00BF70B50A4C4FF0FF3510
:10AF980004F51C762368D03418463BB11B79142B72
:10AFA80004D0F7F7BBFF854228BF0546A642F1D17A
:10AFB800284670BDD462002070B51A4C94F88236C9
:10AFC800022B17D0032B10D00020D4F8943694F815
:10AFD8007E2A1344B3F5807FA8BF4FF48073834261
:10AFE800A8BF0346C4F8943670BDD4F89806F7F79E
:10AFF80095FFEAE700200C49034641F2260603F5CF
:10B00800817201EB021206EB0315D279D20703F124
:10B01800010304D44A5D012A98BF00F50070082B8B
:10B02800EDD1D2E728230020C485002010B50B4BB2
:10B038000B4993F8812A93F8803A097882B00D3247
:10B048001E330424027243728DF8044021B9012191
:10B058000DEB040026F004FC02B010BD28230020EC
:10B068006C41002000B5094B83B01B7804228DF891
:10B0780004201BB1002003B05DF804FB01210DEB97
:10B08800020026F0EDFB03B05DF804FB6C410020E4
:10B0980000B5094B83B01B7802228DF804201BB140
:10B0A800002003B05DF804FB012101A826F0D8FBBD
:10B0B80003B05DF804FB00BF6C41002000B5084BED
:10B0C80083B01B7801218DF804101BB1002003B058
:10B0D8005DF804FB01A826F0C3FB03B05DF804FB90
:10B0E8006C41002000B5074B83B01B7800208DF819
:10B0F80004001BB9012101A826F0B2FB03B05DF8DA
:10B1080004FB00BF6C410020ECE700BFF0B5184617
:10B118008BB01C460E46174629F01AFE1E2828BF7B
:10B128001E200323214602460546002402A88DF866
:10B1380004308DF805708DF806608DF807402AF008
:10B148006BF9064B1B7813B120460BB0F0BD291DD7
:10B1580001A826F085FB0BB0F0BD00BF6C410020B4
:10B1680010B582B000248DF8043001AB8DF805408D
:10B17800FFF7CCFF02B010BD70B50F4C94F8856A8C
:10B18800054646B9012384F8853AFCF7E5FAFCF749
:10B19800B7F984F8856A094B94F8171493F8F921DC
:10B1A80094F8163412F0400F14BF10220D220A44EE
:10B1B8001E332A726B7270BD2823002018000020ED
:10B1C8002DE9F047314C94F8853A13B994F8865A2A
:10B1D80015B10020BDE8F087012384F8853AFCF713
:10B1E800BBFA2B4BB4F8882AB3F800E029464FF095
:10B1F800050A4FF006094FF00708A718A35C97F84F
:10B208000802984202F1010C05F1050012D0261837
:10B21800601987F80832170A80F88CAA80F88E9A85
:10B2280080F88F2A80F8908A80F88D7A0131063567
:10B2380086F88C3A1FFA8CF2724501F101010AD2A4
:10B248006329DADDA4F8882A4DB9002384F8853A01
:10B258000020BDE8F0870023A4F8883AF4E70D4EF3
:10B268000D480421FCF72CF93068F8F747FA2B460B
:10B2780000220A490848FCF7F3F83068F8F744FA5E
:10B2880002210548FCF71CF9DFE700BF282300204E
:10B29800180000205465002000300140B42D002023
:10B2A80070B51A4C94F8182494F8E43C52BB03F097
:10B2B800F703174D174884F8E43C0421FCF700F91C
:10B2C8002868F8F71BFA94F8E46C12480421FCF794
:10B2D800A9F831460F48FCF7A5F82868F8F714FADA
:10B2E80002210C48FCF7ECF894F81A1494F81904A5
:10B2F800FCF772F94FF4F072202104482AF0ECF8B8
:10B30800002070BD43F00803D3E700BF28230020C6
:10B31800546500200030014010B50C4658B1F6F7CE
:10B32800E9FC18B1032383710023C3712146BDE8EA
:10B338001040F8F769B810BD10B50446012100792E
:10B34800FFF7EAFF637921689A0802239340C868E7
:10B35800DB439BB20340CB6010BD10B504462221ED
:10B368000079FFF7D9FF63792268990802238B4097
:10B37800D94389B21161D1689BB20B43D36010BD28
:10B38800F0B5184E002383B004460821D6F8E80C1F
:10B3980086F8A13702ADF7F7C9FDD6F8E80C812188
:10B3A800F7F7C4FD8923D6F8E86C25F8023DE71DB8
:10B3B80014F8010B3246294611F00AFEBC42F7D1B7
:10B3C800BDF806301A0A52FA83F3C3F1FF039BB2A1
:10B3D8003246D8B20021ADF8063011F0F9FD03B0BD
:10B3E800F0BD00BF2823002070B5A0F65C0494F8D7
:10B3F800493893B1B4F8503801339BB2082BA4F8FC
:10B4080050381CD9002184F84918A4F85018E06B6A
:10B4180025F0A6FE94F849388BB93E4E96F8EC3CD8
:10B428001BB901212046FDF7DBFA94F8483853BBD5
:10B43800D4E909239A4203D1002386F8EC3C70BD75
:10B4480096F8EC2C022A12D802F1010214BFFF234D
:10B458007F2386F8EC2CA4F84C38082384F84A3863
:10B46800012384F84838E06BBDE8704064E75A1C53
:10B47800A169A262CB5C21698A4228BF0022DBB2A3
:10B4880028BFA262E7E794F94A38C3B394F84C1886
:10B4980096F8ED5C11F0010123D0012D03D80121AC
:10B4A8002046FDF79DFAAB1E012B03D8002120464C
:10B4B800FDF796FA0135EDB2032D86F8ED5CBED99D
:10B4C800B4F84C385B08A4F84C3894F84A38013B77
:10B4D8005BB2002284F84A3886F8ED2C002BA7D0FE
:10B4E800ADE715F0FD0304D101212046FDF778FAF8
:10B4F800E0E7012BDED12046FDF772FADAE7D4E95E
:10B50800091291429BD184F84838E06BBDE870403D
:10B5180023E700BF2823002038B5A0F506640022E1
:10B52800E06B354D03685A62A1F12903302B31D8FD
:10B5380095F8EE3C0133DBB2012B85F8EE3C0BD9D4
:10B5480095F8EF3C85F8EE2CB4F84E2801335208F4
:10B55800A4F84E2885F8EF3C95F8EF2C0023082A2C
:10B56800A4F8503815D185F8EF3CB5F8F03C013314
:10B578009BB2032BA5F8F03C08D96379DB0705D506
:10B58800E36A94F84E0853B3216B98470023A4F854
:10B598004E3838BD5B396C290ED8B4F84E3885F86A
:10B5A800EE2C5B0843F08003A4F84E3895F8EF3C86
:10B5B800013385F8EF3CCFE794F84938002BCBD11D
:10B5C800012185F8EE3CA5F8F03C802384F8491861
:10B5D800A4F84E3885F8EF1C25F0C2FDBCE7E369F6
:10B5E8006269D054E369E1680133B3FBF1F201FB0E
:10B5F8001233E361CAE700BF2823002038B5A0F55D
:10B6080006646379A579DB0722D594F8443803B337
:10B61800D4F840341A68D36A5B08536294F84838FF
:10B6280023B1B4F852380133A4F85238E94301F091
:10B638000101E06B25F094FD012384F847380023CD
:10B6480084F8453884F84638A4F84E3884F84438E5
:10B6580038BD94F84738012B04BF94F8453884F86E
:10B6680046382046FCF79DFD94F847384BB901232E
:10B67800E94384F847381940E06BBDE8384025F0C5
:10B688006FBD002384F8473805F00101E06BBDE881
:10B69800384025F065BD10B5A0F65C0494F849382B
:10B6A8001BBB94F848288ABBD4E9091399421CD0DB
:10B6B800591CA069A162C35C2069DBB25B0043F43A
:10B6C8000073A4F84C380A2384F84A38012384F814
:10B6D800483894F85738814228BFA262012B01D01C
:10B6E800042B02D1E06BFFF727FE94F84438002BB7
:10B6F8006FD194F845380133DBB2092B84F845380B
:10B7080027D12046BDE81040FCF74BBD94F94A38D4
:10B718007BB1B4F84C184B08A4F84C3801F001017F
:10B728002046FDF75DF994F84A38013B84F84A3819
:10B73800DBE784F84838D4E909239A42D5D194F84C
:10B748005738012B01D0042BCFD1E06BFFF705FE52
:10B75800CBE70A2B3DD194F847382BB9B4F84E38CB
:10B7680043F00103A4F84E386379D9070AD5B4F831
:10B778004E08820501D4C30718D4B4F854380133ED
:10B78800A4F85438012284F8442894F84728002360
:10B79800012A84F845381CD1A17984F84738E06B30
:10B7A80001F00101BDE8104025F0DABCE36AC0F3FE
:10B7B800470013B1216B9847E4E7E3696269D05405
:10B7C800E369E1680133B3FBF1F201FB1233E36192
:10B7D800D8E710BD38B5124C2179E07810F07EFD1D
:10B7E800A378104A013B32F813300F4A13800F4AEE
:10B7F80012889A4202D00E4B02221A700D4D10F098
:10B8080019F9E0782179A3786970AB70287010F085
:10B8180051FDA880F9F728FB4FF0FF3038BD00BF75
:10B8280018000020805F0308F6400020F840002040
:10B83800FA400020D43F002008B5084B93F8F613CF
:10B8480021B9012283F8F623002008BD4B1E594276
:10B858005941492010F02AF9F6E700BF28230020B3
:10B8680010B5044B044C1A8804492046FAF708FA24
:10B87800204610BD644100201A300020508403087F
:10B8880010B5054B0549B3F8FC2303F6F7442046E9
:10B89800FAF7F6F9204610BD282300205084030843
:10B8A80008B5044BB3F8FA0340F4004010F004FB69
:10B8B800002008BD2823002070B5364B86B01A78C2
:10B8C8008DF80C205A788DF80D2000269A78CDF83E
:10B8D8000E608DF80E209A88ADF810201A7ACDF8EF
:10B8E800126003AD8DF8142095E807006C4603C478
:10B8F8002280294A1278022A1C4630D1274B187810
:10B90800274B8DF8000019788DF8011010F0D2FC43
:10B91800244BADF8040093F8FC3CE3B9052010F083
:10B9280079FA214B0A221E788DF80260694628466A
:10B9380029F0AAFD58B19DF8003023709DF8013018
:10B948006370BDF80430A670A380F9F78DFA4FF044
:10B95800FF3006B070BD062010F05CFAE1E7134B2B
:10B968001B7863B90D4B18780D4B8DF800001978CA
:10B978008DF8011010F09EFCADF80400D1E73046B8
:10B9880010F048FA0A4B8DF800601B88ADF80430B7
:10B99800C7E700BFD43F00205C4100205E41002083
:10B9A8005F410020282300206241002066410020DA
:10B9B8006441002008B50C4B93F90030012B0B4B68
:10B9C80004D1002283F8FC2C002008BD93F8FC0C5D
:10B9D80018B9012283F8FC2CF6E7012818BF0220C9
:10B9E80010F018FAF0E700BFE81A0020282300201A
:10B9F80070B5124C124B94F900401A78012C054688
:10BA08000E4605D1012A01D001221A70002070BD0E
:10BA1800012A03D1002010F0FDF9F7E7022AF3D13B
:10BA2800084B002483F8FC4CFFF7C4FF064B314653
:10BA380028461C70FCF7A6FCE8E700BFE81A0020BF
:10BA48005C410020282300206641002008B5074BF0
:10BA580093F90020064B12B91A70002008BD1A7815
:10BA68000AB90122F8E7FCF72FFCF6E7E81A0020EC
:10BA78005E41002008B5074B93F90020064B12B928
:10BA88001A70002008BD1A780AB90122F8E7FCF7F5
:10BA98001BFCF6E7E81A00205F41002008B50A4BB6
:10BAA80093F8EE2442B193F8EF243AB1D3F8002D7D
:10BAB80042F48032C3F8002D002008BD4FF48030D6
:10BAC800F8F740FFF8E700BF2823002008B5064B29
:10BAD80093F8F10428B1054B01385978C0B214F035
:10BAE8003BFB002008BD00BF28230020EC97002066
:10BAF80008B5064B93F8F00428B1054B01381978BE
:10BB0800C0B220F01AFB002008BD00BF2823002087
:10BB1800EC97002038B5144D95F8FA444E2303FBF2
:10BB2800045495F8F13584F8333595F8F23584F8EE
:10BB380032350E4B186820F067FE95F8F33584F817
:10BB4800113595F8F43584F8123595F8F53584F8FB
:10BB58001335B5F8F635A4F83035B5F8F835A4F846
:10BB68002E35002038BD00BF282300209043002038
:10BB780038B5094B094C186800231A5DC254E118FE
:10BB8800C2184D785570033389789170092BF4D118
:10BB980020F03AFE002038BD90430020952900206F
:10BBA80008B5054B93F8FA050138C0B283F86C065E
:10BBB80014F0ECFA002008BD2823002008B5054B36
:10BBC80093F8F0050138C0B283F8FA04F5F772FA71
:10BBD800002008BD2823002010B5054C94F8FA046D
:10BBE800F5F768FA94F86C0614F0D0FA002010BD46
:10BBF8002823002070B52F4D95F88236022B50D19E
:10BC08000EF0F4FD0446D8B92B492C4E05F6045025
:10BC1800FAF736F82246334629492A48FAF730F81F
:10BC28003346224626492848FAF72AF895F88236F4
:10BC380085F87F36B5F88036A5F88636002070BDC1
:10BC4800224E96F824403CB921491C4E05F6045072
:10BC5800FAF716F82246DEE71E4C6378022B15D059
:10BC6800032B1CD11C4905F60450FAF709F841F2D8
:10BC78007813B26AE458114E4FF47A23B4FBF3F404
:10BC88004FF4FA63B2FBF3F2121BC4E713490B4EED
:10BC980005F604500024F9F7F3FF2246BBE70C49E8
:10BCA800F5E70F490F4E05F604500024F9F7E8FFB1
:10BCB8002246B0E728230020578403085484030849
:10BCC8006A840308343000203C3000203C620020A5
:10BCD8006F830308C48500205F8403086584030814
:10BCE800F78203082C8203082DE9F0411E46002341
:10BCF8008B55074608460C46904629F029F8751ECC
:10BD0800301A2118254440426A1A002AA5EB040378
:10BD180012DA234420211A1B002A11DA0023A35522
:10BD2800094B93F81C1D891B234642463846C9B265
:10BD3800BDE8F041F7F760BE2B5C05F80139E3E791
:10BD480003F80119E7E700BF28230020F8B54B1EC8
:10BD5800012B04460D461D4E0CD81D4BD3F804028A
:10BD6800FCF7AEFDD6F888365B680BB10020984723
:10BD7800F9F77AF8174B00271F70236820465B688D
:10BD88009847A37BC6F88876013B022DA37316D18A
:10BD98002046F7F771FE032205210F4B2046F7F7DF
:10BDA8002BFE236820465B6A984721F044F820F070
:10BDB80067FFC820F6F732FF084B094ADA60094ADC
:10BDC800136823F4005313600020F8BD28230020D3
:10BDD80018000020744800207084030800ED00E07B
:10BDE8000400FA05B83F002070B4154A92F990464D
:10BDF80092F89156214491FBF4F304FB1311D2F805
:10BE0800884682F88C16CBB2A1686B43142404FBD5
:10BE180003130021C2F8203D82F8241D1E790E2E3E
:10BE2800CCB201F1010109D1AC42234628BF2B460F
:10BE3800013B82F8243D70BCF7F71EBE1433EDE7D2
:10BE48002823002038B5164BD3F8882652680546B3
:10BE58001C46BAB994F8250D98B10138C0B284F8D7
:10BE6800250D04EBC00000F6285003C80D4B83E8ED
:10BE78000300FCF733FD284694F98C16FFF7B4FF4E
:10BE8800002038BD93F98D06D3F8203D00EB8000E3
:10BE980003EB800090470028DCDA4FF0FF30F0E732
:10BEA80028230020B029002038B505460C4631B3B8
:10BEB8001C4BD3F888268A4223D093F8252D511C91
:10BEC80083F8251D03F5D16103C903EBC20202F60D
:10BED800285282E803000022C3F8884683F88D269A
:10BEE800236833B19847013003D12846BDE838406C
:10BEF800A8E7FCF7F3FC00212846FFF775FF0020B0
:10BF080038BD93F98D1693F8912691FBF2F402FB54
:10BF1800141283F88D26FCF7E1FC21462846FFF72A
:10BF280063FFECE7282300203E4A3F49107870B5AC
:10BF3800D1F8785D0C4600283ED115B9C1F87C5D72
:10BF480070BD3A4BD3F808120029B8BFC3F80802ED
:10BF5800D3F8083204EB8303D3F8803DC4F87C3D62
:10BF6800002BEDD001231370314BC4F88836002321
:10BF7800A4F88C364FF4005007F04CF8D4F87C0D38
:10BF8800F7F76CFDD4F87C0D427A037A112A4FF04A
:10BF9800010138D884F8901D022184F8911D5B08AE
:10BFA800002184F8921D84F81C2D84F89136D4F869
:10BFB8008816BDE8704077E76DB11C48D0F80812C4
:10BFC800013191FBF5F205FB1213C0F8083204EBBE
:10BFD8008303D3F8805DD4F87C6DAE42B0D094F87A
:10BFE8008D2694F88C1694F8913601FB032384F877
:10BFF8008D36336830465B689847B37BC4F87C5D00
:10C00800013BB373BAE7002584F8911D023A022177
:10C01800023B84F8905D84F8921D84F81C2D84F806
:10C028009136C4E774480020282300201800002017
:10C03800140200202DE9F04FBF4AD2F8783D002BBA
:10C048008BB08046934635DBD2F8943D03F54343E5
:10C05800503398422ED3B94BC2F8940D1E784EBB7C
:10C06800B74B1B780293B74B0299DA88A2F2E342E6
:10C0780092B2184609BBB2F5F97F16D8B3F9041085
:10C0880040F2E142914210DCB3F9022040F2D6635B
:10C098009A420ADDAC4B1B78D80706D4FFF744FF59
:10C0A800AA4B4FF4FA72A3F80C22A94B1A68A24BB8
:10C0B800C3F89C2D0BB0BDE8F08FB2F5F97FB3F94A
:10C0C8000210DFF8889214D8B3F9042040F2E14353
:10C0D8009A420EDC40F2D66399420EDD9A4B1B78E9
:10C0E80013F0010F0CBF06240124D9F814320133D0
:10C0F8001BE040F2D66399423EDC40F2E1429142B5
:10C108003CDDB0F9003093423ADD40F2D66293420A
:10C1180038DC8388A3F2E243B3F5FA7F34D80123ED
:10C128000024C9F81032CBF8984D4FF47A72B8FB56
:10C13800F2F20192B9F90C22C9F81432002A25DD6D
:10C14800DBF89C3D1344019A9B1AA9F80C327A4DEE
:10C15800D5F8203D002B40F0B881D5F8A03D019AD4
:10C1680003F5FA739A42A0D9D5F87C0DF7F736FC97
:10C17800019BC5F8A03D98E70124B6E70224B4E77F
:10C188000324B2E70424B0E70524AEE7002CDED090
:10C19800621ED9F81032DBF87C7D674D03934FF0AF
:10C1A800000AD2B253460492039A524525DC033C56
:10C1B800012CA9F80C32CAD8D9F81422142AC6DDE1
:10C1C800A2F1140193FBF1F3322BA9F80C32BEDC77
:10C1D800D5F8983D0BB9C5F8982DDBF8983DD21ADB
:10C1E8005A4BD3F81002052192FBF1F202448A421D
:10C1F800C8BF0A46C3F81022A9E7D5F888360BB994
:10C20800FA2305E0062C06D1FFF78EFE4FF4FA73E9
:10C218000AF1010AC8E7052C05D13846FFF712FED6
:10C228004FF4FA73F4E7022C3FD195F98D3695F85F
:10C23800242D93422EDA013385F88D36049B012B89
:10C24800DED99BF98D36DBF8202D03EB830302EB57
:10C2580083031A79013A0C2AD2D801A151F822F0A5
:10C2680023C200085DC300080BC300081FC30008F1
:10C2780077C3000849C40008CBC300087DC4000880
:10C28800ADC4000809C20008CBC3000899C3000860
:10C2980011C4000895F88C16013149B23846FFF7E9
:10C2A800A3FD002385F88D36C8E7012CC6D195F883
:10C2B8008D16D5F8202D4B1E5BB203EB830002EBE5
:10C2C800800085F88D36007920B9002BC4BF02396B
:10C2D80085F88D1695F98D36591C06D003EB830326
:10C2E80002EB83031B79002B8AD195F88C16013950
:10C2F80049B23846FFF778FD95F8243D85F88D3624
:10C308009CE7042C7FF47CAFD9683846FFF7CCFD56
:10C318004FF4FA737CE79A68002A3FF471AF042C53
:10C328007FF46EAFD9683846904701303FF475AF57
:10C338004FF4FA736CE700BF2823002076480020EA
:10C3480074480020B8400020643F002018000020F6
:10C35800586000209A68002A3FF452AF042C7FF4FA
:10C368004FAFD968384690474FF4FA7350E7DA6808
:10C37800002A3FF445AFA4F1040CDCF1000141EBC5
:10C388000C0111701A7C42F001021A74FA233FE77B
:10C39800D86800283FF434AF042C028808D142F44E
:10C3A800006202801A7C42F001021A74FA232FE715
:10C3B80040F6010192FBF1F101EBC121521A92B250
:10C3C800EFE7D96800293FF41BAF0868042C02780E
:10C3D80012D191F805C0944502D989790A440270AE
:10C3E8001A7C42F001021A749A68002A3FF408AFD6
:10C3F80019463846904703E791F804C09445EFD2B0
:10C408008979521A0270EBE7D8680168042C0A7817
:10C4180011D10079904201D901320A709A6822B18B
:10C42800D968059338469047059B1A7C42F001026B
:10C438001A74FA23ECE6002AF0D0013A0A70EDE704
:10C44800DA68002A3FF4DCAE10680178042C4FFA51
:10C4580081FC07D192F905E0E645C1DD92791144E6
:10C468000170BDE792F904E0E645B9DA9279891AD4
:10C478000170B5E7D96800293FF4C2AE0868042CFA
:10C48800028807D1B1F806C09445A9D909890A4498
:10C498000280A5E7B1F804C09445A1D20989521ACF
:10C4A80002809DE7D96800293FF4AAAE0868042CE9
:10C4B800B0F9002004D1B1F906C0944590DDE5E754
:10C4C800B1F904C094458BDAE8E795F8903DD5F8C2
:10C4D8007C7D002B40F0B58095F8243D97F80890B6
:10C4E800A9EB0309022399FBF3F95FFA89F9DBF851
:10C4F800A43D03F5C333A03398453B6888BFCBF808
:10C50800A48DDB6A88BF029E384698473B7B1FFA9A
:10C5180080F8002B00F09E80D5F8203D1A790E2A6D
:10C5280040F0928000233B73D5F8200D95F88D36A6
:10C5380059B201EB810200EB820201331279DBB2BE
:10C54800002AF5D097F90D2085F88D16002A0EDB04
:10C558008A4226D095F8913D95F8921D03FB0292E8
:10C56800D2B2AD4B3846F7F747FAA8EB0008B8F156
:10C578001D0F7FF6F2AD95F98D2697F90D30934290
:10C5880013D095F8913D95F8921D03FB0292D2B213
:10C59800A24B3846F7F730FA95F88D367B73A8EB3F
:10C5A8000008B8F11D0F7FF6D8AD0023D5F8204D4F
:10C5B80002939DF8086095F89136B3427FF6CDADA9
:10C5C80023790E2B3FF4C9AD227C900718D595F836
:10C5D800921D95F8912D002B18BF013102FB069290
:10C5E8002368D2B2C9B23846F7F706FA237CA8EB1B
:10C5F800000823F00203B8F11D0F23747FF6ADADD8
:10C60800227CD10776D59BF8913D03FB06969BF8D3
:10C61800903DF6B20BB10136F6B223790D2B00F23C
:10C62800F680DFE813F0DD00F400F400390039008B
:10C638006C0098008E00A200A2002D00AB008300C1
:10C6480077004FF0010952E71A7C42F003021A748E
:10C65800143363E7002E3FF467AF9BF8243DDBF803
:10C66800202D03EB830302EB83039A423FF65CAF72
:10C67800117C4C0744BF41F0010111741432F4E7F6
:10C68800E168002900F0C3800C2206A828F062FFA8
:10C698000C23324606A920E00DF1280A4FF00001CC
:10C6A800032B0AF8101D09D1A3683BB1120705D561
:10C6B80098470C220146504628F04CFF57495046EF
:10C6C80028F012FF95F8903D0BB1013EF6B25046A6
:10C6D80028F03EFB3246C3B251463846FFF704FB0A
:10C6E800237C23F001032374A8EB0008B8F11D0F85
:10C6F8007FF633AD029B01331434029359E7E068A7
:10C708000028F1D00378BBB1454906A828F008FFF6
:10C718000323BEE7E3681A689B68117806A853F8F4
:10C7280021100C2228F016FF0C23B2E7E06800283D
:10C73800DAD003881B05E7D43A4906A828F0F0FEAA
:10C74800E6E7E0680028CFD0036806A9187824F047
:10C7580096F805239DE7E0680028C5D0036806A978
:10C7680093F9000024F08BF8F3E7E0680028BBD0C9
:10C77800036806A9188824F082F8EAE7E068002828
:10C78800B2D0036800891B78584300F5C33006A966
:10C79800A03024F074F89DF81A209DF819308DF80F
:10C7A80019202E228DF81A209DF81D208DF818309A
:10C7B800302A01D02E2A0DD14FF000028DF81D200D
:10C7C8009DF81C20302A01D02E2A03D14FF00002F8
:10C7D8008DF81C20302B04BF20238DF81830B8E7C3
:10C7E800D4F80CA0BAF1000F13D0206828F0B0FAE2
:10C7F8009BF8921D0131014453463246C9B238466E
:10C80800F7F7FAF8237C23F0010323746CE7002080
:10C818006AE7504668E700BFD08203087D840308B2
:10C828007F8403088384030818B9094A82F8B0068C
:10C83800704710B5064CC4F8A00627F04BFC4FF61D
:10C84800FF720223A4F8A82684F8B03610BD00BFF2
:10C85800282300200B4A92F88236022B08D0032B9B
:10C8680004D1D2F8980603685B691847002070471E
:10C87800054A41F29C03D358002B01DD0EF0E4BBBE
:10C888000120704728230020C48500200FB400B57C
:10C8980083B004AB054953F8042B01930020F9F742
:10C8A80027F903B05DF804EB04B07047DDD9000840
:10C8B8002DE9F04FDFF810913B49D9F8A85DDFF872
:10C8C8000CA12C4685B005F1100305F1300B44F896
:10C8D800040B02935E4609F6B45309F55C6809F641
:10C8E800CC57F3EC016AB8EC017AF7EC017AB1ECB9
:10C8F800010A0193FDEEE66ABDEEC77AFDEEE77A1E
:10C90800E4EC016A84ED027AC4ED057A00910391A2
:10C9180028F096FEBAEC010A26F8020B28F090FEE1
:10C92800029BB0809C42DDE90013DAD11F4905F172
:10C938002803F1EC017AFDEEE77A17EE902A23F846
:10C94800022B5B45F5D11A4B1A4A588811781A8878
:10C95800AA879A88DB88E887A5F84020A5F842309E
:10C9680071B105F14403144A03EB4101F2EC017A79
:10C97800FDEEE77A17EE900A23F8020B9942F5D1FB
:10C988000E490F4A0F4BB9F8020E498852681B88A6
:10C99800A5F85E00A5F86410A5F86620A5F868302B
:10C9A80005B0BDE8F08F00BFC4670020683F0020D5
:10C9B800643D0020413D0020003100208C400020D3
:10C9C800784000207E3F0020282300207C43002060
:10C9D8002DE9F04F974C94F882369A1E012A87B0B9
:10C9E80040F2A580032184F88216802014F048FBC9
:10C9F8000646002800F0A280802114F037FB7579E4
:10CA08008D4B96F9027053F8252084F8080EB2F57C
:10CA1800613F14BF00260226022100230092CDE9BF
:10CA2800011638461A46802113F06AFF0C3D032D83
:10CA3800C4F8980600F2EC80402384F87E3A002877
:10CA48007CD07E4B7E495D7D7E4A7F4B0F6894F893
:10CA58008366116898797D4A93F80580DFF8FCC1F0
:10CA680092F800E094F86C2F794BBCF802C0DFF81C
:10CA7800F0B1DFF8F0A1A4F868CF002DC7F3C037F4
:10CA880018BF0127003618BF012611F0020F08BF92
:10CA98000026002110F0FD0F14BF4FF00109894650
:10CAA800B8EB0108B4F88006C4F8101EA2F1190CFE
:10CAB80018BF4FF00108BEEB010E03F1140518BFB3
:10CAC8004FF0010EBCFA8CFC012A4FEA5C1C03F102
:10CAD800800208BF4FF0010CC4F8A85DC3E901113A
:10CAE80003F1EC05C3E903119AF800A0DBF8003064
:10CAF800C4F8AC2D10F1FF3BC4F8B05D0A460D46F2
:10CB0800049318BF4FF0010B01200596D3B2591EAC
:10CB1800152924D8DFE801F030303030303030309B
:10CB28003A26264E2C264A3E3E3E56215226032BB6
:10CB38003FF45BAF474B5A78012A05D8002384F8A5
:10CB48007E3607B0BDE8F08F41F2B5129B5C002B32
:10CB5800F4D1402384F87E3A73E7059931B100FA9D
:10CB680002F10D430133DBB2162B2FD80132CDE78A
:10CB780049460029F3D1F9E79A4534BF002101213C
:10CB88000029EFD000FA02F10D43EBE761460029D6
:10CB9800E5D1EBE7049E02EB4201314411F82E1C6B
:10CBA800003118BF01210029ECD1DBE73946002903
:10CBB800D5D1DBE741460029D1D1D7E77146002915
:10CBC800CDD1D3E759460029C9D1CFE71B20C4F8F6
:10CBD800705F20F013FDD4F87C5FD4F8841F84F8CC
:10CBE800740F00230222C4F8B836A4F8BC36A4F89F
:10CBF800C036A4F8C236C4F8B43684F88C3FC4F8FA
:10CC0800785FC4F8801F84F87E2607B0BDE8F08FEF
:10CC1800D4F80C3E104A03EB4303A2FB03235B0941
:10CC280006D0402BA8BF4023DBB284F87E3A06E743
:10CC38000123FAE72823002028600308A47A0020AB
:10CC4800A06B002048430020843F0020603D002066
:10CC580038310020C4850020D34D62108C4000205C
:10CC680090430020413D002010B5084C94F88236CE
:10CC7800032B05D0FFF7ACFE012384F88D3F10BDD0
:10CC8800802027F02DF90028F4D010BD282300209B
:10CC980038B5364B5B68C3F30803B3B9EFF31183B8
:10CCA8009BB9334A334C1368A06800BF11688B42A4
:10CCB800F9D1314A14684FF47A7101FB04F2101A61
:10CCC800B0FBF4F001FB030320E0EFF31181102324
:10CCD80083F312882748294A84680368DB0344BF22
:10CCE80001231360224B48BF84681D681368C9B2CA
:10CCF80081F31188204A10684FF47A712B4401FBA4
:10CD080000F2121BB2FBF0F201FB03231C4CD4F817
:10CD18009C279A1AB2F5FA6FC4BF002284F8A0279C
:10CD280094F8A02762B1174A12781B2A18D000225B
:10CD38001549D4F814070FF007FF94F8A03723B962
:10CD48000023C4F81437012038BD1048FEF718FB3B
:10CD5800002384F8A0370023C4F81437012038BD15
:10CD6800D4F89C170A4A5B1AD380E0E700ED00E08C
:10CD78005860002010E000E0BC600020B86000208F
:10CD880028230020603D0020C82A0020C45803083A
:10CD9800643D00202DE9F8432C220446002128F0A8
:10CDA8009BFB0123174D184ADFF86480237529205F
:10CDB80040F26C731549A07513262020A261A38345
:10CDC8000E22022384F82060616284F8220084F82D
:10CDD80028202372A377C1462E4605F10807412172
:10CDE800304628F090FB30B1B842A0EB05003CBFBC
:10CDF800A9EB0803235419F8011F0029F0D1BDE855
:10CE0800F88300BFCC580308DC051A0475034308EF
:10CE1800C8840308F8B5F5F74BFE274E054600F120
:10CE2800FA07344696F8B03F06EB8303D3F8900F21
:10CE3800F6F7D6FC38BB94F8B03F04EB8303D3F87D
:10CE4800900FF6F7CDFC28B3F5F732FED4F8B83FCB
:10CE5800401B9842C4F8B40F2BD805F5FA7594F81E
:10CE6800B03F04EB8303D3F8900FF6F7B9FCB0B9E1
:10CE780094F8B03F04EB8303D3F8900FF6F7B0FCB7
:10CE880090B1002005E0F5F713FEB842CAD94FF07B
:10CE9800FF30F8BDF5F70CFEB842CCD9F7E7F5F747
:10CEA80007FEA842DBD9F2E7F5F702FEA842DFD970
:10CEB800EDE70120EDE700BF2823002038B5002466
:10CEC80005460470FFF7A6FF431C11D0012803D1C3
:10CED8002B78A040184328700134082CF2D1054A59
:10CEE8002B7892F8BC1F4B4082F8BC3F012038BD1C
:10CEF8000020FCE72823002003685B6A18470368C2
:10CF08001B6A18470368DB69184703685B69184799
:10CF180010B103685B681847FF2070472DE9F04F90
:10CF28000C46002185B0074608461646F6F724FC4D
:10CF380000210120F6F720FC12F0A0FB022E00F0E1
:10CF48009181042E44F6C01818BF4FF49648C04883
:10CF580000231C25024602E001330A2B06D005FBFC
:10CF68000301897911F00401F6D0D9B22144C9B27C
:10CF7800092913D8032E00F07B81C1EBC103B54802
:10CF880002EB8303C3631C2303FB0121CB799907BD
:10CF980040F16E81B04B0022C3F8C02F05B0BDE848
:10CFA800F08F012E08D1D4F84004414627F01CF830
:10CFB800E06B26F0F5FFC9E1022E08D1E06BFEF721
:10CFC800BBF94146D4F8400427F00EF8BEE1032E21
:10CFD80040F082804FF0000984F858984022494672
:10CFE8009E48DFF87CB228F077FA994B8DF80E90BE
:10CFF8009DF80E20072A09D901219648FBF7F0FC75
:10D008004146D4F8400426F0EFFF9FE19DF80E203A
:10D0180002EB42020BEBC202527C002A4ED09DF872
:10D028000E2002EB42020BEBC2025269002A45D0E5
:10D0380000228DF80F204FF01C0A9DF80F20092AB6
:10D048002CD89DF80E909DF80F2001930AFB023210
:10D058005FFA89F909EB490910790BEBC909F4F76B
:10D0680049FED9F81420019B82422ED19DF80F0069
:10D07800C0EBC00003EB8000FEF75EF99DF80F20BF
:10D08800019B0AFB023A9AF80720D20706D594F8C2
:10D09800582805EBC202012182F8CC169DF80E2013
:10D0A80094F8581802EB42020BEBC20205EBC100E0
:10D0B8005269C0F8C826013184F858189DF80E2026
:10D0C8000132D2B28DF80E2092E79DF80F2001327E
:10D0D800D2B28DF80F20B0E7042E40F03781E06B14
:10D0E800FEF72AF95FE7D5F8C00FF5F713FF0146F9
:10D0F8003846F5F71BFF38E13846F5F70BFF95F88A
:10D10800D32F03469AB9242803D14FF0010285F89A
:10D11800D32F012E05D1194638460193F5F706FF9E
:10D12800019BD5F8C00F1946F5F700FF33E1012A36
:10D1380006D14D2814BF0022022285F8D32FE8E734
:10D14800022A06D13C2814BF0022032285F8D32FD7
:10D15800DFE7032A10D10A2802D985F8D38FD8E748
:10D16800042285F8C60F85F8C58F85F8C88F85F81D
:10D17800C70F85F8D32FCCE7042A09D195F8C72F14
:10D1880085F8D40F424085F8C72F85F8D3BFC0E78C
:10D19800052ABED195F8C51F95F8C69F95F8C70F03
:10D1A800494509D24A1C2944584085F8C70F85F8D3
:10D1B800C52F81F8C93FACE79842CED195F8D41F66
:10D1C80085F8D3AFF429A4D1B9F1000FA1D1242156
:10D1D800384685F8D39FF5F7A9FE4D213846F5F76F
:10D1E800A5FE3E213846F5F7A1FE49463846F5F733
:10D1F8009DFEF4213846F5F799FEF4213846F5F7F7
:10D2080095FE032E17D0E06B437901689D08022331
:10D21800AB40DB439BB20B61CD682B40CB60007900
:10D228002021FEF779F8E06B494623F0ECFEE36B2A
:10D2380018680EF07FF8D4F84004002123F0E3FECC
:10D24800D4F84034186805B0BDE8F04F0EF072B855
:10D25800F47B0308E07A002028230020F02900202E
:10D26800E06C0020FF2C4FF416487FF470AE0326C4
:10D27800514C524D84F8576895F8C40F22F008FFB6
:10D288004F4B236004F1400103234FF48062637124
:10D298006161002304F244414FF00109032EC4F8F0
:10D2A8004004C4F80880A371E362E260C4E907336C
:10D2B800A1612261C4E9093384F84838A4F8449884
:10D2C800C4F85038A4F8543884F856380DD0D4F837
:10D2D8003CA09AF80400F4F70DFDA0635046FEF751
:10D2E8003CF849462046FBF77BFB3220F5F796FCD5
:10D2F800002E7FF456AED4F84084D8F800000EF023
:10D3080019F840462F4A2221F5F79CF92E4BC4F80C
:10D318005C3832462D494046F5F7E8F8D4F83C80A9
:10D32800D8F800000EF006F8264A4FF6FF7140467E
:10D33800F5F788F93146404623F012FF244BC4F82C
:10D348006038324623494046F5F7D0F8C5F8C04F53
:10D358004FF0060A022E12D0D5F8C00FF5F7E2FDFD
:10D3680068B101210020F6F707FAD5F8C00FF5F7E4
:10D37800D9FD014600287FF4B6AEF6F7FDF9384628
:10D38800F5F7D0FD88B101210846F6F7F5F94FF019
:10D39800050B4FF000083846F5F7C4FD0146002894
:10D3A8007FF4AAAE0120F6F7E7F9042ED4D00520C1
:10D3B800F5F734FCCEE700BFE07A002028230020F0
:10D3C800E458030840420F00F1B300083C830020F2
:10D3D80021B50008408300202DE9F04F764A85B03A
:10D3E8001378029003F0FF070392002B40F082802D
:10D3F800724CDFF8D0C1B4F8DC1F01914FF03C0942
:10D40800B4F8DE1F94F8D82F94F8D95F94F8DA3F6F
:10D41800009149469CF802609CF803E0C6F1FF06BB
:10D42800B6B2002E00F0C480C6F1FF060EFB06F669
:10D43800BCF80080B8FBF9FA3612BAF1050F0ED81D
:10D44800DFE80AF0035B6E7F92A3F3B2AEEB060649
:10D4580008FB06F6B6FBF1F51D44EDB272460298DC
:10D4680001280BBF2E02160246EA024646EA054686
:10D478004FF0170E1E4307EB0E0B012000FA0EFAB1
:10D4880000981AEA060F82460198ABEB0E0808BF0F
:10D4980082461FFA88F84A481EF1FF3E00F808A0A5
:10D4A800EBD21837BFB2B7F5407F0CF1040CB1D1FD
:10D4B80084F8D82F84F8DA3F039AA4F8E07F202371
:10D4C800A4F8E23F0123137094F8E43F84F8D95F8D
:10D4D80083B1D4F8E83F40F22A325A60D4F8EC2FEE
:10D4E80000215162118841F0010111801A6842F04F
:10D4F80001021A6005B0BDE8F08FB8FBF1F201FB3C
:10D5080012881FFA88F8F3B2C8F13C08AEEB060699
:10D5180006FB08F2B2FBF1F21A44D2B275469EE756
:10D52800B8FBF1F301FB1388F2B21FFA88F8AEEBEF
:10D53800060608FB06F3B3FBF1F31344DBB27546AA
:10D548008DE7B8FBF1F301FB13881FFA88F8F2B2F4
:10D55800C8F13C08AEEB060606FB08F6B6FBF1F58B
:10D568001544EDB273467AE7B8FBF1F301FB138873
:10D57800F5B21FFA88F8AEEB060608FB06F6B6FB0E
:10D58800F1F22A44D2B2734669E7B8FBF1F301FB22
:10D5980013881FFA88F8F5B2C8F13C08AEEB060606
:10D5A80006FB08F3B3FBF1F32B44DBB2724656E7F4
:10D5B80073467546724652E79340002028230020A0
:10D5C800F4440020DC3E002038B54E4C94F900109D
:10D5D800002959D04C4B93F8F7230AB983F8F7136D
:10D5E800B3F8FC231AB9E2880AB1A3F8FC23474A26
:10D5F800108810B9A08800B110800229E27805D1FE
:10D6080012F0080118BF012183F8FC1C404B414966
:10D618001B78414DCB5C85F81832404B1B78002BAA
:10D6280033D194F901303E48082193FBF1F1405C75
:10D63800594201F0070103F0070358BF4B42313349
:10D64800DBB285F81B3202F00A030A2B85F81A02AE
:10D6580034481DD1E2883449F8F712FB202385F8B5
:10D668002132E3789A0730D513F0040F0CBF4F230B
:10D67800492385F823325223502285F82432002387
:10D6880085F8222285F8253238BD46235520D8E76B
:10D69800D10704D5A2882449F8F7F2FADEE794F90D
:10D6A8000130594201F007014FF0080293FBF2F2F2
:10D6B80003F0070358BF4B4203EBC2031B4A1A4946
:10D6C80032F81320F8F7DCFAC8E794F9002094F947
:10D6D8000230022A164A07D152F833201549164853
:10D6E800BDE83840F8F7CCBA272B06DC182B06DC47
:10D6F8000F2BD4BF00230123EEE70323ECE702231B
:10D70800EAE700BFE81A002028230020644100202F
:10D718005C41002087840308180000205D41002038
:10D728008B8403083502002050840308205F030817
:10D73800985E0308DE8103083A020020074BD3F8FD
:10D74800782D042A08D0511CC3F8781D03EB8203F6
:10D75800C3F8800D0120704700207047282300205F
:10D7680070B5144E96F88236022B05460DD0017816
:10D778000446E1B1D6F89806F5F7D8FB15F8011F6D
:10D788000029F7D12C1B204670BD27F0E1FA04468A
:10D79800D6F89C06037E13F0060FF4D090F82830D4
:10D7A800002BF0D1294622460CF0FAFBEBE70C4699
:10D7B800204670BD2823002010B51A4B93F8822606
:10D7C800022A82B006D00146D3F89806F5F7AEFBD8
:10D7D80002B010BDD3F89C368DF8070093F91A10E3
:10D7E8004A1C0FD05A6840F2FF14C2F30802A24242
:10D7F80008D002EB41220C4950545A6801325A6051
:10D8080002B010BD1A7E12F0060FE1D093F828205E
:10D81800002ADDD1184601220DF107010CF0C0FBEA
:10D82800D6E700BF28230020DC850020F8B5021FBA
:10D838000446064600F10807002152F8043F03F1A8
:10D8480020003F2803F1080503F102033DD80F2DFE
:10D8580018D8032B02D9002908BF01219742ECD11F
:10D86800012921D002290FD1206800F03F0040F0A3
:10D878008000FFF7A1FF2079FFF79EFF207ABDE81F
:10D88800F84099E70221E9E7D4E90030A2681B01D2
:10D89800800000F00C0003F03003034302F00300A3
:10D8A8001843BDE8F84087E7206800F00F0040F013
:10D8B8004000FFF781FFD4E9013000F00F0040EA93
:10D8C8000310C0B2BDE8F84076E704F10C073A4609
:10D8D800002552F8043D03F18001FF2903F50040BB
:10D8E8004FEA850506D9B0F5803F03F500031AD243
:10D8F80045F00105A242ECD165F03F00C0B2FFF748
:10D908005BFF05F00303022B327828D0032B104667
:10D9180017D0012B0FD0FFF74FFF0436B7424FEA5D
:10D92800A505EED1F8BDB3F1807F34BF45F00205FF
:10D9380045F00305DEE7FFF73FFF7078FFF73CFF90
:10D94800EBE7FFF739FF7078FFF736FFB6F902000B
:10D95800C0B2FFF731FF96F90300C0B2DBE710460B
:10D96800FFF72AFF7078FFF727FFB6F90200C0B269
:10D97800FFF722FFD1E700BF0EB470B583B007AC44
:10D988000646482054F8045BFFF716FF2020FFF7EF
:10D9980013FF3046FFF7E4FE3A20FFF70DFF2A4653
:10D9A80023460A4901940020F8F7A2F804460A2001
:10D9B800FFF702FF064AD2F8943603341B1BC2F85D
:10D9C800943603B0BDE8704003B07047DDD9000855
:10D9D800282300200846EFE62DE9F04F5C4DD5F8E6
:10D9E800F44F85B0904600290CBF04220622661C1D
:10D9F800DDF838900F9F009260D0A1453BDDA3EB86
:10DA0800080A57B1109BDA1B04FB02F20123B95C28
:10DA1800D5F8702F8B40134226D0D5F8F06F04FB51
:10DA28000AF408EB040B96BB58F8040027F090F9A9
:10DA3800411D0846FAF76EFF78BBD5F8940695F8AD
:10DA4800F82F401AC5F8940692BB012285F8F82FE2
:10DA58003EBB58F80400FFF783FE9BF904104B1CEB
:10DA680002D03C48FEF712FFD5F8F44F01344C457C
:10DA7800C5F8F44FC5DBA14552D0D5F8F00F009B8F
:10DA8800834294BF0020012005B0BDE8F08F032138
:10DA98000846FAF73FFF0028CFD0012005B0BDE8BF
:10DAA800F08FB3442C489BF80410FEF7EFFEDBE739
:10DAB8002C20FFF781FED5F8F06FC9E7D5F8F0AF55
:10DAC800924503D3002005B0BDE8F08F234A02EB4E
:10DAD8008A020646526E01921046CDE9021327F0DB
:10DAE80037F90B30FAF716FFDDE901210446039BED
:10DAF8000028D2D1BAF1030F98BF314618480193D4
:10DB0800FEF7C4FED5F89416D5F8F42F85F8F84F2B
:10DB1800091A541CC5F89416C5F8F44F019B6CE714
:10DB28000120FAF7F7FE0028A7D1D5F894360A2085
:10DB3800013BC5F89436FFF73FFED5F8F00F4FF0DC
:10DB4800FF330130C5F8F00FC5F8F43F97E700BF81
:10DB580028230020E4840308EC840308A858030859
:10DB6800D48403087F2810B5044607D964F07F00E1
:10DB7800C0B2E409FFF720FE7F2CF7D8E0B2BDE879
:10DB8800104019E638B5044600EB410534F9023B6C
:10DB9800D81780EA4300FFF7E5FFA542F6D138BD64
:10DBA800C31783EA4000DDE7F8B50F4BD3F8A85D4B
:10DBB800D3F8AC4DD3F8B06DA9B1831E00EB410783
:10DBC80027441E4404441D4434F9022B36F9023F0D
:10DBD80035F9020F134403EBD373A0EB6300FFF78F
:10DBE800DFFFA742F0D1F8BD28230020F0B52B4D68
:10DBF8002B49D5F8FC4FD5F8B4762A48D5F8843F98
:10DC080095F8F96F95F8FA2F097890F82000A7424F
:10DC180085B0254C27DB04F8F46C44F8F83C04F88C
:10DC2800F30C04F8F21C04F8F12C01AE5320FFF7B2
:10DC3800C3FD54F8F80CFFF795FF14F8F40CFFF740
:10DC480091FF14F8F31C14F8F22C14F8F13C039328
:10DC58003046CDE90112FFF7E9FD0023C5F8B436D7
:10DC6800012005B0F0BD54F8F87C8DF80860BB427F
:10DC78008DF80B2001938DF809008DF80A10A4F196
:10DC8800F80201AE04D096E8030082E80300CDE76D
:10DC9800716853689942F6D10020E2E728230020F2
:10DCA800663F0020943F0020203400202DE9F04FEB
:10DCB800784CB4F8BC368BB00546002B40F0F680A3
:10DCC800B4F88036002B00F09E802846FEF7F0FD61
:10DCD800D4F8A86D49203546FFF76EFDD4F8B8068C
:10DCE800FFF740FF55F8040BFFF73CFF284626F0E6
:10DCF80027FA06F1100026F023FAD4F8703FDA0369
:10DD080000F19D80D4F8703F9B0300F18F80D4F818
:10DD1800703F5F0300F1BA80032106F12800FFF786
:10DD280031FF5D4BB6F92E001B8AC01AFFF71AFFA8
:10DD3800D4F8703FDD0400F19A80980400F18D80DA
:10DD4800190400F18580032106F13000FFF71AFF5E
:10DD5800D4F8703FDA025FD49F0257D4B6F9443042
:10DD680007EE903A4D4BF8EEE77A13ED3C7A77EEF2
:10DD7800C77AFCEEE77A17EE900AFFF7F3FE484BF6
:10DD88001B78012B0ED906F1440707EB430706F170
:10DD9800460535F9020BB6F94430C01AFFF700FF03
:10DDA800AF42F6D1D4F8703F9D0525D4D4F8A81D0C
:10DDB8003C483D4AC4F8AC1D0B1A9B1003EBC30545
:10DDC80003EB4503C3EB432303EB8343C3F1010395
:10DDD80082FB0352A2EBE37202EB42029B1A6C2213
:10DDE80002FB03030122C4F8B01DC4F8A83D84F85F
:10DDF8008C2F0BB0BDE8F08FB6F95E00A0F2DC50B6
:10DE0800FFF7CEFED2E7FFF7F1FE5EE7042106F149
:10DE18003C00FFF7B7FEA1E7032106F13600FFF744
:10DE2800B1FED4F8703F9F0298D5EFE7306AFFF74C
:10DE3800B7FED4F8703F5F037FF56EAF26E0F06958
:10DE4800FFF7AEFED4F8703F9B037FF560AFEDE7B8
:10DE5800B6F86800FFF786FE75E7B6F86600FFF7C4
:10DE680081FED4F8703F19047FF56DAFF0E7B6F87E
:10DE78006430B4F8680FC01AC0F30D00FFF772FEE3
:10DE8800D4F8703F98047FF55BAFE6E7706AFFF758
:10DE980087FE41E728230020A06D002020340020C1
:10DEA800413D00204C31002056555555D4F87C6F23
:10DEB800D4F8783FB34207D094F87E36C4F8786F28
:10DEC800093B012B40F27481D4F8807FD4F8846F29
:10DED800B74207D094F87E36C4F8806F093B012B0F
:10DEE80040F25981B4F8C236002B82D1B4F880369A
:10DEF800002B3FF47EAFFFF779FE2846FEF7D8FCEB
:10DF08005020D4F8A88DD4F8AC9DFFF755FCD4F870
:10DF1800A83DD4F8B02DD4F8AC1D12681B68086869
:10DF28001344A3EB400002AEFFF73AFE09F10402E6
:10DF380008F10401304625F021FF304626F000F9AB
:10DF480009F1100208F11001304625F017FF30469C
:10DF5800FFF76CFC10250127D4F8703F07FA05F28B
:10DF68001A4240F0C6800135132DF5D108F1280278
:10DF780009F12800B24608F13007314632F9023B70
:10DF880030F9025B9742A3EB050341F8043BF5D156
:10DF980006AA002552F8043DAD0003F10801EDB2D0
:10DFA80033B10F2903F1800300F29C8045F001058D
:10DFB8009642EFD14FF0000B2846FFF7FDFB5F4676
:10DFC8005A4605F00303022B00F08380032B71D01F
:10DFD800012B64D00137042F4FEA9505F1D1002AAF
:10DFE80040F02581D4F8703FD80403F4005203F4BC
:10DFF800004100F19780002A40F0EF8059B1B8F84D
:10E008006830B9F868209B1A0293029BD81780EAF7
:10E018004300FFF7A7FD03213020FFF7C5FDD4F823
:10E02800703FD90200F1F4809A0200F1EC80824B33
:10E0380044201978FFF7B8FDD4F8703F9B0506D542
:10E04800B8F95E00B9F95E30C01AFFF7A9FDD4F837
:10E05800A81D7A487A4A0B1A9B1003EBC30503EBF9
:10E068004503C3EB432303EB8343C3F1010382FB63
:10E078000352A2EBE37202EB42029B1A6C2202FBF0
:10E088000303D4F8AC2DC4F8A83D0123C4F8AC1D93
:10E09800C4F8B02D84F88C3F0BB0BDE8F08F56F86B
:10E0A8002710002A40F0BB804FEA011B5FFA8BFB68
:10E0B8001A468FE756F827000192002A60D1C0F36C
:10E0C8000720FFF779FB16F82700FFF775FB019A81
:10E0D80080E756F827000192BAB9C0B2FFF76CFB87
:10E0E800019A77E7FF2B94BF45F0020545F0030539
:10E0F8005EE7AB0008EB03024B4452F8240C53F8DC
:10E10800243CC01AFFF74CFD2DE7C0F3031040EA8A
:10E118000B00FFF751FB56F82730019A1B015FFAF5
:10E1280083FB57E7B8F86430B9F864001B1A029308
:10E13800002A47D0B8F86630B9F866209B1A0393CE
:10E148000225002953D1AD007319002053F8042D7E
:10E158004000C0B20AB140F001009E42F6D1FFF77C
:10E168002BFB2E4402E056453FF455AF5AF8043BCA
:10E17800002BF8D0D81780EA4300FFF7F3FCF2E74A
:10E18800C0F3033040EA0B00FFF716FB56F82700F0
:10E19800C0F30710BDE74520FFF70EFB1E20FFF771
:10E1A8000BFB3046FFF7DEFC3846FFF7DBFC99E651
:10E1B8004520FFF701FB0020FFF7FEFA3046FFF786
:10E1C800D1FC81E600293FF421AFB8F86830B9F8EE
:10E1D80068209B1A03930225B5E7B8F86630B9F8AA
:10E1E80066209B1A0293012500293FF40EAFB8F868
:10E1F8006830B9F868100AAA02EB85025B1A42F87F
:10E20800203C01359FE704213C20FFF7CDFC0EE7B9
:10E2180003213620FFF7C8FCD4F8703F04E701F06B
:10E228000F0141EA0B00FFF7C7FA0022D2E6584671
:10E23800FFF7C2FAD6E600BF413D00204C3100206E
:10E24800565555551F4A204B116800221F29C3F8FF
:10E25800B826A3F8BC26A3F8C026A3F8C226C3F89C
:10E26800B42625D03F291ED04FF4FA42B2FBF1F173
:10E27800A3F8BE16B3F88016B3F9BE2629B19142A9
:10E2880001DD1F2A19DC92FBF1F1A3F8C41693F8FB
:10E29800821600314FEA022218BF0121C3F8FC2F71
:10E2A80083F87E1670474FF40072A3F8BE26E1E7A4
:10E2B8004FF48062A3F8BE26DCE70121A3F8C41658
:10E2C800E5E700BFC06700202823002038B5084CC8
:10E2D800B4F9BE56B4F9C4162846F7F799FEB4F84F
:10E2E8008036C0B200FB03F090FBF5F0C0B238BD39
:10E2F800282300202DE9F041A74C94F87E36013BF5
:10E3080090B005460A2B28D8DFE813F051006000CA
:10E318007200A70027002700C600DE0058017C0114
:10E328008D019E4B5A78032A2FD141F2A401012274
:10E33800595C84F8B026002900F0CF8641F2E80144
:10E34800595C002900F0A28641F22C129A5C002A3E
:10E3580000F09B86002384F8B03694F88236022BAE
:10E3680012D094F88436012B00F0AC81022B08D12E
:10E3780094F87E36012B04D194F88D3F002B00F0E1
:10E38800DD8110B0BDE8F081844B41F2B5129B5C91
:10E39800002BE6D094F88D3F012284F87E26002BCE
:10E3A800EFD0002384F88D3F10B0BDE8F0817C4B9E
:10E3B8001B78DE07D1D5802025F092FD08B112F038
:10E3C80087FAFEF705FB94F88236C8E794F8823698
:10E3D800022B00F01F85734A1268C4F8F42F00233B
:10E3E8000322C4F89436C4F8F03F84F87E26B8E7D0
:10E3F800FCF7E2FD6B4AD4F8F43F126864339342A9
:10E40800ABD24020FAF786FA0028A6D1D4F8F03F1C
:10E41800654D40260EE0FFF7CFF9D4F89426D4F8DE
:10E42800F03F013A0133013EC4F89426C4F8F03FA6
:10E4380000F016862B4493F87C301846002BEAD15E
:10E44800042300214FF0FF3284F87E36C4F8F01F11
:10E45800C4F8F42F94F8823681E7FCF7ADFD534AEF
:10E468000292A2F10C03252101930091A2F10A0363
:10E478005021163A4920FFF7AFFA00287FF46DAF14
:10E4880007234FF0FF3284F87E36C4F8F00FC4F843
:10E49800F42F94F8823662E7FCF78EFD444B052092
:10E4A80000210090A3F10802CDE901115320FFF7E4
:10E4B80093FA00287FF451AF082384F87E36C4F815
:10E4C800F00F94F882364AE73A4DFCF775FD15EDE2
:10E4D8003C0A27F0B5F815ED3B0A064627F0B0F8D8
:10E4E80001464020FAF716FA00287FF436AF324A80
:10E4F800D4F8F03F50784A2B00F25885DFE813F043
:10E50800BC010402FD01ED01E701E001D001C901F0
:10E51800C201F102EA02F802E302DA02D002C902F9
:10E52800BB02B402AD02A6029D0294028B028202D3
:10E5380074027C046E04630458044D0442043704D6
:10E548002C0421041604AC03A10398039003880348
:10E55800800378036F0366035D0355034D0344038B
:10E568003B0333032B0323031B0314030D0306038D
:10E57800FF02A801A001980185017E0177017001C1
:10E58800690162015A0152014B0144013D01360102
:10E598002801B601AF0100BF28230020C485002050
:10E5A800643F002058600020A85803088A590308CF
:10E5B800385B030820340020EC9700201B201FF054
:10E5C80079F8D0B1B4F8BC36BBB94520D4F8B866F0
:10E5D800FFF7F2F80E20FFF7EFF83046FFF7C2FA20
:10E5E8002846FFF7BFFAD4F8FC3FC4F8B4362846EB
:10E5F8000A2384F87E36FFF759FBFAF7BBF994F83B
:10E608008236ACE694F8743F002B57D01B201FF0DD
:10E6180051F8002852D194F88D3F002B4ED1092390
:10E6280084F87E36E9E794F88236022B31D194F8E3
:10E638008C3FD4F89C56002B40F083801DB32B7878
:10E648000BB395F82830002B7FF49EAE2A7E696ABA
:10E65800AB63042085F83C3012F0080385F82800E5
:10E66800C5E90B1103D0AE4B41F294129B586B6372
:10E6780000266E62C5E90266284625F02BFD0523B3
:10E688002E6485F8283000220423C4F89C2684F8D8
:10E69800B036A44AD4F8F43F1268C833934204D37E
:10E6A800FEF7D8F800283FF458AE94F88236032BCA
:10E6B80000F08C84012284F87E2650E62846FFF775
:10E6C800F5FA9AE7984B94F87E561B78DB0702D444
:10E6D8001EF0FEFE30BB934E944A336852F89C2CD1
:10E6E8009A4227D8012D3FF44CAE94F88D3F002B69
:10E6F8003FF447AE0B2D0ED80123AB4040F6030282
:10E7080013EA02077FF44DAE13F4C06F03D0093D3E
:10E71800012D40F2CC843368C4F8F43F0B2384F80D
:10E728007E363EE67F4B814A1B6803F59C530833CF
:10E7380042F89C3C012D7FF424AE1DE6FEF794FAC6
:10E748001FE6284600210BF027F900289BD104E694
:10E75800774B7849DA897848FFF70EF9D4F8F02F23
:10E7680094F882360132C4F8F02FF8E5704B7149FD
:10E778001A887248FFF700F9F0E76D4B6D499A78EF
:10E788006F48FFF7F9F8E9E7694B6A491A796D4864
:10E79800FFF7F2F8E2E76C4B66491A7A6B48FFF725
:10E7A800EBF8DBE7684B634993F822206848FFF7EA
:10E7B800E3F8D3E7644B5F4993F820206548FFF7F7
:10E7C800DBF8CBE7604B5B499A7F6348FFF7D4F8E7
:10E7D800C4E715F8A02C57496048FFF7CDF8BDE706
:10E7E80015F8AD2C53495E48FFF7C6F8B6E75D4B00
:10E7F80050495A795C48FFF7BFF8AFE715F8BD2CC8
:10E808004C495A48FFF7B8F8A8E735F8C03C9FEDDF
:10E81800587A4849574807EE903AF8EEE77A67EE93
:10E82800877AFDEEE77A17EE902AFFF7A5F895E7C5
:10E83800514A5249538A5248D289FFF79DF88DE7C9
:10E848004D4A4E49138A4F489289FFF795F885E754
:10E85800494B38495A794C48FFF78EF87EE7D4F887
:10E86800002D34494948FFF787F877E7927831490E
:10E878004748FFF781F871E7464A47494748FFF795
:10E888007BF86BE72A4B2B491A8A4548FFF774F83F
:10E8980064E7B4F8802627494248FFF76DF85DE73A
:10E8A800FFF714FDB4F9C4160546B4F9BE06F7F728
:10E8B800AFFB2A46C3B23C493C48FFF75DF84DE739
:10E8C800B4F9BE261B493A48FFF756F846E7394AD5
:10E8D80031493948FFF750F840E705A8F6F7B8FC82
:10E8E80005A935F9E82C08A80023F7F7DFF908AAE5
:10E8F80029493248FFF740F830E7314B314A32496D
:10E908003248FFF739F829E7314A324B3249334860
:10E91800CDE90032324B334AFFF72EF81EE700BF2D
:10E92800C485002058600020643F00202034002067
:10E93800A06D0020EC840308C0890308B08903088F
:10E948009C89030888890308A47A0020748903082D
:10E95800588903083C890308288903081089030893
:10E96800008903087C490020F0880308E088030830
:10E978000000C842D4880308A06700200C8603085A
:10E98800C0880308B0880308A0880308E089030842
:10E99800D4890308008503080C850308108503083B
:10E9A800E0850308D8850308C4850308CC850308D7
:10E9B800B88503083C330020AC8503089885030814
:10E9C800688503087485030880850308888503081B
:10E9D80058850308468403083485030844850308DA
:10E9E800208503082885030804EB00109E4990F849
:10E9F800103690F80F2690F8110600909B48FEF705
:10EA0800BBFFABE604EB00109949B0F81A26994809
:10EA1800FEF7B2FFA2E604EB0010954990F818261D
:10EA28009548FEF7A9FF99E604EB0010904990F885
:10EA38000D269248FEF7A0FF90E604EB00108C49E3
:10EA480090F80C268E48FEF797FF87E615F8D02C2D
:10EA580087498C48FEF790FF80E68B4B84499A786B
:10EA68008A48FEF789FF79E6894B81491A688948FF
:10EA7800FEF782FF72E6884B9B79012B7FF46EAE1E
:10EA8800B4F90634B4F9082484498548FEF774FFBC
:10EA980064E6B4F8682F83498348FEF76DFF5DE6A6
:10EAA8007D48824983784278007800908048FEF754
:10EAB80063FF53E6D4F8703FDA0400F106830F23AE
:10EAC800C4F8F03F4AE67B4B76499A8A7A48FEF7C3
:10EAD80053FF43E64FF07E5278497948FEF74CFFE2
:10EAE8003CE6784B62495A8A7748FEF745FF35E697
:10EAF8008BB2B2B269497548FEF73EFF2EE6624B0B
:10EB08005B491A797248FEF737FF27E65E4B58498A
:10EB1800DA787048FEF730FF20E615F8C72C54491C
:10EB28006D48FEF729FF19E615F8C82C50496B48BF
:10EB3800FEF722FF12E66A4B4D491B6869485A8D59
:10EB4800FEF71AFF0AE6664B49491B6866481A8DA4
:10EB5800FEF712FF02E6624B45491B6863485A8F6D
:10EB6800FEF70AFFFAE55E4B41491B6860481A8FB9
:10EB7800FEF702FFF2E55A4B3D491B685D4893F8E2
:10EB88003720FEF7F9FEE9E5554B39491B685A4825
:10EB980093F83620FEF7F0FEE0E5514B34491B6848
:10EBA80056489A8EFEF7E8FED8E54D4B30491B686B
:10EBB80053485A8EFEF7E0FED0E5494B2C491B68B6
:10EBC800504893F82D20FEF7D7FEC7E5444B284957
:10EBD8001B684D4893F82C20FEF7CEFEBEE5404B4F
:10EBE80023491B68494893F82720FEF7C5FEB5E579
:10EBF8003B4B1F491B6846489A8CFEF7BDFEADE5A6
:10EC0800374B1B491B6843485A8CFEF7B5FEA5E5F0
:10EC1800334B17491B684048DA8BFEF7ADFE9DE57C
:10EC28002F4B13491B683D481A8CFEF7A5FE95E546
:10EC38002B4B0F491B683A4893F82620FEF79CFE99
:10EC48008CE5274B08491D6836482B7FEA7E6D7F87
:10EC58000095FEF791FE81E5214B05491B68324876
:10EC68001A7EFEF789FE79E5C8860308D48603086C
:10EC7800EC840308B8860308AC860308A08603085A
:10EC88009886030884860308A06700207486030812
:10EC9800C067002068860308843F00200C860308AC
:10ECA8005886030858BB03085086030834860308AF
:10ECB800408603085443002020860308F88503088B
:10ECC80000860308A06D0020EC850308148603085D
:10ECD8008C880308808803087088030874880308F0
:10ECE800904300205C8803084C8803084088030888
:10ECF8003088030818880308FC870308E887030896
:10ED0800D0870308BC870308AC8703089C870308DF
:10ED180088870308788703086C8703085C870308DB
:10ED2800488703084087030838870308B74BB84962
:10ED38001D68B848AB7D6A7DED7D0095FEF71CFE29
:10ED48000CE5B24BB2491D68B348EB7CAA7C2D7D1B
:10ED58000095FEF711FE01E5AC4BAD491D68AF48C3
:10ED68002B7CEA7B6D7C0095FEF706FEF6E4A74B4C
:10ED7800A7491D68AA486B7B2A7BAD7B0095FEF7E7
:10ED8800FBFDEBE4A14BA2491D68A648AB7A6A7A61
:10ED9800ED7A0095FEF7F0FDE0E49C4B9C491D6878
:10EDA800A148EB79AA792D7A0095FEF7E5FDD5E41F
:10EDB800964B97491D689D482B79EA786D7900959F
:10EDC800FEF7DAFDCAE4914B91491D6898486B78C3
:10EDD8002A78AD780095FEF7CFFDBFE404EB00106C
:10EDE8008B4990F8163690F8152690F8170600907B
:10EDF8009048FEF7C1FDB1E404EB0010844990F897
:10EE0800133690F8122690F8140600908A48FEF7F8
:10EE1800B3FDA3E494F8B036052B3FF6B5AA01A2DA
:10EE280052F823F02BE3000891E3000845EE0008B0
:10EE38001DEF000853EF0008AFEE00087F4F804E2B
:10EE4800DFF81882D4F8A00605AA39460AF090FC23
:10EE5800012831464FF003027FF47FAA059D28461A
:10EE680085B32B7873B326F063FB03224146002851
:10EE7800E8D105F1080026F05BFB03460028E1D144
:10EE880055F8030F08902A798DF8242008A88DF8E2
:10EE98002530F6F789FAD4F8AC36984238BF1846C8
:10EEA800C4F8AC06CEE7674A674B1268C4F8F42F7B
:10EEB80003210022C4F89426C4F8F02F84F87E16A3
:10EEC800FFF763BAD4F8A01691F91A20551C0AD096
:10EED8005D4B02F5817203EB0213FF20DA796FF3C1
:10EEE8000002DA71887691F91B20501C0FD0564B1E
:10EEF80002F5817203EB0213FF25DA79C2F34500AC
:10EF0800013820EAE07060F34602DA71CD76032317
:10EF180084F8B0364D480378002B7FF41EAAD4F845
:10EF2800A056002D00F0A98095F82830002B7FF41A
:10EF380014AA28384422294626F06EFA28460021C9
:10EF48000AF02AFD0023C4F8A036414BD4F8AC5689
:10EF5800404F0FCB08AE07C60DF1270133706B1C6D
:10EF68000DF12205A7FB0302D20802EB8200A3EBF6
:10EF78004003303301F801398D421346F2D1324B48
:10EF880041F2A4010122595C84F8B026002900F05E
:10EF98008C8041F2E801595C41B341F22C129A5C31
:10EFA8001AB3042384F8B036FFF7D7B9FDF752FC3B
:10EFB80000283FF4D2A9D4F8FC3FC4F8B4360A2399
:10EFC80084F87E3694F88236FFF7C9B9D4F89806E3
:10EFD80011F052FC94F8083E0022022BC4F898263F
:10EFE80048D094F88236FFF765BB022202EB021282
:10EFF80003EB820303F58550174B009308A93C23C4
:10F00800202204300FF00AF8FFF7A7B99043002038
:10F01800C88603082C870308248703081C8703086D
:10F02800148703080C87030804870308F886030875
:10F03800F0860308E8860308E0860308CC29002048
:10F04800F884030858600020C4850020A497002095
:10F05800F8890308CDCCCCCC55890008FC8403087A
:10F068001D4494F8823695F87C20002A7FF477A90D
:10F07800FFF7E6B912F03AF8B3E726F003F90028EB
:10F088003FF46BA9D4F8A05658E70222442101FBAB
:10F09800023303F58550124B0093102213231149B4
:10F0A80004300EF0BBFFFFF758B90A469EE745202B
:10F0B800FEF782FBFF20FEF77FFB0B48FEF750FBB5
:10F0C8003846FEF779FBFFF726BB94F80124074979
:10F0D8000748FEF751FCFFF741BB0A46D6E700BFD9
:10F0E80031C80008F0840308EC89030858BB0308FA
:10F0F800288603082DE9F04F2DED028BA54B1B7DCB
:10F10800012B85B000F0CD83022BA34B01931A4647
:10F118000CBF0723002302F8983CA04B1B78132B45
:10F1280000F2358101229E499A400A4208BF002315
:10F1380001989C4900F8973C00230B60C1E9013312
:10F14800CB609949934A00F8963C0C46927981F82D
:10F158005E3023203D2381F8643081F86120F3F785
:10F168005DFD924BA069636102232374002800F0BF
:10F17800B3831C2200238271C3710D21F4F744F973
:10F18800894B1C469869F4F7BFFA4FF4807160699F
:10F19800F8F796F9A36913B11A689B881385824B0F
:10F1A8001C4658696B21F8F73DF980216069F8F72A
:10F1B80039F9A36913B11A689B88936106237C4CBB
:10F1C800DFF8F8817B4DDFF8F89100937A4F4FF024
:10F1D800960E4FF0100C4FF47A767B68C3F3080351
:10F1E800002B40F0B180EFF31183002B40F0AC808E
:10F1F8002168AA6800BF23689942F9D1D8F80000AD
:10F2080006FB00F39A1AB2FBF0F206FB01217B68B9
:10F21800C3F30803002B77D1EFF31183002B73D1CD
:10F228002368A86800BF22689342F9D1D8F800A0E3
:10F2380006FB0AF2101AB0FBFAF006FB03035B1A8E
:10F24800B3F57A7FE3D3BEF1010EC6D1564B9B6965
:10F2580013B11A689B881385534B586940F2E933F8
:10F2680002E0002B00F090800289013B12F0020FAF
:10F278009BB2F6D0F523037340F2E93302E0002B8A
:10F2880000F082800289013B12F0010F9BB2F6D098
:10F29800037B454B5869838940F2E93301E0002B31
:10F2A8006FD00289013B12F0020F9BB2F7D0FF2307
:10F2B800037340F2E93301E0002B62D00289013B7D
:10F2C80012F0010F9BB2F7D0037BDBB29B46364BA3
:10F2D800986910B1036882889A615B46682B71D07F
:10F2E800009B013B13F0FF0300937FF46FAF2E4B9D
:10F2F80093F85C30032B18BF002000F0848005B021
:10F30800BDEC028BBDE8F08FEFF311808CF312880F
:10F31800D5F808A02B68DB0304D50123C9F8003011
:10F32800D5F808A02368D9F80020C0B280F3118866
:10F33800D8F80000134406FB00F2A2EB0A02B2FB65
:10F34800F0F206FB03237AE7EFF311828CF31288BD
:10F35800A8682B68D90303D50123C9F80030A86829
:10F368002368D9F80010D2B282F31188D8F80020A7
:10F37800194406FB02F31B1AB3FBF2F306FB013137
:10F3880045E7F4F791FBA2E7F4F78EFB81E700234A
:10F39800CEE600BFA067002020340020603D00209A
:10F3A80048800800C0670020D06700200030014076
:10F3B8005860002010E000E000ED00E0BC60002094
:10F3C800B8600020F4F79AF9AE4B1C468C215869B6
:10F3D800F8F728F801230DF10F0200216069F8F70A
:10F3E8003FF8A069F4F790F99DF80F30142BFFF45B
:10F3F8007EAF182B03D9543B062B3FF678AFA14AB2
:10F40800032382F85C30A0499E4C0B689F4DA04AAC
:10F41800E26143F001030B60EA789E4B9E4863600B
:10F4280003210023206084F85E10EB71002A40F06D
:10F43800498294499FED997A032381F85F30934B71
:10F448009B78904807EE903AF8EEE77A013B67EE32
:10F45800877A80F86330FCEEE77A914B80F8622077
:10F46800C3ED007A0446F4F73BFB884B1B780BB1DD
:10F4780084F85E3022F000FC019E8A4A884B46F8E8
:10F48800802C1C68884BB3FBF4F34FF47A7102F1BB
:10F4980028059BB2A832B3FBF1F34FF4FA7146F892
:10F4A800943C102346F8742C26F8901C7F4A06F8E2
:10F4B8008E3C202126F8883C142326F87C3C46F80C
:10F4C8008C2C26F8781C80220021794846F8845C28
:10F4D80026F002F880220021764825F0FDFF002161
:10F4E8008022754825F0F8FF74499FED755ADFEDC5
:10F4F800755ADFED753A9FED752ADFED752A9FED98
:10F50800753A9FED751ADFED751ADFED756A002300
:10F5180006E00133F6EE007A202BE1EC017A55D0B3
:10F5280007EE903AB8EEE77A27EE057A77EE257A75
:10F53800BDEEE76A16EE102A2032402AE9D8B4EE6A
:10F54800E57AF1EE10FA40F34F819FED666A01E02B
:10F55800F0EE477AF4EEC67AF1EE10FA37EEE67A74
:10F56800F6DCB4EEE37AF1EE10FA40F13A819FED61
:10F578005E6A01E0B0EE677AB4EEC67AF1EE10FA90
:10F5880077EE267AF6D4F4EEE57AF1EE10FA40F347
:10F59800208171EEE77A27EEA76AB0EE624AA6EEFE
:10F5A800024A0133202BF0EE430AE4EE060AB7EED6
:10F5B800007A66EE674A77EE677AB6EE007AE4EE8E
:10F5C800A07A67EE877AE1EC017AA9D10C2303FBD4
:10F5D80004F306EE103AB8EE466ADFED447A9FED82
:10F5E800391A434BDFED3D3A9FED374A9FED372AF5
:10F5F800DFED372A9FED373ADFED3E6ABCEEC66A8B
:10F60800F0EE411AB8EE466A03F16C0226EE276A5C
:10F6180003F1D80EFDEEC67A36EE011A17EE905AAF
:10F62800FDEEC17A203517EE904A00212034F7EE1E
:10F63800004A0EEB0100C826402D868000F2D780D4
:10F64800B4EEE36AF1EE10FA40F34E81B0EE467A7A
:10F658009FED235ADFED235A01E0B0EE677AB4EE4E
:10F66800E57AF1EE10FA77EE457AF6DCF4EEC47A34
:10F67800F1EE10FA40F13B819FED195ADFED1A5A6D
:10F688003EE000BFD067002048430020A06700206C
:10F6980090C1793DF5460008E93A00080000FA42B1
:10F6A800C0670020585B030840420F000000F84183
:10F6B800B033002030340020B03400203035002032
:10F6C8003C8C4F3EDB0FC93FDB0F49C092E741B985
:10F6D8009730083C15A82ABEDB0FC9BFDB0F49408D
:10F6E800DB0FC940E4CB1641E4CB16C1E5A6C5390A
:10F6F800B035002000000000F304353FF0EE477AF3
:10F70800F4EEE57AF1EE10FA37EE857AF6D4B4EE37
:10F71800E17AF1EE10FA40F3BA8033EEC77A67EE79
:10F72800077AF0EE620AE7EE820A402CB0EE430A4E
:10F73800A0EEA70A27EE275A5FED115AA5EE007A28
:10F74800F0EE640AF0EE647AE7EE250AE7EE657AF1
:10F7580087EEA00A51D9B0EE667AF6EE005AB7EEF7
:10F76800005AC4EEA07A0831DFF8B8C1634F644E7E
:10F778006448C2F800C018299760D660106103F188
:10F78800240302F1240203ED050A65EEA75A25EECB
:10F79800275A67EE277A43ED095A43ED075A03EDD6
:10F7A800085A43ED067A43ED036A43ED046A43EDD4
:10F7B800016A43ED026A42ED086A42ED036A42EDCE
:10F7C800046A42ED016A42ED026A7FF432AF012019
:10F7D80095E5F4EEC17AF1EE10FA48BF73EEE77AD8
:10F7E800D9E6F0EE477ACEE6B0EE677AB9E6B7EE3C
:10F7F800000A402CF0EE400AADD8B4EEE16AF1EE12
:10F8080010FA77DDB0EE417A9FED3F5ADFED3F5AAF
:10F8180001E0B0EE677AB4EEE57AF1EE10FA77EE31
:10F82800457AF6DCF4EEC47AF1EE10FA0FD5B0EEB4
:10F83800677A9FED355ADFED365A01E0B0EE677A08
:10F84800B4EEE57AF1EE10FA77EE857AF6D4F4EEB6
:10F85800E17AF1EE10FA2BDD73EEE77A67EEA75A3C
:10F86800B0EE625AA5EE825AF0EE438AE5EE858A3A
:10F8780025EEA78AB8EE007AE8EE287AF6EE005A66
:10F8880034EEE75A27EE877A65EE255A69E7DFED09
:10F89800217AB4EEE77AF1EE10FA48BF34EE477AEF
:10F8A8003DE71D4B01931A46042302F8983C34E4C3
:10F8B8009FED187AF4EEC77AF1EE10FA48BF74EEAD
:10F8C800677ACBE7072A3FF4B4AD14499FED147A61
:10F8D80081F85F300123B4E51F20F2F70BFAA0612D
:10F8E80000283FF44AAC44E4F0EE467ABEE6B0EEB7
:10F8F800677A0CE7F0EE417A94E700BF00DFCDBEEF
:10F90800BA32BDBE0184483EDB0FC940E4CB164184
:10F91800E4CB16C1DB0FC9BF20340020D06700201C
:10F9280000007A4400DFCD3E023990ED007AD0ED38
:10F93800017AD0ED026A062913D8DFE801F0424DBA
:10F9480056616A790400B1EE676AF1EE666AF1EE13
:10F95800477A80ED006AB0EE467AC0ED017AC0EDD4
:10F96800026A384B93F8373253BB374B93EDA36A8F
:10F9780093EDA05AD3EDA65A27EE866AA5EE076A3C
:10F98800A5EEA66A80ED006A93EDA46A93EDA15AEC
:10F99800D3EDA75A27EE866AA5EE076AA5EEA66AF2
:10F9A80080ED016A93EDA55AD3EDA25A93EDA86AAA
:10F9B80067EE857AE5EE877AE6EE267AC0ED027A7A
:10F9C8007047B1EE476AC0ED007AB0EE677A80ED15
:10F9D800016AF0EE467AC4E7B1EE477AF1EE677A4B
:10F9E80080ED007AC0ED017ABBE7B1EE676A80ED81
:10F9F800017AF0EE477A80ED006AB0EE467AB0E719
:10FA0800B1EE477AF1EE666A80ED007AC0ED026ADF
:10FA1800A7E7B0EE476AF1EE666A80ED017AC0EDBD
:10FA2800007AB0EE677AC0ED026AF0EE467A98E79F
:10FA3800F1EE677AF1EE666AC0ED017AC0ED026A0E
:10FA48008FE700BF1800002020340020944B954A0F
:10FA5800596A32F8C03CA2F8A432002900F00D819E
:10FA680007EE903AB8EE676A07EE901AF8EE677AF2
:10FA78009FED8D7A9FED8D0ADFED8D2A9FED8D3AF2
:10FA88009FED8D1ADFED8D1A9FED8D2A9FED8D5A12
:10FA980026EE276AF0EE400A26EE076A2DED028B65
:10FAA800FDEEC67A36EE000A17EE900AFDEEC07A31
:10FAB80002F52A7317EE901A2030203102F54572AC
:10FAC800F7EE004A402800F2A580B4EEE26AF1EEB3
:10FAD80010FA40F3DC80B0EE467ADFED7B5ADFEDBA
:10FAE8007B6A01E0B0EE677AB4EEE67AF1EE10FADE
:10FAF80077EE657AF6DCF4EEC37AF1EE10FA40F1AF
:10FB0800BD80DFED715ADFED726A01E0F0EE477AF1
:10FB1800F4EEE67AF1EE10FA37EEA57AF6D4B4EE02
:10FB2800E07AF1EE10FA00F3A280DFED6A7AB4EE23
:10FB3800E77AF1EE10FA48BF33EE477A67EE077AB4
:10FB4800B0EE614AA7EE814A4029F0EE423AE7EE6C
:10FB5800843A67EE275ADFED606AA5EEA37AB0EE25
:10FB6800644AF0EE647AA7EE264AE7EE667AC7EEB4
:10FB7800843A55D8B4EEE06AF1EE10FA40F38A8080
:10FB8800B0EE407ADFED505ADFED506A01E0B0EE9A
:10FB9800677AB4EEE67AF1EE10FA77EE657AF6DC7B
:10FBA800F4EEC37AF1EE10FA77D5DFED475ADFEDC0
:10FBB800486A01E0F0EE477AF4EEE67AF1EE10FAE0
:10FBC80037EEA57AF6D4B4EEE07AF1EE10FA51DC0D
:10FBD800DFED407AB4EEE77AF1EE10FA48BF33EE83
:10FBE800477A67EE077AF0EE616AE7EE816AF0EE2F
:10FBF800428AE7EEA68A67EE275AB8EE008AA5EE93
:10FC0800A87AF6EE006A74EEC75A27EE087A65EE0F
:10FC1800A66A0BE0F7EE003A4029B0EE634AA9D98C
:10FC2800B0EE457AF6EE006AF7EE005AC4EE847A32
:10FC3800243343ED053A67EEA66A67EEA55A27EE28
:10FC4800877A43ED096A43ED076A43ED085A03EDE5
:10FC5800067A03ED035A03ED045A03ED015A03ED46
:10FC6800025A9A427FF42EAFBDEC028B704732EEF7
:10FC7800C77A63E732EEC77AB3E77047B0EE677AC0
:10FC8800B4EEE07AF1EE10FA7FF74FAFEFE7F0EE5F
:10FC9800467A30E7F0EE407A82E7B0EE677A92E78C
:10FCA800544300202034002027D4D236DB0FC93F2C
:10FCB800DB0F4940DB0F49C092E741B99730083C58
:10FCC80015A82ABE00000000DB0FC940E4CB16418E
:10FCD800E4CB16C1DB0FC9BFF304353FF8B5284C98
:10FCE800284D38220021204625F0F6FB264B15F832
:10FCF800BD6CB3F85C20A283103393E8070015F8B5
:10FD0800BC7C84F8207004F1080383E807001EB166
:10FD1800072E01D0012E02D0237F032B01D0002013
:10FD2800F8BD1A4A1A491368216043F002031360A8
:10FD380003214FF48073174E1148A3826660A177A0
:10FD4800F0F772FDB5F8A4324FF47A7262627BB1B3
:10FD5800114E06F16C07B5F8A432616A00EE103A4C
:10FD68003046B8EE400A2436F6F7DCF9B742F2D14D
:10FD780015F8BE3C13B1A3770120F8BD0120F8BDEA
:10FD88005443002020340020D0670020484300203E
:10FD980031080008AD470008C83600202DE9F843AF
:10FDA80088460178A9B10C4E04468146354606F1CD
:10FDB8000807284625F0A7FB38B1B842A0EB060093
:10FDC8003CBFA9EB040308F8003019F8011F00290B
:10FDD800EFD1BDE8F88300BFCC580308254B5B681A
:10FDE800C3F3080370B4B3B9EFF311839BB9224A84
:10FDF800224C1368A06800BF11688B42F9D12049D2
:10FE08000D684FF47A7404FB05F1081AB0FBF5F09D
:10FE180004FB03031FE0EFF31180102383F3128820
:10FE2800164A184995681368DB0342BF01230B6023
:10FE38009568114AC0B216680B6880F3118810499A
:10FE48000C684FF47A70334400FB04F1491BB1FB92
:10FE5800F4F100FB03130C480C491268826001247A
:10FE6800022280F8214081F81823C1F8143370BCAD
:10FE7800704700BF00ED00E05860002010E000E08F
:10FE8800BC600020B8600020943F0020203400208F
:10FE9800274B5B68C3F3080330B4B3B9EFF311839E
:10FEA8009BB9244A244C1368A06800BF11688B4290
:10FEB800F9D1224A14684FF47A7101FB04F2101A3E
:10FEC800B0FBF4F001FB030320E0EFF311811023F2
:10FED80083F3128818481A4A84680368DB0344BF0E
:10FEE80001231360134B48BF84681D681368C9B2A7
:10FEF80081F31188114A10684FF47A712B4401FB81
:10FF080000F2121BB2FBF0F201FB03230D490E486D
:10FF18008A68022403F5B71303F5587302F2DC521A
:10FF280080F81843C0F814338A6030BC704700BFAB
:10FF380000ED00E05860002010E000E0BC60002008
:10FF4800B8600020943F0020203400202DE9F04FB5
:10FF58008F4D904C904E914BB5F818C0904A9148EF
:10FF6800914FDFF88082C4F8D839DFF87C92C4F862
:10FF7800B009002385B00FFA8CF1C4F8D079C4F821
:10FF8800D48986F8193306F5467002F1240ED9F89B
:10FF9800003022F8021F03F59673964540F8043F97
:10FFA800F5D1DFF84892DFF848A2D9F800E07F4B96
:10FFB8001EF4805F08BFB5F92410AAF8061003F1F3
:10FFC800640007E08AB2597804312AF81120053311
:10FFD80098421AD01A78002AF9D193F802B0DA7840
:10FFE8009345F4D20BF1FF3101EB810101EB810163
:08FFF80001F561710132BBF15A
:020000040801F1
:10000000000FE3D102EB820202EB820202F5617281
:10001000DDE71EF0080F32D11EF4804F41D11EF0F3
:10002000010F0EF4005315D103BB1EF4004F22D173
:100030006B7D13B1022384F86E3795F8282094F86D
:10004000CC19131D8B42A8BF0B4686F8383405B077
:10005000BDE8F08F44F62062A4F8CE2993B30822BD
:10006000554B84F8CC29C4F8D039DEE744F6206338
:10007000A4F8CE39F3E7012384F86E37DDE72B7A55
:100080000C2B26D8DFE813F0BA00BA00A8019602BC
:10009000320162016201F80125006002BA00250008
:1000A0002F00122344F6206284F8CC39434BA4F885
:1000B000CE29C4F8D039424A424BC4F8D429C4F8F6
:1000C000B039ACE70C22404B84F8CC29C4F8D039C5
:1000D000ABE70820F4F73AFCD9F800E0C4F8D0798F
:1000E000C4F8D48998E70A224FEA0C13374993FBE6
:1000F000F2F3374AC4F8D029A3F5B063C4F8DC1989
:100100009BB2002221F812300132122AFAD142F6B3
:10011000F8203049304BA4F8CE09402084F8CC298F
:10012000C4F8D419C4F8D83910F0AEFF0028D0D0E4
:10013000AB7A697A90F90200284A002B0CBF0023A1
:100140000823002918BF43F001034FF0030C4FF4BC
:10015000E131CDE901C300910023402110F0D4FB2F
:10016000C4F8E80C002800F0B8801D4B1A78002A6B
:1001700040F0B9821B4A1C49116002221A70012307
:1001800094F86E2784F89837002A40F0A68003235D
:1001900084F86E37A1E000BFA47A00202823002055
:1001A0002034002035A90008B6400020A0860100B8
:1001B0002DA9000884370020C1A9000839A900082A
:1001C00049A90008400D0300B1A9000834380020F7
:1001D00071A00008B18A000899CC0008258F00089A
:1001E0003B440020D83D002089B3000831A9000815
:1001F00058600020A06B0020B8400020BC4BC4F821
:100200000C39402010F040FF824600283FF461AFD7
:100210004FF0000B84F8E9B80CF0E8FF2A7A012AC5
:1002200003460FD0C0F04B820A2A1FD1D9F8002014
:1002300012F480621CBF80F00102D2B202F001020F
:1002400084F8E9280321072284F80A1984F8102980
:1002500001214FF4006284F8E018C4F800290C2151
:1002600042F6F82284F8CC19A4F8CE29697AA1487C
:10027000A14AC4F8D4290031C4F8D00918BF01211B
:100280004AB29AF9020094F8E9C8002B40F0F581CF
:10029000BCF1000F00F02982032342F008024FF462
:1002A000E131CDE9013200910023944A402110F060
:1002B0002BFB934B18606B7D94F8CC29013BDBB290
:1002C0009A4284F8FC389CBF002384F8FC3820B1A3
:1002D00094F8E938002B40F02B82031C18BF01234F
:1002E000002B3FF4F6AED9F800E095E6082342F67D
:1002F000F821844A84F8CC394020834BA4F8CE19E5
:10030000C4F8D029C4F8D43910F0BEFE82460028C3
:100310003FF4DFAE0CF06AFF6A7A9AF902100032FD
:10032000034618BF0122002800F087814FF4E13313
:100330004FF0030C02920846CDE9003C734A0023BB
:10034000402110F0E1FA724B1860C6E7062B4FF01F
:100350000C0240F05E8184F8FE3784F8CC2900233B
:1003600084F8F427DFF8DCA184F8CC37212284F864
:10037000FD3784F8FC3784F8F32742F6F821654A04
:10038000654BA4F8CE194020C4F8D029C4F8D4395C
:1003900010F07AFE834600283FF49BAE0CF026FF57
:1003A000697A9BF902C0AB7A003118BF01214AB2C9
:1003B000002840F07781002B00F0ED8142F0080228
:1003C0000121029203460191CDF800A06046534AF4
:1003D000402110F099FA80E75149524BC4F8D039C6
:1003E0000A204FEA0C1292FBF0F201F12400A2F570
:1003F000B062C4F8DC1992B2C4F8E009002321F815
:1004000013200133122BFAD142F6F821464A84F820
:10041000CC394020A4F8CE19C4F8D42910F034FE09
:10042000824600283FF455AE0CF0E0FE6B7A95F85A
:100430000AC03E499AF90220009100280CBF012110
:100440000321002B14BF06230723BCF1000F0CBFB0
:100450004FF0000C4FF0080C43EA0C038246019168
:1004600002931046324B334A402110F04DFABAF154
:10047000000F3FF432AF66E70E234FF0000A44F658
:1004800020612D4A84F8CC3940202C4B84F874AA82
:10049000A4F8CE19C4F8D029C4F8D43910F0F4FD6A
:1004A00000283FF416AE01886B7A90F90200B3EB96
:1004B0000A0201F4825118BF0122B1F5825F00F0F7
:1004C0003B81AB7A84F87DAA002B0CBF0023082364
:1004D000012113434FF4E132CDE9011300920023CF
:1004E000174A402110F010FA031C18BF0123F7E649
:1004F000F42C0020159B0008459B00088D9F0008E8
:100500008C440020559600086D960008E19600087E
:1005100034440020159100082D91000855940008DE
:10052000EC37002071A0000885A00008A08601001B
:100530001038002065A2000861A90008D1A90008B0
:100540005DAD000890D0030098490A234FEA0C12D1
:1005500092FBF3F20023A2F5B06241F823200133AD
:10056000102BFAD141F60B21914A84F8CC39402066
:10057000904BA4F8CE19C4F8D029C4F8D43910F09F
:1005800083FD00283FF4A5AD6B7A8B4A90F90200F9
:100590000092003318BF01230322CDE9012340213B
:1005A0000023864A10F0B0F9854A031C18BF0123C6
:1005B000106095E6102342F6F821824A84F8CC397F
:1005C0004020814BA4F8CE19C4F8D029C4F8D439FE
:1005D00010F05AFD824600283FF47BAD0CF006FE79
:1005E000697A9AF902C0AB7A003118BF01214AB288
:1005F00080B3002B40F0C0804FF0030E4FF4E13287
:100600000291CDE9002E6046704A402110F07CF93D
:1006100099E6002384F8CC2984F8F42784F8CC37B1
:100620001B2284F8FD3784F8FC37052384F8F32770
:1006300084F8FE374FF4E13A9FE64FF0010E4FF495
:10064000E13C02920846CDE900CE614A402110F01B
:100650005BF942E6002B00F0828042F008024FF086
:10066000010E4FF4E13102920346CDE9001E6046CF
:10067000564A402110F048F92FE6BCF1000F3BD05C
:1006800042F008020321CDE901124FF4E133009357
:100690000023504A402110F037F94F4B18604F4B60
:1006A000186008E6002B4CD1032202910192CDF88C
:1006B00000A060464A4A402110F026F943E6022293
:1006C000032184F80A294FF4806284F81019C4F8D1
:1006D0000029072145F2F05284F8E0B884F8CC19DB
:1006E000A4F8CE29C2E500234AE595F80AC0BCF17A
:1006F000000F0DD00123D0E5AB7A8BB142F0080397
:100700004FF4E13103220293CDE900126346C0E7C2
:100710004FF0010C4FF4E132CDE901C10092C4E584
:100720004FF0030C4FF4E132CDE901C10092B0E784
:10073000012386F8C833D0E584F87DAA0321082375
:10074000C7E642F00802032302920193CDF800A00D
:1007500060460023224A402110F0D6F8F3E54FF01E
:10076000010E4FF4E1320291CDE9002E6046174AA6
:10077000402110F0C9F8B0E542F0080203214FF41F
:10078000E133CDE900310292604600230F4A402157
:1007900010F0BAF8D7E5012202910192CDF800A03D
:1007A00060460F4A402110F0AFF896E5442C002037
:1007B00069A30008A1A30008A06806006DA50008B1
:1007C0007C4400202D9700084197000811990008EB
:1007D000E19600088D9F00088C44002034440020DE
:1007E00055940008F7B50023494C4A4E8DF8033064
:1007F0006023C4F8B83F3378152B07460ED0122B70
:100800000CD0012B0CBF02258C25FCF707FB002820
:1008100007DA013DF9D1002003B0F0BD44F62065B0
:10082000F3E70A25FCF7FAFA0130F4D0013D15F0A0
:10083000FF05F7D1D4F8B42F930803EB5203C4F8A3
:10084000B83FFCF7EBFA431CE5D00028F9DC0023A5
:100850000DF1030084F8BC3FFCF734FB0028DAD02C
:100860009DF803301B2BD6D10DF10300FCF72AFBBA
:100870000028D0D0284B9DF8032093F839349A42B1
:10088000C9D10DF10500FCF71DFB9DF80530012BCA
:10089000C1D801A8FCF716FB9DF80430002BBAD094
:1008A0000DF10300FCF70EFB0028B4D09DF80330D7
:1008B0000E2BB0D10DF10300FCF704FB0028AAD0E9
:1008C0009DF8032033789A42A5D10DF10300FCF77F
:1008D000F9FA00289FD09DF80330002B9BD13D46AC
:1008E000BDF80430EA1B92B2023B9A4209DB0DF1DB
:1008F0000300FCF7E7FA94F8BC0FB0FA80F0400967
:100900008AE72846FCF7DEFA002884D00135E7E7BD
:1009100028230020C4830020203400200B4B10B576
:1009200001241C7018F060FE002018F0F7FD20462E
:1009300018F0F4FD0E2018F0F1FD204618F0EEFD41
:1009400018F034FE0248BDE810404BE7C483002095
:10095000C5830020F8B504780546002C3DD004F18D
:100960000A06002718F040FE300A18F0D7FDF0B252
:1009700018F0D4FD0E2018F0D1FD1A4B187818F09D
:10098000CDFD384618F0CAFD204618F0C7FD0020FE
:1009900018F0C4FD002018F0C1FD002018F0BEFDC5
:1009A000002018F0BBFD002018F0B8FD002018F062
:1009B000B5FD002018F0B2FD6B68187818F0AEFD98
:1009C0006B68013C013314F0FF046B60F4D118F044
:1009D000EDFD0548BDE8F84004E74FF485760127B2
:1009E000C0E700BFC4830020C583002038B505469A
:1009F000047818F0F9FD002018F090FD042018F09C
:100A00008DFD0E2018F08AFD0A4BB4FA84F4187894
:100A1000640918F083FD204618F080FD287818F04E
:100A20007DFDA02018F07AFD18F0C0FD6868BDE8D3
:100A30003840D7E6C483002038B5154B026893438D
:100A4000044622D0134B06251D7018F0CDFD002062
:100A500018F064FD052018F061FD0E2018F05EFD11
:100A6000284618F05BFD002018F058FD002018F013
:100A700055FD607818F052FDA07818F04FFD18F081
:100A800095FD0548BDE83840ACE6012038BD00BF03
:100A900000FFFF00C4830020C58300200C4B1B789F
:100AA000DB0700D570470B4A1368002BFAD04FF4D0
:100AB0007A7101FB03F39842F4D3074B1B781BB9FF
:100AC000064B99681B690B6000231360704700BFD9
:100AD000643F0020AC4A0020A04A00208C4A00203D
:100AE00010B5094C238823EA00009842208009D0E1
:100AF000064B41F20241FF2219809A700E2010F03D
:100B0000BDFB2388184610BDE04000209C5F0020FC
:100B1000024B1A785978FCF705BA00BF603B0020F9
:100B200008B51CF0B1F8024B024ADA60FEE700BFDC
:100B300000ED00E00400FA052DE9F04F2DED028BE9
:100B4000A0F10A0385B00C46ED2B00F2AB86DFE87E
:100B500013F07A03A906A906A906A906A906A906FB
:100B6000A906A906A906A906A906A906A906A9060D
:100B7000A906A906A906A906A906A906A906A906FD
:100B8000A9065C03A906A906A9067404A906A90674
:100B9000A9066804A9061F04A9062702A9061C02C3
:100BA000A9061502A906F001A906DC01A906A906F5
:100BB000A906D701D101A906BF01A906A906A70167
:100BC000A9068001A906A906A906AD01A906A906DC
:100BD000A906A9066201A9065F02A9067106E0043A
:100BE000A906A906A906A906A906A906A906B20486
:100BF000A9065705A9060305A9068205A9069F04AB
:100C0000A906A906A906A906820430062906D60562
:100C10009606A906A90625036706A9061A01FE007D
:100C2000A906A906A906A906EE00A906A9063B037E
:100C3000A906A906A90695027F021203D102A906F8
:100C4000A906A906C302A906A906A302A906A90620
:100C5000A906A906A906A906A906A906A906A9061C
:100C6000A906A906A906A906A9068204A906A90635
:100C7000A906A906A906A906A906A906A906A906FC
:100C8000A906A906A906A906A906A906A906A906EC
:100C9000A906A906A906A906A906A906A906A906DC
:100CA000A906A906A906A906A906A906A906A906CC
:100CB000A906A9061104A906A906A906A906A90656
:100CC000A906A906A906A906A906A906A906A906AC
:100CD000A906A906A906A906A906A906A906A9069C
:100CE000A906A906A906A906A906A906A906A9068C
:100CF000A906A906A906A906A906A906A906A9067C
:100D0000A906A906A906A906A906A906A906A9066B
:100D1000A906A906A906A906A906A906A9060704FF
:100D2000DD03A906A906A906A906A9068C03A849F8
:100D300052232268501C2060137011F8013F002BD1
:100D4000F7D1012005B0BDEC028BBDE8F08FA148C2
:100D500000232268056803EB4301561C6D5C266086
:100D60001570026825680A446E1C527826602A7045
:100D7000026825680A4401339278691C0A2B2160B5
:100D80002A70E6D1DDE7944D0B682A68591CD278A9
:100D900021601A702B6822689979531C2360002304
:100DA00011702A6821681A440133527A481C032BB7
:100DB00020600A70F5D123682A68591C127B2160D3
:100DC0001A7023682A68591C127821601A702368E7
:100DD0002A68591C527821601A702B682046D989DC
:100DE000F4F780FE23682A68591C127A21601A7071
:100DF00023682A68591C527921601A7023682A686E
:100E0000591C127921601A702A682368D279591CFA
:100E100021601A7095E70B68704D591C2A79216082
:100E20001A7023686A79591C21601A702988204633
:100E3000F4F758FE2368AA79591C21601A70698852
:100E40002046F4F74FFE2368EA79591C21601A7096
:100E500077E70B68624A634D1178634A581C20603B
:100E6000197011682046F4F725FE23685F4A591C63
:100E7000127A21601A7029882046F4F733FEA98877
:100E80002046F4F72FFE29892046F4F72BFE204652
:100E90000021F4F727FE20460021F4F723FE50E757
:100EA000084608225149F4F7EDFD4AE70B68002592
:100EB0005A1C0A60204629461D70F4F7FBFD29469E
:100EC0002046F4F7F7FD29462046F4F7F3FD38E70E
:100ED0000B68474A581C5178206019702368454AAE
:100EE0000021581C206019702368127A591C216057
:100EF0001A7026E70B680122991821601A7020E702
:100F000008460021F4F7D6FD1BE73B4D3B4E05F1AB
:100F1000300795F902103A4B93F906208A4203F103
:100F2000080300F0C7849E42F6D10835AF42F0D1E5
:100F300007E7344B03F15A0522685979501C2060A9
:100F4000117022681978501C20601170226859783D
:100F5000501C2060117022689978501C206011701C
:100F60002268D978501C20601170226819790633E4
:100F7000501CAB4220601170DED1E2E60B681B4AC8
:100F8000591C527D21601A70DBE61F4D05F1800669
:100F900055F8041F2046F4F78DFDAE42F8D1D0E697
:100FA0001A4D05F14006B5F880102046F4F79AFD79
:100FB000236895F88220591C21601A70236895F8DF
:100FC00083200435591CAE4221601A70EBD1B8E67B
:100FD000E05D03089043002094430020B05D0020B2
:100FE00094320020A456002028300020A47A00204B
:100FF00080330020603B002000620020807A0020C7
:10100000507A0020D4580020E43D0020E83D002024
:10101000AD4F3B78002B3FF494AEDFF8E88200251B
:101020004646236818F81520591C21601A707178FB
:1010300001EB810101EB810101F2EE212046F4F781
:1010400051FD3B780135AB4206F10206E9DC78E65A
:101050000A689E4B9E491878551C256010702268BE
:101060005878551C2560107022689B78501C2060B1
:1010700013702046C988F4F735FD62E6944D0846A2
:101080002988F4F72FFD69882046F4F72BFDA988FD
:101090002046F4F727FD54E60B688E4F591C3A782A
:1010A00021601A703B78002B3FF44BAE0025EEB266
:1010B00030460BF013FB23684278591C2160304600
:1010C0001A700BF00BFB01892046F4F70BFD3B78FF
:1010D0000135AB42EBDC34E67F4D0846298AF4F754
:1010E00001FD698A2046F4F7FDFCA98A2046F4F741
:1010F000F9FC26E6DFF810C20027FEB261460023A5
:101100002268501C206016702268501C20601370EA
:10111000226811F8010F0133551C062B2560107051
:10112000EED10137062F0CF1060CE6D16B490023F6
:101130002268501C206017702268501C20601370B9
:10114000226811F8010F0133551C0B2B256010701C
:10115000EED12368624A581C072120601970236869
:101160000021581C20601970236892F8F020591C47
:1011700021601A70E5E50B685A4A5B4910785B4AB2
:101180005D1C2560187023688978581C20601970D0
:1011900023689278591C21601A70D2E5544D084694
:1011A0002988F4F79FFC69882046F4F79BFCB5F981
:1011B0000430504AD91782FB0323C1EBA301204618
:1011C00089B2F4F78FFCBCE54B4D05F16006A988A8
:1011D0002046F4F787FCE9882046F4F783FC298948
:1011E0002046F4F77FFC2368AA7A591C21601A7004
:1011F0002368EA7A591C21601A7055F80C1B2046A6
:10120000F4F758FCB542E2D19BE53C4D05F164068C
:10121000287816F0FBFA2368027A591C21601A70AC
:1012200023686A78591C21601A702368AA78591CAF
:1012300021601A702368EA780535591CAE42216096
:101240001A70E5D17DE52E4D284623F085FD002856
:101250003FF477AD2B460544226813F8011B501C60
:101260009D4220601170F7D16BE501A8F3F7F4FF00
:1012700000283FF466ADBDF804102046F4F732FCB8
:1012800023689DF80620591C21601A7023689DF878
:101290000720591C21601A7023689DF80820591CEA
:1012A00021601A7023689DF80920591C21601A706A
:1012B00023689DF80A20591C21601A702046BDF849
:1012C0000C10F4F70FFC3CE5F42C00205833002000
:1012D000905D0020413D0020A06D0020CB3E00200D
:1012E000E83D0020A067002060330020703300201C
:1012F0004C430020676666667458002084370020DF
:101300003C330020A0380020A73E0020AC4B03F166
:10131000700522681978501C206011702268597875
:10132000501C2060117022689978501C2060117048
:101330002268D978501C2060117022681979501CDD
:101340002060117022685979501C20601170226849
:1013500099790733501CAB4220601170D9D1F0E469
:10136000984D0846E989F4F7BDFBA9892046F4F7B2
:10137000B9FBE6E40B68944A591C1278216001A875
:101380001A70F3F769FF23685A1C22601870D8E4BA
:101390008E4D0B682A7A591C21601A70A98B204641
:1013A000F4F7A0FB298B2046F4F79CFB698B2046C1
:1013B000F4F798FB2368EA7C591C21601A70A98C09
:1013C0002046F4F78FFBE98C2046F4F78BFB23686B
:1013D000AA7F591C21601A70236895F82020591C97
:1013E00021601A7095F8223003EB8303590001F550
:1013F0007A712046F4F776FB2368EA7A591C21605B
:101400001A70E9682046F4F755FB23682A7C591CBA
:1014100021601A70236895F82120591C21601A70E8
:101420008FE40B686A4A581C117820601970236891
:101430005278591C21601A7083E4664D0846298849
:10144000F4F750FBA9882046F4F74CFB2989204685
:10145000F4F748FB75E4002306461D46DFF89C813F
:10146000CDE90133994602E02B2D00F06B8229462D
:101470004046F4F7B3FFEFB201350028F4D0384608
:1014800016F014F9002840F0108209F10109EBE789
:101490000B684C4A5049D078504A5D1C2560187042
:1014A00023684979581C206019702368D278591C28
:1014B00021601A7045E44A4B1D68002D00F0CC8273
:1014C00004A9002301F80C3D2846FBF719FD284626
:1014D000FBF722FD2268434B511C216010702268EB
:1014E0001978501C2060117022685978501C2060B7
:1014F000117022689978501C2060117022689DF844
:101500000410501C2060117020469988F4F7EAFA04
:1015100017E40B68344D591C012221601A702368AE
:10152000AA78591C21601A70FCF7D4FE23682F4A50
:101530002F495E1C26601870B1F90010B2F9000046
:10154000F4F76AFD23685A1C226018702988204627
:10155000F4F7C8FAFFF7F5BB264E0B687279264DF3
:10156000591C21601A702B682046198CF4F7BAFABE
:101570002B682046D98BF4F7B5FAB1892046F4F7E9
:10158000B1FAF1892046F4F7ADFA2B682046598C60
:10159000F4F7A8FA2B682046998CF4F7A3FA318A5D
:1015A0002046F4F79FFA718A2046F4F79BFA2A68DE
:1015B000236892F82620591C21601A70FFF7C1BBDE
:1015C0001057002060330020962A0020A47A0020C3
:1015D00094320020A45600207C4900207033002063
:1015E000C83F0020D43F0020A8290020E629002081
:1015F000EC290020A067002090430020D44900205F
:101600000B68BB4EBB4AB178BB4D581C20601970AB
:1016100023681278591C21601A7023682A79591C92
:1016200021601A702368AA78591C21601A702988D1
:101630002046F4F757FAE9892046F4F753FA23686D
:10164000F279591C21601A702368EA78591C2160CC
:101650001A70FFF776BB20460021F4F743FA2046C4
:101660000021F4F73FFA20460021F4F73BFA236803
:10167000A24D00265A1C22601E7023682A68591C3D
:1016800092F82C2021601A7023682A68591C92F85D
:10169000362021601A7023682A68591C92F8372076
:1016A00021601A7023685A1C22601E7023685A1C1D
:1016B00022601E7023685A1C22601E702B68204610
:1016C000598FF4F70FFA2B682046198FF4F70AFAAE
:1016D00023682A68591C92F82E2021601A7023680A
:1016E0005A1C22601E702B682046598EF4F7FAF9B6
:1016F0002B682046998EF4F7F5F9FFF722BBDFF847
:1017000034A2DFF834B27E4E7E4F9FED7F8ADFF841
:101710002C82DFED7E8ADFF828920AF1C0050EE008
:10172000FCEEE77A17EE903A99B220460AF1180AD1
:10173000F4F7D8F955450BF1040B3FF402AB9AF8D6
:1017400011100029F1D03378DBED007A012BE7D1BD
:101750003B68DB0440F14F81F5EE407AF1EE10FA80
:1017600000F06381F4EEC87AF1EE10FA00F15D81C9
:10177000BDEEE77AF4EEE87AF1EE10FA17EE103AE1
:1017800000F27481A3F130026FF4F97303FB02F3EA
:1017900089FB03121A44D917C1EB622101F2DB5114
:1017A00089B2C2E7084610225949F4F76BF9FFF7EE
:1017B000C8BA584B9B8AB3F5006F00F23381B3F57A
:1017C000806F00F25081B3F5007FB7EE008AF6EE2D
:1017D000007A28BFB0EE678A4F4D05F10C06B5ECD4
:1017E000010A20EE080A23F02FFF81B22046F4F709
:1017F00079F9AE42F3D1494D494F05F10C06B5ECEC
:10180000010AD7ED077A80EE270A23F01DFF81B287
:101810002046F4F767F9B542F1D10021FFF734BB58
:1018200020460021F4F746F920460021F4F75AF942
:10183000FFF787BA0B683B4D01269A190A601E70A4
:1018400008F0D8FF002840F0F680374B2268511C82
:1018500021601070226841F2B410511C185C2160A4
:1018600041F27811107059582046890AF4F722F98C
:10187000A96A20464908F4F71DF9FFF762BA2B4F11
:101880003B78002B3FF45DAA294E002536F9021B58
:10189000204689B2F4F726F93B780135AB42F5DCF6
:1018A000FFF74FBA0020FFF74DBA494601A8F4F7F9
:1018B00085FDEAE523685A1C2260197029882046B4
:1018C000F4F710F92368EA78591C21601A7023682C
:1018D0002A79591C21601A702368AA79591C216041
:1018E0001A7023686A79591C21601A70FFF71DBBB2
:1018F000A067002050330020A06D002090430020FE
:10190000B66D0020A06B00200000404200E0824441
:1019100020310020544300207C430020C467002075
:10192000D06700203C620020C4850020F42C0020F9
:10193000B8400020E06C002000310020DB9B91418A
:1019400021053483584B594DB3F850102046F4F715
:10195000C9F800212046F4F7C5F8554B19684B012A
:1019600003F02002C1F340031343C1F3800243EAB2
:101970004203C1F3C00243EA8203C1F3401243EAC7
:10198000C20301F0100119432046F4F7ABF801A996
:1019900004222046F4F776F823682978454A581C33
:1019A0002060197011886429A8BF64212046F4F7CB
:1019B00099F8962E45D000212046F4F793F8216837
:1019C000B9F1190348BFA9F11203A3F3C4034A1CD8
:1019D000226020461A460B7002A9F4F753F82368D8
:1019E000354A581C12212060197020461168F4F7FE
:1019F00061F8FFF7A6B9F4EEC87AF1EE10FA17DB3A
:101A0000FDEEE77A40F2E73217EE903A303B02FB08
:101A100003F388FB0321DB17C3EB612101F2E931FA
:101A200089B282E6B4EE008AD6E640F2DC517CE66A
:101A30004FF47A7179E695F82420204B32BB30467A
:101A400004E723680322591C21601A7023686A780E
:101A5000591C21601A70B2E70B68FF22591C2160E3
:101A60001A70FFF76EB9B5EE008AB5E6A3F583628A
:101A700040F2F31303FB02F389FB03121A44D91754
:101A8000C1EB622101F2DD5189B24EE6597802299B
:101A900004D003290CBF04203046D7E6042A34BF03
:101AA00002200320D2E600BF381C0020EC97002063
:101AB0004843002072580020B83F0020C485002011
:101AC0002DE9F04F2DED028BDFF8748398F800308C
:101AD000012B8FB0064600F0C181BF4BBF4F187875
:101AE0000BF08EFB3B788342044608D0002840F080
:101AF0003881BB4D28680EF0C3FE2C603C70DFF8C7
:101B0000449399F80030012B00F05581B54BB64C49
:101B10001D6894F800B0ADB128460BF067FB88B1A2
:101B2000BBF1000F06D1B14B1B681BB1B0490122BC
:101B30000B602270AF4B1B78D3B10FB0BDEC028BA2
:101B4000BDE8F08FAC4B18780BF05AFB5845824635
:101B5000F0D0002840F09581A54D28680EF090FE49
:101B6000A44BC5F800A01B7884F800A0002BE4D19A
:101B7000A24B1B685B05E0D598F80030012B00F004
:101B80003182DFF8C4823B78002B3CD0DFF8BCB256
:101B90009B49DBF81420B21A8A4200F25582994D13
:101BA00095F800A0BAF1000F00F09182DFF8A0C212
:101BB000DCF800203AB3DBF8241040F6B730711A95
:101BC000814220D99BF82050002D00F052849BF8D0
:101BD000297083499BF828E00868013DEDB2013780
:101BE0008BF82050FFB2002D00F0388412F8011B52
:101BF0008BF829708E44CCF800208BF828E0F1F7A0
